:100000000BC500003AC5000038C5000036C5000029
:1000100034C5000032C5000030C500002EC5000008
:100020002CC500002AC5000028C5000026C5000018
:1000300024C5000022C5000020C500000C94081A49
:100040001CC500001AC5000018C5000016C5000038
:1000500014C5000012C5000010C500000C943C1827
:100060000CC500000C94D7160C94AE1606C5000003
:1000700004C5000002C5000000C50000FEC4000069
:10008000FCC40000FAC40000F8C40000F6C400007C
:100090000C9416190C9486180C94CD180C94D63127
:1000A000ECC40000EAC40000E8C40000E6C400009C
:1000B000E4C40000E2C40000E0C40000DEC40000AC
:1000C000DCC40000DAC40000D8C400000C9485161B
:1000D0000C945C16D2C40000D0C40000CEC4000052
:1000E000CCC400000B08FC07050814080B080B081B
:1000F000140805080B080B085C08430843086E0841
:100100005C086B086E086E085C085C0840093C09D6
:100110003C09430940094009430943094009400992
:100120009D0BA20BA70BB10BBB0B340CC50BCD0B5E
:10013000D50BDF0BE90BF30B020C0C0C340C160C7B
:10014000200C2A0C70147314621466146C14AA1414
:1001500077147B148114851489148F1493149714C5
:10016000AA149D14A114A514021D111DEF1C2E1D0F
:100170002E1D2E1D2E1D2E1D2E1D2E1D2E1D2E1D27
:10018000531BB31CC91CE91C3622362236223622E8
:10019000332233223A223A223A223A223A223A228D
:1001A0003A223A22332233223A223A223A223A227D
:1001B0003A2238223622DF37E237FA3711385A38F6
:1001C0006C388B3807634236B79BD8A71A39685604
:1001D00018AEBAAB558C1D3CB7CC5763BD6DEDFD69
:1001E000753EF6177231BF000000803F0800000026
:1001F000BE922449123EABAAAA2ABECDCCCC4C3E1C
:1002000000000080BEABAAAAAA3E00000000BF000A
:100210000000803F0000000000084178D3BB438706
:10022000D1133D190E3CC3BD4282AD2B3E68EC821A
:1002300076BED98FE1A93E4C80EFFFBE01C4FF7F9F
:100240003F00000000006364696E6F70737578583A
:100250005B00496E76616C6964204D41433A2073BE
:1002600065742064656661756C74000A4C617A7906
:10027000686F6D652E7275204C6967687448756289
:1002800020636F6E74726F6C6C65722076302E39DD
:100290003400496E76616C696420636F6D6D616EC8
:1002A00064003E3E2000312D7769726520636F75D2
:1002B0006E743A200020416464723A0064657623CB
:1002C0000020616C69766500204E6F64653A0053CA
:1002D0006561726368696E67004D6F646275732053
:1002E000706F6F6C696E67206572726F723D004D42
:1002F0006F646275732056616C3A20004D6F6462C2
:10030000757320706F6F6C696E67206572726F72A3
:100310003D002D002050492056616C203A004D6F61
:100320006462757320706F6F6C696E67206572729E
:100330006F723D002D0020464D2056616C203A0022
:100340002F6D79686F6D652F735F6F75742F002047
:100350002D2D00204F464600204F4E00204F464690
:100360000020636D643A002043757274656D703AC5
:1003700000205365743A0020457870697265640006
:10038000203D0020543A00204974656D3A00205603
:10039000616C3D002053746F726520003A3D003A55
:1003A000003D3E003D00564323004D6F646275736F
:1003B000206F70206661696C65640020636D643D28
:1003C000003D0056435F6865617423003D0050693D
:1003D0006E3A003D0050696E3A00573A002048617D
:1003E0006C74656400466F72636520576869746554
:1003F000003D00526573746F7265643A20003A20C4
:100400004E6F2073746F7265642076616C756573CE
:10041000202D2064656661756C7400526573746F7D
:100420007265642066726F6D3A00436D643D000032
:10043000002100240027002A002D00300033000195
:10044000010000040107010A010000220025002824
:10045000002B002E003100340002010000050108CD
:10046000010B01000020002300260029002C002F92
:100470000032000001000003010601090105050525
:1004800005070508080808020202020A0A0808040B
:100490000404040101010101010101030303030339
:1004A000030303040707070C0C0C0C0C0C0C0C02C8
:1004B00002020206060606060606060B0B0B0B0BCF
:1004C0000B0B0B01021020200808102040102040C8
:1004D0008002010201080402010102040810204008
:1004E0008080402010080402018004020180402026
:1004F000100804020108040201010204081020404F
:1005000080010204081020408000000A0B02090C40
:100510000D0E0807030401000000000000000000A9
:1005200000000000000000000000000000000000CB
:100530000000000000121110000000000000000088
:100540000000000000000000000000000000005259
:100550006562696E642073756363657373004572C9
:10056000726F723A20726562696E64206661696CAE
:100570000052656E65776564207375636365737398
:10058000004572726F723A2072656E6577656420FD
:100590006661696C002074727920616761696E2000
:1005A000696E2035207365636F6E647300666169E0
:1005B0006C65642C2072633D00636F6E6E656374BE
:1005C00065642061732000202E2E2E002075736537
:1005D000723A003A00417474656D7074696E6720F8
:1005E0004D51545420636F6E6E656374696F6E2055
:1005F000746F20004661696C656420746F20636FBE
:100600006E6669677572652045746865726E65749B
:10061000207573696E6720444843500053746172BB
:1006200074696E67206C616E00005EBCE2613FDD44
:1006300083C29C7E20A3FD1F419DC3217FFCA2405D
:100640001E5F01E3BD3E6082DC237D9FC1421CFE34
:10065000A0E1BF5D0380DE3C62BEE0025CDF81633F
:100660003D7C22C09E1D43A1FF4618FAA427799B1A
:10067000C584DA3866E5BB5907DB856739BAE40615
:10068000581947A5FB7826C49A653BD987045AB800
:10069000E6A7F91B45C6987A24F8A6441A99C725F7
:1006A0007B3A6486D85B05E7B98CD2306EEDB351E6
:1006B0000F4E10F2AC2F7193CD114FADF3702ECCC5
:1006C00092D38D6F31B2EC0E50AFF1134DCE9072CC
:1006D0002C6D33D18F0C52B0EE326C8ED0530DEFA7
:1006E000B1F0AE4C1291CF2D73CA947628ABF517AA
:1006F000490856B4EA6937D58B5709EBB536688A8D
:10070000D495CB2977F4AA4816E9B7550B88D63487
:100710006A2B7597C94A14F6A8742AC896154BA96E
:10072000F7B6E80A54D7896B355573652074686548
:1007300020636F6D6D616E64733A202768656C701D
:1007400027202D207468697320746578740A2773D4
:1007500061766527202D207361766520636F6E6654
:10076000696720696E204E5652414D0A27676574AD
:1007700027202D2067657420636F6E666967206689
:10078000726F6D207072652D636F6E66696775722A
:1007900065642055524C0A276C6F616427202D2018
:1007A0006C6F616420636F6E6669672066726F6D3F
:1007B000204E5652414D0A276B696C6C27202D2024
:1007C00074657374207761746368646F6700444D67
:1007D00058696E2042756666657220616C6C6F6345
:1007E0002065727200496E697420696E2063683AF0
:1007F0000009526573657420646F6E650009436873
:1008000065636B696E6720666F7220312D57697260
:100810006520646576696365732E2E2E004453321D
:100820003438322D3130302070726573656E74004B
:1008300020416464723A006465762300312D776943
:10084000726520006D71747420006D6F6462757341
:100850002000696E7075747320006974656D732073
:1008600000436F6E666967757265643A00444D585F
:1008700020696E20737461727465642E2043686110
:100880006E6E656C733A00444D58206F757420731A
:100890007461727465642E204368616E6E656C735A
:1008A0003A20006C6F6164206661696C6564004C7D
:1008B0006F61646564006C6F6164696E6720436F8B
:1008C0006E6669670072657175657374204D515469
:1008D0005420436F6E666967005361766564005308
:1008E0006176696E6720636F6E6669672E2E00639E
:1008F0006F756C64206E6F742070617273653A203E
:100900000055706461746564006F6E006F66660008
:10091000485454502F312E3120256900204854541A
:10092000502F312E310D0A486F73743A2025730D04
:100930000A4163636570743A202A2F2A0D0A436FB7
:100940006E6E656374696F6E3A20636C6F73650DCC
:100950000A0025730020000D0A004745540020744A
:10096000727920616761696E20696E203520736538
:10097000636F6E6473006661696C656420746F20D8
:10098000636F6E6E656374004552524F523A205346
:1009900065727665722072657475726E656420008A
:1009A000436F6E6669672070617273696E67206657
:1009B00061696C656400676F7420436F6E66696778
:1009C00000436F6E666967205552493A20002D3EFC
:1009D000004F4F4D21005B002E004D7920495020E3
:1009E000616464726573733A20003A004D79206D3A
:1009F000616320616464726573733A20002F6D79BE
:100A0000686F6D652F735F6F75742F004E6F742064
:100A100066696E640000125811241FBECFEFD1E248
:100A2000DEBFCDBF00E00CBF15E0A0E0B2E0EEE11C
:100A3000FEEC00E00BBF02C007900D92AE30B10794
:100A4000D9F72BE0AEE0B5E001C01D92A039B207A6
:100A5000E1F715E0CCE0D5E000E006C02197010900
:100A6000802FFE010E94BB65CB30D10780E00807D4
:100A7000A9F70E94E54D0C940D67C2CAEF92FF9250
:100A80000F931F93CF93DF937B018901C0E0D0E0E8
:100A9000CE15DF0559F0CC33D10541F0F801619155
:100AA0008F012196CE010E94F11AF2CFDF91CF91F2
:100AB0001F910F91FF90EF900895CF92DF92EF92E8
:100AC000FF920F931F93CF93DF93E091EA07F0918A
:100AD000EB07309791F09085953079F469017A01B0
:100AE000EB01682FCF010E9471429601A701BE0160
:100AF000FC01818592850E941E49DF91CF911F9153
:100B00000F91FF90EF90DF90CF900895AF92BF923A
:100B1000CF92DF92EF92FF920F931F93CF93DF93C9
:100B2000E1E0F0E0C0E0D0E0CC24C394D12C4091CF
:100B30008C0550918D05B6010C2E02C0660F771FF3
:100B40000A94E2F77F0184E0E80EF11CCF01B12C9A
:100B50009C01A0910402B0910502A817B90720F4E6
:100B60002091040230910502A0919E05B0919F054D
:100B7000A20FB31FAC90A091E607B091E7079C01CC
:100B800021503109A20FB31F0A2D10E02C9130E043
:100B90000217130729F0462B572BAC92BB24B394B2
:100BA00001968E159F05A1F650938D0540938C05F7
:100BB000BB2009F18091E6079091E707E80FF91F44
:100BC000028110E0218130E0408150E03197608166
:100BD00070E0CE0172DF0E943018DC01CB01845D31
:100BE0009E4FAF4FBF4F8093880590938905A09388
:100BF0008A05B0938B052196F701C430D10509F021
:100C000096CFDF91CF911F910F91FF90EF90DF90E2
:100C1000CF90BF90AF900895DC011296ED91FC91BA
:100C20001397309721F081E09085953009F080E0AE
:100C30000895CF92DF92EF92FF92CF93DF93DC0182
:100C40001696ED91FC911797309721F1208522306F
:100C500009F56A017B01EC0164E973E08CE898E036
:100C60000E9402156EE873E08CE898E00E9402157D
:100C70002AE030E0B701A6018CE898E00E948315D5
:100C80008CE898E00E941316EE81FF81C186D2861F
:100C9000E386F486DF91CF91FF90EF90DF90CF90C5
:100CA0000895FC0186819781009789F0FC012085D9
:100CB000223041F0253079F460E00E9471420097C3
:100CC00079F0FC01618572858385948508956FEFC5
:100CD0007FEFCB0108956EEF7FEF8FEF9FEF0895C9
:100CE0006DEF7FEF8FEF9FEF0895FC018481958179
:100CF000009761F0FC012085223029F0253049F46D
:100D00000E947142FC018185928508958FEF9FEFCB
:100D100008958EEF9FEF0895CF93C62F63E0FC01F7
:100D2000828193810E947142009749F04C2F50E0DC
:100D300060E070E0FC014187528763877487CF9140
:100D4000089563E0FC01828193810E9471420097C3
:100D500019F0FC01818508958FEF08958F929F927D
:100D6000BF92CF92DF92EF92FF920F931F93CF9398
:100D7000DF93EC0151DF882309F47EC08A819B81D7
:100D80000E941C23082F10E06801CC0CDD1CE12C14
:100D9000F12C92E0B92E0430110504F5F701EC0DA9
:100DA000FD1DEC5DFD4F808091800E94BD1000977D
:100DB00051F0FC01B086A401990C660B770B4187BA
:100DC000528763877487BC018A819B810E94BC42E1
:100DD0000F5F1F4FF2E0EF0EF11CDDCF0A811B8188
:100DE00060E0C8010E947142FC018185888761E052
:100DF000C8010E9471429D838C8362E0C8010E94F9
:100E000071429F838E8367E873E08CE898E00E94CC
:100E10000215EA81FB81608171818CE898E00E9473
:100E20004B1663E873E08CE898E00E940215488551
:100E300050E060E070E02AE08CE898E00E943B150A
:100E400060E873E08CE898E00E94021560E070E0D2
:100E5000CE014BDF4AE050E0BC018CE898E0DF9126
:100E6000CF911F910F91FF90EF90DF90CF90BF90A7
:100E70009F908F900C941616DF91CF911F910F9138
:100E8000FF90EF90DF90CF90BF909F908F9008954C
:100E9000CF93DF93EC0182E292E09983888361151E
:100EA000710549F080912E0590912F050E947E4298
:100EB0009B838A8302C01B821A82CE01DF91CF916D
:100EC0004DCF3F924F925F926F927F928F929F92FF
:100ED000AF92BF92CF92DF92EF92FF920F931F9348
:100EE000CF93DF93CDB7DEB761970FB6F894DEBF2F
:100EF0000FBECDBF6C015B012A017901302E6AE281
:100F000074E08CE898E00E9402154AE050E0B501D8
:100F10008CE898E00E9416161B861A861D861C8691
:100F20001F861E86E114F10421F47E012AE0E20E00
:100F3000F11C60E070E0C601D8DE8C0133E0A3163E
:100F4000B104C1F084E0A816B10481F5C601F9DE50
:100F5000823009F47BC038F4882309F477C08130EB
:100F600009F450C1C2C1853009F470C0893009F458
:100F700049C1BBC1D60118968C91873009F4B5C11F
:100F8000C601DFDE853079F46BE174E08CE898E02F
:100F90000E9402154AE050E065E070E08CE898E0BD
:100FA0000E94161653C08DEF9FEF56C6B1E0AB16E8
:100FB000B10409F44BC024F4A114B10461F095C14B
:100FC000F2E0AF16B10409F41DC125E0A216B10488
:100FD00009F431C18AC169E0C6019EDED6011896C6
:100FE0008C9190E08A309105F8F4FC018827EE5846
:100FF000FF4F8F4F0C94BB65F70182819381892B42
:1010000021F48FE7D60118968C93F7014081518126
:101010006281748107C0D7014D915C91052E000C4F
:10102000660B770BC60105DE0E9430186093800BBB
:101030007093810B8093820B9093830BF6018281D6
:10104000938190938F0580938E054FC1C60179DE01
:10105000813009F49FC0C60124DEAB01BC01141627
:101060001506160617060CF043C0D60118968C918B
:1010700090E08A30910590F5FC018827E458FF4FF5
:101080008F4F0C94BB65F70140835183862F660F09
:10109000990B93838283872F770F990B9583848392
:1010A000970143E050E060E070E0C6010E94904983
:1010B00063E0A62EB12C43C0D7014D935C939701FA
:1010C00041E050E060E070E0C6010E949049AA242F
:1010D000A394B12C34C0F7015183408320E030E069
:1010E00040E050E061E070E0C6010E94904925C0F8
:1010F0002AE030E08CE898E00E9483156EEF73E000
:101100008CE898E00E943B16D60118968C918830A6
:1011100031F484E190E0F701918380830EC084E68E
:1011200090E0D70111969C938E9313961C921E9279
:10113000129715969C938E931497A12CB12C47016E
:10114000612C712C6A147B0409F163EF73E08CE865
:1011500098E00E9402154AE050E0B3018CE898E064
:101160000E94CA1561EF73E08CE898E00E940215B6
:10117000F401619171914F014AE050E08CE898E0F0
:101180000E941616FFEF6F1A7F0ADCCF61E0C601DE
:10119000C3DD28C0D60118968C91813019F565EE13
:1011A00073E08CE898E00E943B168FE7F601808799
:1011B000D70113961C921E92129784E690E0159622
:1011C0009C938E9314974C9111965C9160E074E619
:1011D000C6012FDD970143E050E060E070E0C601FA
:1011E0000E949049F6018085813009F077C0D701CF
:1011F00012968D919C911397892B09F06FC08FE700
:1012000080876CC0C6019DDD853009F46BC0F70195
:1012100011821082138212821582148262E0C6014A
:101220007BDD20E030E040E050E062E070E0C601AD
:101230000E94904957C0C601EFDC882309F455C0CD
:10124000C6017FDD823009F450C0853009F44DC0FD
:10125000813051F1C60125DD362F272FD601189692
:101260004C9150E04A30510570F4FA018827EA5752
:10127000FF4F8F4F0C94BB65892E990F990805C0BD
:10128000832E922E02C0812C912C6CE973E08CE8A5
:1012900098E00E9402154AE050E0B4018CE898E022
:1012A0000E941616892809F1F70111821082138213
:1012B00012821582148265E0C6012EDD20E030E046
:1012C00040E050E062E070E0C6010E9490496DEDA0
:1012D00073E08CE898E00E943B1607C0AA24A39410
:1012E000B12C03C032E0A32EB12CD60118968C91FC
:1012F000843009F461C158F4813009F448C0B8F170
:10130000823009F479C0833009F4B0C1F6C3883063
:1013100009F44CC338F4863009F481C1873009F4EC
:101320005CC1EBC3893009F4C4C28F3709F0E5C34F
:1013300060E0C8010E94F11A60E0C80101960E94B5
:10134000F11A60E0C80102960E94F11AF701A48127
:10135000B5812FEF30E00E94CA6524E630E040E01E
:1013600050E00E94ED61622FC801039622C1F7018F
:10137000A081B1812FEF30E00E94CA6524E630E001
:1013800040E050E00E94ED61622FC80112C1D70118
:1013900012962D913C91139784E690E0821B930B5B
:1013A00014962D913C911597829FD001839FB00D8B
:1013B000929FB00D11242FEF30E00E94CA6520E10A
:1013C00037E240E050E00E94ED61622FC8010396D1
:1013D000288B398B0E94F11A6AED73E08CE898E053
:1013E0000E9402154AE050E02889622F3989732F44
:1013F0008CE898E00E941616F701A481B5812FEFC2
:1014000030E00E94CA6524E6422E512C612C712CDA
:10141000A30192010E94ED61C22EA22EF701A281CA
:10142000B3812FEF30E00E94CA65A30192010E94B0
:10143000ED61D22EB22EF701A081B1812FEF30E005
:101440000E94CA652DE631E040E050E00E94ED6167
:10145000522F422F4F71440F440F842F880F45E5C0
:10146000682F649F060E60E0611D1124922F907416
:10147000207257FD21C091110BC0211104C0862F8D
:101480008095562F11C055E5560F40E06BEA33C0EA
:1014900021110DC0482F5AEA459F040E40E0411D1E
:1014A00011248BEA841B560F682F40E024C080E093
:1014B000562F5095462F0EC0911111C021110CC00E
:1014C000482F2AEA429F040E40E0411D11245BEAA6
:1014D000541B4B5A60E00FC0462F40950BC02111A2
:1014E00004C085E5860F4BEA03C08AEA860F90E0C8
:1014F000461B682F50E0FFEFBF1609F426C0BB2043
:1015000009F1662329F02D2D629F060E60E0611D12
:10151000552329F03D2D539F050E50E0511D4423C6
:1015200029F02D2D429F040E40E0411D1124D0943E
:101530002D2D229F020E20E0211D1124620F520F3B
:10154000420F03C04FEF5FEF6FEF3FEFA31609F4B9
:1015500021C020E03C2D332321F0339F212D09F0C1
:101560002F5F2223A1F0662321F0629F060E60E028
:10157000611D552321F0529F050E50E0511D44235B
:1015800021F0429F040E40E0411D112403C040E0C1
:1015900050E060E0C801498B588B0E94F11A5889CD
:1015A000652FC80101960E94F11A4989642FC8016C
:1015B00002960E94F11AA1C2D60114960D911C91B7
:1015C0001597F8018085853009F097C2C8010E94FF
:1015D0001C23833009F091C2FEC1D6011496ED910F
:1015E000FC9115978085853009F087C2C680D78029
:1015F000C114D10409F481C2F60161857285CE015E
:10160000019646DC032D9701A201B501CE0101969A
:1016100058DCD6011296CD90DC901397E9CFE02EDE
:1016200061E0802F0E94BC17FF24F394AA94AB289A
:1016300009F0F12C6F2D8E2D0E948D1765ED73E052
:101640008CE898E00E9402154AE050E0B8018CE86E
:1016500098E00E94CA1563ED73E08CE898E00E9460
:1016600002156F2D70E04AE050E01EC117FF07C061
:10167000119501951109AA24A394B12C02C0A12CA3
:10168000B12CD02E61E0802F0E94BC178091A10068
:10169000887F8093A10080919100887F8093910042
:1016A0008091A10082608093A1008091910082606E
:1016B00080939100F701A081B181AB2899F0CD0111
:1016C000BB0FAA0BBB0B9C01AD012456310941098C
:1016D0005109AFEFB0E00E9409622CE93FEF4FEFF4
:1016E0005FEF08C02FEF30E00E94CA6524E630E0CB
:1016F00040E050E00E94ED61790161E08D2D0E9493
:10170000BC17E114F10409F4B3C0FFEFEF16F104C4
:1017100009F4B0C0F801FF27E75FFA4FE4914E2FBC
:1017200050E0FA013197E231F10508F09DC08827B9
:10173000E057FF4F8F4F0C94BB6584B5806884BD24
:10174000E7BC9CC084B5806284BDE8BC97C0809132
:101750008000806880938000F0928900E092880089
:101760008DC080918000806280938000F0928B0019
:10177000E0928A0083C0809180008860809380001E
:10178000F0928D00E0928C0079C08091B00080686A
:101790008093B000E092B30071C08091B00080628D
:1017A0008093B000E092B40069C08091900080689E
:1017B00080939000F0929900E09298005FC0809131
:1017C0009000806280939000F0929B00E0929A00DB
:1017D00055C080919000886080939000F0929D00A9
:1017E000E0929C004BC08091A00080688093A00094
:1017F0008091A0008F7B8093A000F092A900E092DE
:10180000A8003CC08091A00080628093A000F0926C
:10181000AB00E092AA0032C08091A0008860809363
:10182000A000F092AD00E092AC0028C080912001B1
:10183000806880932001F0922901E09228011EC067
:1018400080912001806280932001F0922B01E09230
:101850002A0114C080912001886080932001F092B9
:101860002D01E0922C010AC020E8E216F10414F4E4
:1018700060E001C061E08D2D0E948D176EEC73E079
:101880008CE898E00E9402154AE050E0B8018CE82C
:1018900098E00E94CA156CEC73E08CE898E00E9416
:1018A00002154AE050E0B7018CE898E00E94161655
:1018B00024C1D7011C9160E070E0C60116DA082F40
:1018C000F92E66EA73E08CE898E00E9402154AE07F
:1018D00050E0602F7F2D8CE898E00E94CA1564EAE2
:1018E00073E08CE898E00E940215612F012E000C35
:1018F000770B4AE050E08CE898E00E941616809141
:10190000280590912905892B09F094C081E090E089
:10191000909329058093280526E040E855E260E091
:1019200070E08FEE97E00E9400170093E2098FEEBF
:1019300097E09093E1098093E0091092ED0A1092EC
:10194000EF0A1092EE0A80ED97E09093680A809378
:10195000670A10926A0A1092690A112339F085E029
:1019600090E090936C0A80936B0A04C010926C0A0A
:1019700010926B0A86E00E944B2062E370E080E0E8
:1019800090E00E94F81782ED97E09093680A8093A8
:10199000670A10926A0A1092690AB4E61B02C00133
:1019A000112490936C0A80936B0AA0C0D601149600
:1019B000ED91FC91159761857285CE01019668DAEB
:1019C000CE01019629D9882309F497C089858930E9
:1019D00009F093C097C060E0C8010E947142FC0109
:1019E0005184752C628461E0C8010E947142DC015F
:1019F00019968D909D90AD90BC901C9762E0C801A7
:101A00000E947142FC0101851285F701A081B1811C
:101A10002FE330E00E94CA6524E630E040E050E069
:101A20000E94ED6169017A01809128059091290554
:101A3000892B39F06AEA73E08CE898E00E943B1643
:101A40005CC081E090E0909329058093280526E210
:101A500040E855E260E070E08FEE97E00E940017EA
:101A60005092E2098FEE97E09093E1098093E009AC
:101A70001092ED0A1092EF0A1092EE0A012B09F46F
:101A80003DC0DC2CCC24CC24CA944AE050E0672D25
:101A9000762D8CE898E00E94CA1561EA73E08CE824
:101AA00098E0B0D7B501A4016627772720E18CE83C
:101AB00098E0E1D76FE973E08CE898E0A3D7A6013E
:101AC00060E070E020E18CE898E0D5D78CE898E001
:101AD0000E9413169092680A8092670A10926A0A0E
:101AE0001092690AD0926C0AC0926B0A86E00E943A
:101AF0004B201092290510922805AEC0DD24DD246C
:101B0000DA94C3CF0A2DD7011C9160E070E0CE01BA
:101B10000196EBD8F82EE92E63EC73E08CE898E0A0
:101B200071D74AE050E06F2D7E2D8CE898E00E943E
:101B3000CA1561EC73E08CE898E064D7612F012E40
:101B4000000C770B4AE050E08CE898E00E94CA1540
:101B50006BEB73E08CE898E055D76A2DAA0C770BF5
:101B60004AE050E08CE898E00E9416168091280523
:101B700090912905892B09F05DCF81E090E0909349
:101B800029058093280526E040E855E260E070E0F2
:101B90008FEE97E00E940017F092E2098FEE97E037
:101BA0009093E1098093E0091092ED0A1092EF0AF8
:101BB0001092EE0A0230A9F1053099F1612F110F50
:101BC000770B880B990B0E942C6322E538EB42E1DE
:101BD00052E40E94296220E030E040E251E40E9499
:101BE000E0632DEE3EE94CE35EE30E9491626B01FF
:101BF0007C0120E030E0A9010E94DC6320E030E0BD
:101C000040E05FE387FD05C0C701B6010E9429627D
:101C100004C0C701B6010E9428620E94F9628B01CC
:101C200002C000E010E0A80160E070E02AE08CE86B
:101C300098E021D78CE898E0F6D783ED97E0909371
:101C4000680A8093670A10926A0A1092690A1093D0
:101C50006C0A00936B0A4ACF61960FB6F894DEBF08
:101C60000FBECDBFDF91CF911F910F91FF90EF90ED
:101C7000DF90CF90BF90AF909F908F907F906F90AC
:101C80005F904F903F900895CF93DF93EC016DEEFE
:101C900073E00E943766892B41F160EF73E0CE015B
:101CA0000E943766892B21F164EF73E0CE010E9418
:101CB0003766892B01F169EF73E0CE010E94376628
:101CC000892BE1F060E074E0CE010E943766892B39
:101CD000C1F088818D32C1F090ED980F9A30A0F05C
:101CE0008B37A9F48EEF9FEF14C081E090E011C014
:101CF00082E090E00EC083E090E00BC084E090E0D2
:101D000008C085E090E005C080E090E002C08FEF61
:101D10009FEFDF91CF910895EF92FF920F931F9362
:101D2000CF93DF9380918C0590918D05C4E0D0E036
:101D300021E030E0A90148235923452B29F0A901CE
:101D40004095509584239523220F331F219791F7B7
:101D500090938D0580938C050E9430180091880522
:101D60001091890520918A0530918B0560177107C4
:101D70008207930708F458C0012B022B032B09F4A8
:101D800053C0109288051092890510928A0510920E
:101D90008B05E12CF12CE091E607F091E707EC0FC1
:101DA000FD1F038110E0228130E0418150E060811D
:101DB00070E0C7010E945D058FEFE81AF80A2496CB
:101DC00084E0E816F10439F7C1E0D0E08091040224
:101DD000909105028C179D0728F480910402909140
:101DE000050201C0CE0120919E0530919F05F901A9
:101DF000E80FF91F408150E060E070E02AE08CE8D5
:101E000098E039D665E074E08CE898E044D72196F4
:101E1000C131D105D9F68CE898E0DF91CF911F91BF
:101E20000F91FF90EF90FFC6DF91CF911F910F911F
:101E3000FF90EF900895FC01A285B3851097A9F05B
:101E400086859785029788F0CD01019693878287D2
:101E50006C93868597850197978786870284F3859B
:101E6000E02D108281E090E0089580E090E00895F8
:101E7000FC01868197818F3F2FEF920729F02FEF8A
:101E80003FEF378326830895A085B185109789F0A9
:101E9000248535852115310561F0CD0101969187A5
:101EA00080878C912150310935872487082E000CBA
:101EB000990B0895FC0186819781019639F481E0A0
:101EC00024853585232B19F480E0089581E0089559
:101ED000CF92DF92EF92FF920F931F93CF93DF93F6
:101EE0007C016A018B01C0E0D0E0CC15DD0589F0F2
:101EF000D701ED91FC910284F385E02DC70119957E
:101F00008F3FBFEF9B0729F0F80181938F01219646
:101F1000ECCFCE01DF91CF911F910F91FF90EF9009
:101F2000DF90CF900895CF93DF931F92CDB7DEB7A8
:101F3000DC01ED91FC910088F189E02D6983199510
:101F4000DC01ED91FC910190F081E02D69810F9011
:101F5000DF91CF911994CF93DF93FC0126813781D4
:101F60002F3F3F4FF9F4EC01288539858A859B8501
:101F7000820F931F8115904198F4E881F9810284C2
:101F8000F385E02DCE011995813291056CF3E8813E
:101F9000F9810684F785E02D682FCE01199502C0DE
:101FA00080E001C081E0DF91CF910895062E000C02
:101FB000770BFC01778366830895CF93DF93DC0171
:101FC00016962D913C9117972F3F3F4F31F5EC011D
:101FD000E881F9810088F189E02DCE011995DC01B5
:101FE000ED91FC910084F185E02D1995892B99F0F4
:101FF000E881F9810284F385E02DCE0119958132C3
:10200000910534F3E881F9810684F785E02D682F86
:10201000CE01199502C080E001C081E0DF91CF912F
:102020000895FC018481958108950895FC0122851D
:10203000338580859185820F931F811540E1940738
:1020400048F02F5F3F4F338722870E94BD6181E0B8
:1020500090E0089580E090E00895FC0186819781EA
:102060008F3F2FEF920729F02FEF3FEF3783268323
:1020700008952085318582859385AC014F5F5F4F40
:1020800053874287820F931F0E94B561082E000C70
:10209000990B0895FC01868197818F3F2FEF92075E
:1020A00029F02FEF3FEF37832683089580859185B0
:1020B0000C94965BCF92DF92EF92FF92CF93DF93D7
:1020C000EC018E819F818F3F2FEF920759F02FEF08
:1020D0003FEF3F832E83DF91CF91FF90EF90DF9012
:1020E000CF900895BDD76B017C01A4EFCA0EA1E08B
:1020F000DA1EE11CF11CE881F9810088F189E02DEC
:10210000CE011995DC01ED91FC910084F185E02D63
:102110001995892B31F4A4D76C157D058E059F0583
:1021200050F3E881F9810088F189E02DCE011995FD
:10213000DC01ED91FC910284F385E02DDF91CF91DC
:10214000FF90EF90DF90CF9019941F93CF93DF9380
:10215000182F66E270E00E948C28C82FD0E067E25A
:1021600070E0812F0E948C28DC2FCC279E01282B29
:10217000C901DF91CF911F9108958DE090E00E94F9
:102180005659009729F02DE0FC0111922A95E9F7A4
:1021900008952C9A08952C9808951F93CF93DF9358
:1021A000182F60E270E00E948C28C82FD0E061E216
:1021B00070E0812F0E948C28DC2FCC279E01282BD9
:1021C000C901DF91CF911F9108958EBD00000DB41C
:1021D00007FEFDCF8EB50895CF92DF92EF92FF926A
:1021E0000F931F93CF93DF93EC017A018B016C0166
:1021F000C40ED51ECC15DD0579F0CDDF8FE0E5DF0F
:102200008D2FE3DF8C2FE1DF219680E0DEDFF80108
:1022100081938F01BEDFEECFC701DF91CF911F9178
:102220000F91FF90EF90DF90CF900895CF92DF92C3
:10223000EF92FF920F931F93CF93DF93EC017A01FC
:102240008B016C01C40ED51ECC15DD0571F0A3DF2A
:1022500080EFBBDF8D2FB9DF8C2FB7DF2196F80120
:1022600081918F01B2DF95DFEFCFC701DF91CF9171
:102270001F910F91FF90EF90DF90CF9008951F93E3
:10228000CF93DF931F921F92CDB7DEB7182F6A83CB
:10229000998381DF80EF99DF9981892F96DF812FE4
:1022A00094DF6A81862F91DF74DF81E00F900F90B9
:1022B000DF91CF911F9108951F93CF93DF931F92CA
:1022C0001F92CDB7DEB7182F80E590E069837A833F
:1022D0000E946F4321E041E050E069817A81812FC3
:1022E0000E9401250E946E4381E090E00F900F90C4
:1022F000DF91CF911F910895CF93DF931F92CDB7B8
:10230000DEB7FC01218D328D232B41F0BE016F5FC2
:102310007F4F808DD1DF898190E002C08FEF9FEFEA
:102320000F90DF91CF910895FF920F931F93CF935A
:10233000DF93F82E80E590E00E946F43C0E0D0E08C
:102340008F2D03DF8C01892B19F08F2DFEDEEC0120
:10235000C017D107A9F70E946E43CE01DF91CF913C
:102360001F910F91FF900895AF92BF92CF92DF928D
:10237000EF92FF921F93CF93DF93182F5B017A01A7
:1023800080E590E00E946F43C0E0D0E0812FDDDE69
:102390006C01892B19F0812FD8DEEC01CC15DD05FD
:1023A000A9F7209799F463E070E0812F0E948C28B0
:1023B0008431F1F08823E1F0C1E0D0E08C3111F4F8
:1023C000C0E0D0E0D195C195D10912C0EC16FD0650
:1023D0000CF4E7011C161D065CF420E0AE01B5010B
:1023E000812F0E94012560E470E0812F0E94F32478
:1023F0000E946E43CE01DF91CF911F91FF90EF902D
:10240000DF90CF90BF90AF900895CF93DF93FC0102
:10241000218D328D2115310519F48FEF9FEF10C0FA
:10242000EC014217530708F0A901888D9DDF1816AB
:1024300019069CF7298D3A8D281B390B3A8F298F65
:10244000DF91CF910895CF93C82F80E590E00E944F
:102450006F4360E170E08C2F0E94F3244FEF62E045
:1024600070E08C2F0E948228CF910C946E43FF92D3
:102470000F931F93CF93DF931F921F92CDB7DEB7B9
:10248000F82E8A012A836983DEDF80E590E00E94CE
:102490006F432A816981462F422B60E070E08F2DC7
:1024A0000E9482280115110551F4009190051091A8
:1024B00091050F5F1F4F1093910500939005412FD9
:1024C00064E070E08F2D0E948228402F65E070E06C
:1024D0008F2D0E94822861E070E08F2D0E94F324EE
:1024E0000E946E4381E00F900F90DF91CF911F917A
:1024F0000F91FF900895BF92CF92DF92EF92FF92DB
:102500000F931F93CF93DF9300D000D0CDB7DEB7EA
:10251000FC01208D243009F050C06A017B018C0140
:10252000B12C63E070E08B2D0E948C28811103C0D8
:10253000F801B08E06C08831D9F3B394F4E0BF122D
:10254000F0CFF801808D8430C1F196E0ECE2F2E04A
:10255000DE01119601900D929A95E1F7F7019381B2
:102560009F779C8394819D8395819E83B7016E5F45
:102570007F4F90E0982F882744E050E0845F9B4F86
:1025800055DEB601F801808D0E94E528F801808DA6
:1025900090E0982F882746E050E0BE016F5F7F4FA4
:1025A0008A5F9B4F43DEF801128E118E20E8A60150
:1025B00062E0808D5CDF81E001C080E026960FB68E
:1025C000F894DEBF0FBECDBFDF91CF911F910F9169
:1025D000FF90EF90DF90CF90BF9008951F93CF931F
:1025E000DF931F92CDB7DEB7182F80E590E00E94F1
:1025F0006F4363E070E0812F0E948C2889830E94E2
:102600006E4389810F90DF91CF911F910895CF92F2
:10261000DF92EF92FF920F931F93CF93DF936C01A2
:102620007A018B01C0E0D0E0CE15DF0589F0D8013A
:102630006D918D01D601ED91FC910190F081E02D1D
:10264000C6011995892B11F47E0102C02196ECCFA9
:10265000C701DF91CF911F910F91FF90EF90DF9015
:10266000CF900895FC01A089B1898C91A689B78982
:1026700082FD0FC09C91818D8F5F8F73228D821799
:1026800049F0218DDF01A20FB11D5D969C93818FD2
:1026900008958C910895FC01538D448D252F30E0D1
:1026A000842F90E0821B930B541710F0CF9608955F
:1026B00001970895FC01918D828D981761F0828DAC
:1026C000DF01A80FB11D5D968C91928D9F5F9F7366
:1026D000928F90E008958FEF9FEF0895FC01918D08
:1026E000828D981731F0828DE80FF11D858D90E075
:1026F00008958FEF9FEF0895FC01918D228D892F12
:1027000090E0805C9F4F821B91098F7399270895F9
:102710008FEE97E0F1DF21E0892B09F420E0822F92
:1027200008958CE898E0E8DF21E0892B09F420E0A7
:10273000822F0895FC01848DDF01A80FB11DA35ADB
:10274000BF4F2C91848D90E001968F739927848FD1
:10275000A689B7892C93A089B1898C9180648C93C8
:10276000938D848D981306C00288F389E02D8081B3
:102770008F7D80830895EF92FF920F931F93CF93E5
:10278000DF93EC0181E0888F9B8D8C8D981305C0C1
:10279000E889F989808185FD23C0F62E0B8D10E034
:1027A0000F5F1F4F0F731127E02E8C8DE8120BC0A7
:1027B0000FB607FCFACFE889F989808185FFF5CF4C
:1027C000CE01B8DFF2CF8B8DFE01E80FF11DE35A89
:1027D000FF4FF0820B8FEA89FB898081806207C0FE
:1027E000EE89FF896083E889F9898081806480832C
:1027F00081E090E0DF91CF911F910F91FF90EF90DA
:102800000895CF93DF93EC01888D8823C1F0EA8986
:10281000FB89808185FD05C0A889B9898C9186FDD9
:102820000EC00FB607FCF5CF808185FFF2CFA889D7
:10283000B9898C9185FFEDCFCE017CDFE8CFDF91A8
:10284000CF91089580E090E0892B19F06ADF811123
:1028500020C080E090E0892B41F080E090E0892B5F
:1028600021F00E940000811117C080E090E0892BC8
:1028700019F04EDF811113C080E090E0892BA1F0A8
:1028800080E090E0892B81F00E94000081110AC055
:1028900008950E940000DDCF0E940000E6CF0E9454
:1028A0000000EACF0C940000089590E0FC013197FD
:1028B000E231F10508F04EC08827EE55FF4F8F4FEB
:1028C0000C94BB65809180008F7703C0809180005D
:1028D0008F7D80938000089580918000877FF9CF5D
:1028E00084B58F7702C084B58F7D84BD08958091B3
:1028F000B0008F7703C08091B0008F7D8093B000CF
:102900000895809190008F7707C0809190008F7D0F
:1029100003C080919000877F8093900008958091FC
:10292000A0008F7707C08091A0008F7D03C08091A9
:10293000A000877F8093A0000895809120018F7769
:1029400007C0809120018F7D03C080912001877F87
:102950008093200108953FB7F8948091AC05909141
:10296000AD05A091AE05B091AF0526B5A89B05C0F9
:102970002F3F19F00196A11DB11D3FBFBA2FA92FFE
:10298000982F8827820F911DA11DB11DBC01CD017B
:1029900042E0660F771F881F991F4A95D1F7089567
:1029A000CF93DF931F92CDB7DEB789832091A00527
:1029B0003981E091A105F091A205822F90E08095E8
:1029C0009095F8940080082200824BE000C05DE002
:1029D00000005A95E9F7008008220894379508F41A
:1029E000022A00824A9599F778940F90DF91CF914F
:1029F00008950E94E465DC01ED91FC910190F08165
:102A0000E02D1994EF92FF920F931F93CF93DF93D2
:102A10008C017B01C0E0D0E0F701EC0FFD1F649159
:102A2000662361F0D801ED91FC910190F081E02DD9
:102A3000C8011995892B11F02196EECFCE01DF91B7
:102A4000CF911F910F91FF90EF900895611571053F
:102A500079F0FB0101900020E9F73197AF01461BA7
:102A6000570BDC01ED91FC910280F381E02D19946C
:102A700080E090E008954F925F926F927F92EF9284
:102A8000FF920F931F93CF93DF93CDB7DEB7A1973C
:102A90000FB6F894DEBF0FBECDBF7C01FA01CB01AB
:102AA00019A2223008F42AE08E010F5D1F4F422E3A
:102AB000512C612C712CBF01A30192010E94CB61AA
:102AC000F901CA01015011096A3014F4605D01C0B6
:102AD000695CD8016C93232B242B252B61F7B8015B
:102AE000C701B4DFA1960FB6F894DEBF0FBECDBF0D
:102AF000DF91CF911F910F91FF90EF907F906F909A
:102B00005F904F900895CF92DF92EF92FF920F93D4
:102B10001F93CF93DF93EC016A017B0121153105EF
:102B200079F4E881F9810190F081E02D642FDF9143
:102B3000CF911F910F91FF90EF90DF90CF9019945C
:102B40002A303105D9F477FF18C06DE254DF8C01CB
:102B500044275527BA014C195D096E097F092AE0FF
:102B6000CE0189DF800F911FDF91CF911F910F91CF
:102B7000FF90EF90DF90CF9008952AE0B701A60173
:102B8000CE01DF91CF911F910F91FF90EF90DF90D9
:102B9000CF9071CF9A01AB01770F660B770BB3CF54
:102BA0008F929F92AF92BF92CF92DF92EF92FF925D
:102BB0000F931F93CF93DF937C018B016C0182E015
:102BC000C80ED11C4701E5E08E0E911CC0E0D0E09C
:102BD000F60141916F0150E060E070E02AE0C80129
:102BE0004ADF5C016EE2C80106DF8A0D9B1DC80F3B
:102BF000D91FC814D90461F7F701458150E060E09E
:102C000070E02AE0C80137DF8C0F9D1FDF91CF9164
:102C10001F910F91FF90EF90DF90CF90BF90AF90FA
:102C20009F908F9008956BEA73E010CF0F931F93DE
:102C3000CF93DF93EC019A01AB01770F660B770B13
:102C400062DF8C01CE01EFDF800F911FDF91CF910A
:102C50001F910F9108950F931F93CF93DF93EC0172
:102C6000F5DE8C01CE01DFDF800F911FDF91CF9168
:102C70001F910F9108950F931F93CF93DF93EC0152
:102C8000C1DE8C01CE01CFDF800F911FDF91CF918C
:102C90001F910F910895DACE21E333E0FC013183D7
:102CA0002083FB014081518162817381FC01428359
:102CB00053836483758308951F920F920FB60F920A
:102CC00011240BB60F922F933F934F935F936F9303
:102CD0007F938F939F93AF93BF93EF93FF938FEE69
:102CE00097E028DDFF91EF91BF91AF919F918F9178
:102CF0007F916F915F914F913F912F910F900BBEFC
:102D00000F900FBE0F901F9018951F920F920FB645
:102D10000F9211240BB60F922F933F934F935F9313
:102D20006F937F938F939F93AF93BF93EF93FF9393
:102D30008FEE97E097DCFF91EF91BF91AF919F915C
:102D40008F917F916F915F914F913F912F910F9054
:102D50000BBE0F900FBE0F901F9018951F920F92F1
:102D60000FB60F9211240BB60F922F933F934F93F0
:102D70005F936F937F938F939F93AF93BF93EF93E3
:102D8000FF938CE898E0D6DCFF91EF91BF91AF9173
:102D90009F918F917F916F915F914F913F912F9173
:102DA0000F900BBE0F900FBE0F901F9018951F92A3
:102DB0000F920FB60F9211240BB60F922F933F93E1
:102DC0004F935F936F937F938F939F93AF93BF9333
:102DD000EF93FF938CE898E045DCFF91EF91BF9172
:102DE000AF919F918F917F916F915F914F913F91A3
:102DF0002F910F900BBE0F900FBE0F901F90189544
:102E0000CF92DF92EF92FF921F93CF93DF93EC016B
:102E10006A017B01122FE889F98982E080834115DC
:102E2000514E61057105B1F060E079E08DE390E00D
:102E3000A70196010E94CB61DA01C9010197A1099E
:102E4000B109B695A79597958795AC01411580E195
:102E50005807A8F0E889F989108260E874E88EE1E3
:102E600090E0A70196010E94CB61BA01A9014150EF
:102E70005109610971097695679557954795EC85D4
:102E8000FD855083EE85FF854083188EEC89FD8992
:102E90001083EA89FB89808180618083EA89FB89CC
:102EA000808188608083EA89FB8980818068808353
:102EB000EA89FB8980818F7D8083DF91CF911F918B
:102EC000FF90EF90DF90CF900895CF93DF93282F5E
:102ED00030E0F901E75FFA4F8491F901ED53FB4FC0
:102EE000D491F901E358FB4FC491CC2389F08111AF
:102EF000DCDCEC2FF0E0EE0FFF1FED59FB4FA5914E
:102F0000B491EC91ED2381E090E021F480E002C0E7
:102F100080E090E0DF91CF9108951F93CF93DF93EE
:102F2000282F30E0F901E75FFA4F8491F901ED5362
:102F3000FB4FD491F901E358FB4FC491CC23C1F06E
:102F4000162F8111B2DCEC2FF0E0EE0FFF1FE75BD4
:102F5000FB4FA591B4918FB7F894111105C09C91C6
:102F6000ED2FE095E92302C0EC91ED2BEC938FBFA0
:102F7000DF91CF911F910895CF93DF9390E0FC01F3
:102F8000ED53FB4F2491FC01E358FB4F84918823C0
:102F900061F190E0880F991FFC01E15DFB4FC59145
:102FA000D491FC01E75BFB4FA591B491611109C07D
:102FB0009FB7F8948881209582238883EC912E23F3
:102FC0000BC0623061F49FB7F8943881822F8095EE
:102FD00083238883EC912E2B2C939FBF06C08FB741
:102FE000F894E8812E2B28838FBFDF91CF9108952D
:102FF0008F929F92AF92BF92CF92DF92EF92FF9209
:103000006B017C01A8DC4B015C01C114D104E1041B
:10301000F104E9F0A0DCDC01CB0188199909AA09C7
:10302000BB09883E9340A105B10578F321E0C21A9F
:10303000D108E108F10888EE880E83E0981EA11CF3
:10304000B11CC114D104E104F10421F7DECFFF90DB
:10305000EF90DF90CF90BF90AF909F908F900895AA
:103060002FB7F8946091A8057091A9058091AA05E1
:103070009091AB052FBF08951F920F920FB60F923C
:1030800011242F933F938F939F93AF93BF9380917E
:10309000A8059091A905A091AA05B091AB05309122
:1030A000A70523E0230F2D3720F40196A11DB11DA4
:1030B00005C026E8230F0296A11DB11D2093A70588
:1030C0008093A8059093A905A093AA05B093AB059A
:1030D0008091AC059091AD05A091AE05B091AF0582
:1030E0000196A11DB11D8093AC059093AD05A093F1
:1030F000AE05B093AF05BF91AF919F918F913F9176
:103100002F910F900FBE0F901F9018951F920F9246
:103110000FB60F9211240BB60F922F933F934F933C
:103120005F938F939F93EF93FF9320919E05309130
:103130009F0580919C0590919D05AC014F5F5F4F6D
:1031400050939D0540939C05F901E80FF91F80817C
:103150008093CE00809104029091050220919C05FD
:1031600030919D058217930748F48FEF9FEF90935E
:103170009D0580939C0588E48093C900FF91EF91A1
:103180009F918F915F914F913F912F910F900BBE27
:103190000F900FBE0F901F9018951F920F920FB6B1
:1031A0000F9211242F933F938F939F9320919A0511
:1031B00030919B0580919C0590919D0521303105B2
:1031C000A9F48F3F2FEF920789F41092C800109254
:1031D000CD0089E08093CC0086E28093CA001092F3
:1031E000CE0010929D0510929C0517C0892BA9F462
:1031F0001092C8001092CD0083E08093CC008EE046
:103200008093CA0088E28093C9001092CE0081E0CA
:1032100090E090939D0580939C059F918F913F91A5
:103220002F910F900FBE0F901F9018951F920F9225
:103230000FB60F9211240BB60F922F933F934F931B
:103240005F936F937F938F939F93AF93BF93EF930E
:10325000FF932091C8008091CE009091990524FFA2
:1032600008C081E08093990580919E0590919F050B
:1032700054C0913091F481110DC082E08093990582
:10328000EFDE6093240570932505809326059093C7
:1032900027053EC01092990544C0923009F041C004
:1032A000E0919705F09198059081981721F091E0B1
:1032B0009093030280832091970530919805809127
:1032C0009505909196052817390711F510929905E3
:1032D000809103028823D1F0809193059091940509
:1032E000892BA1F01092C900E0919305F09194050B
:1032F000199580E98093C9001092C8001092CD0002
:1033000083E08093CC008EE08093CA001092030289
:1033100080919705909198050196909398058093D8
:103320009705FF91EF91BF91AF919F918F917F9101
:103330006F915F914F913F912F910F900BBE0F9026
:103340000FBE0F901F9018950F931F93CF93DF938D
:10335000EC010E940B27FE01E35DFD4F918380830A
:1033600001978231924008F04BC042E152E08E0159
:10337000055E1F4FB801CE0148D8F801A2E3B2E0C4
:1033800048E04A0F21918D9130E0082E000C990BF6
:1033900028173907A9F54A13F5CF0CA110E0102F13
:1033A00000278BA1082BFE01E15DFD4F11830083F7
:1033B000011580E5180701F54FA1329640838AA5D3
:1033C00090E0982F882729A5822B319691838083BE
:1033D0006BA570E0762F66272CA5622B3296718341
:1033E000608332960190F081E02D309759F09E0174
:1033F000235D3F4F199506C0011520E2120711F019
:1034000000E010E0C801DF91CF911F910F91089566
:1034100078941F920F920FB60F9211240BB60F9251
:10342000CF92DF92EF92FF920F931F932F933F93D0
:103430004F935F936F937F938F939F93AF93BF93BC
:10344000CF93DF93EF93FF93809170008E7F8093F3
:1034500070000FE310E08BE1E82EF12C9BE2C92E07
:10346000D12CC091A305D091A4052097F9F4033283
:10347000110508F43AC003521109E091A105F09139
:10348000A20590818091A005282F209592239083FA
:103490009BE0D7011197F1F79150D9F79081892BD3
:1034A0008083C6010197F1F780E00DC00B30110554
:1034B000E0F00B501109E091A505F091A605EC0F85
:1034C000FD1F319780816CDA2196D093A405C093BB
:1034D000A30580910102909102028C179D0708F0CC
:1034E000C0CF1092A4051092A30580917000816056
:1034F00080937000FF91EF91DF91CF91BF91AF91D9
:103500009F918F917F916F915F914F913F912F91FB
:103510001F910F91FF90EF90DF90CF900F900BBE17
:103520000F900FBE0F901F90189581E08093920529
:1035300080910002282F30E0F901E358FB4FE4911D
:10354000F0E0EE0FFF1FE75BFB4F45915491509366
:10355000A2054093A105F901ED53FB4FE491E093DF
:10356000A00561E009DD83E08093B100E0E7F0E0D1
:103570008081816080830895CF93DF9318161906A8
:1035800044F0809170008E7F8093700010929205BD
:1035900019C0EC018091A5059091A6050E94EB59F8
:1035A000CE01C130D24014F080E092E0909302024C
:1035B000809301020E9456599093A6058093A50519
:1035C000892B29F4109202021092010207C0809107
:1035D0009205811103C0DF91CF91A7CFDF91CF91E9
:1035E0000895EF92FF921F93CF93DF931F921F9244
:1035F000CDB7DEB7162F20919205211105C0898322
:103600009A8393DF9A8189817C0121E0E21AF10893
:10361000E114E2E0FE0690F42091010230910202F2
:103620002817390708F4A8DF8091A5059091A60511
:10363000009721F08E0D9F1DFC0110830F900F90BD
:10364000DF91CF911F91FF90EF9008956DEE73E0A1
:1036500087E094E00C94F1234F925F926F927F92F7
:103660008F929F92AF92BF92CF92DF92EF92FF9292
:103670000F931F93CF93DF93CDB7DEB729970FB684
:10368000F894DEBF0FBECDBFE0911706F09118068B
:103690003C96E031F10508F0E1C18827EC54FF4F7A
:1036A0008F4F0C94BB656CE176E08CE898E0E3DA30
:1036B00080910F06811107C084EF95E00E940128D8
:1036C00081E080930F0681EB95E090933C09809315
:1036D0003B096CE271E080E090E08ADC1FB7F8946F
:1036E0008091B005811123C0E2EBF4E08491E8EF12
:1036F000F4E09491E82FF0E0EE0FFF1FE15DFB4F47
:10370000A591B491EC91E92319F461E085E305DC1E
:1037100061E085E331DC8CB580618CBD8CB5806463
:103720008CBD61E084E328DC61E083E325DC8091EB
:10373000B0058F5F8093B0051FBF249A80E590E0AD
:103740000E946F4367E080E090E00E943F1165E5D2
:103750008BE190E00E943F1165E58AE190E00E94D4
:103760003F110E946E4380E090E490936506809341
:10377000640680E090E690936D0680936C0680E08E
:1037800098E4909367068093660680E098E69093AD
:103790006F0680936E0680E090E5909369068093B3
:1037A000680680E090E7909371068093700680E051
:1037B00098E590936B0680936A0680E098E7909373
:1037C00073068093720680E590E00E946F4346E0A6
:1037D00050E060E175E089E090E00E94161181E31D
:1037E00093E09A8389831B821C821D821E82CE01F4
:1037F00003960E9467430E946E4380913B0990911B
:103800003C09DC0192961D921D921D921C92959787
:10381000FC0116A217A210A611A69A961D921D923F
:103820001D921C929D9740E65AEE60E070E046AB18
:1038300057AB60AF71AF40EA5FE060E070E0DA96EE
:103840004D935D936D937C93DD97189626E0FD0173
:10385000322F11923A95E9F7AC01425F5F4F34E1A4
:10386000FA0111923A95E9F7E0E1F5E001900D9245
:103870002A95E1F7FC01EE5BFF4F10820E94F82EC3
:103880008130910509F04DC080E590E00E946F43C2
:1038900060913B0970913C09625F7F4FCE010196B8
:1038A000FBD9CE0103960E94674360913B0970915A
:1038B0003C096A5E7F4FCE010196EED944E050E0AC
:1038C000BE016D5F7F4F81E090E00E941611609114
:1038D0003B0970913C096E5E7F4FCE010196DCD9A9
:1038E00044E050E0BE016D5F7F4F85E090E00E94B4
:1038F00016110E946E4360913B0970913C09625E13
:103900007F4FCE010196C8D98B819C81AD81BE814C
:103910008093370990933809A0933909B0933A09F5
:103920001DC0892BD9F464EF75E08CE898E0A3D929
:1039300086EF9FEF909318068093170691DBDC01CA
:10394000CB0188579C4EAF4FBF4F80937A0B90931B
:103950007B0BA0937C0BB0937D0B80C00E94C4486E
:1039600081E090E077C060E070E080E090E00E944D
:1039700060459093180680931706809136059091C4
:103980003705009709F46AC066E379E10E94B12720
:1039900065C099E288E10FB6F894A895809360001D
:1039A0000FBE909360001986E7D6811157C0009131
:1039B000E8071091E9070115110509F44FC0C80186
:1039C0003BD6682E712CF2E06F1671040CF095C195
:1039D00045C0D2D6811142C082E090E03BC040DBBE
:1039E00000917A0B10917B0B20917C0B30917D0B19
:1039F000061717072807390788F51092180610923E
:103A000017062CC02DDB00917A0B10917B0B2091B7
:103A10007C0B30917D0B0617170728073907E0F25A
:103A20001DC060E070E080E090E00E944647892B76
:103A300099F616DBDC01CB0188579C4EAF4FBF4F88
:103A400080937A0B90937B0BA0937C0BB0937D0BB0
:103A500086EF9FEF90931806809317060FB6F894A1
:103A6000A89580916000886180936000109260004A
:103A70000FBE00913B0910913C090115110509F495
:103A800017C1EEDA4B015C017801BEE3EB0EF11CCD
:103A9000F70180819181A281B381A5019401281B46
:103AA000390B4A0B5B0BCA01B901683E33E073075F
:103AB0008105910508F446C028EE33E040E050E06F
:103AC0000E94CB61861A970AA80AB90AD7018D927B
:103AD0009D92AD92BC921397F80186A597A5A0A9D7
:103AE000B1A969017A01CC0CDD1CEE1CFF1C8C1500
:103AF0009D05AE05BF0528F416A617A610AA11AAA3
:103B000009C0821B930BA40BB50BF80186A797A7DE
:103B1000A0ABB1ABF80182A993A9A4A9B5A98C1552
:103B20009D05AE05BF0528F412AA13AA14AA15AA6A
:103B300009C0821B930BA40BB50BF80182AB93ABAE
:103B4000A4ABB5ABF80186A597A5A0A9B1A9892B0F
:103B50008A2B8B2B69F4EE5BFF4F8081833041F41D
:103B600084E08083C8010E94F82E01967C0102C087
:103B7000E12CF12CF80182A993A9A4A9B5A9892B5C
:103B80008A2B8B2BA1F4EE5BFF4F8081833011F0E9
:103B900081110DC01082F8013E9684E1DF011D9273
:103BA0008A95E9F7C8010E94F82E03967C01B2E0DD
:103BB000EB16F10429F0E4E0EE16F10409F04CC034
:103BC00080E590E00E946F4360913B0970913C0951
:103BD000625F7F4FCE0101965FD8CE0103960E94AF
:103BE000674360913B0970913C096A5E7F4FCE014B
:103BF000019652D844E050E0BE016D5F7F4F81E0F6
:103C000090E00E94161160913B0970913C096E5E34
:103C10007F4FCE01019640D844E050E0BE016D5F79
:103C20007F4F85E090E00E9416110E946E436091E4
:103C30003B0970913C09625E7F4FCE0101962CD802
:103C40008B819C81AD81BE81809337099093380927
:103C5000A0933909B0933A09F2E0EF16F10491F01C
:103C600034F4EA94EF2821F561E875E010C043E0F0
:103C7000E416F10451F054E0E516F104C9F46FE4E0
:103C800075E010C061E775E00DC06EE575E08CE889
:103C900098E00E943B1686EF9FEF90931806809362
:103CA000170606C08CE898E00E943B160E94C448A4
:103CB00099E288E10FB6F894A895809360000FBE52
:103CC00090936000809117069091180629960FB680
:103CD000F894DEBF0FBECDBFDF91CF911F910F9142
:103CE000FF90EF90DF90CF90BF90AF909F908F901C
:103CF0007F906F905F904F90089560E0C8010E94A0
:103D00007142DC011996AD90BC901A9761E0C80130
:103D10000E947142FC0181849284F2E06F1671046A
:103D200009F475C162E0C8010E947142DC01199674
:103D3000CD90DC901A97B3E06B16710409F46BC157
:103D400063E0C8010E947142FC01E184F284F4E066
:103D50006F16710451F064E0C8010E947142DC01E9
:103D600019960D911C911A9703C08E01075F1F4F82
:103D70009092D9098092D809D092DB09C092DA09D1
:103D800065ED75E08CE898E00E940215B4018CE8BE
:103D900098E00E944B1663ED75E08CE898E00E9475
:103DA00002154AE050E0B6018CE898E00E94CA157E
:103DB0006CEC75E08CE898E00E940215B7018CE885
:103DC00098E00E944B1667EC75E08CE898E00E9442
:103DD0000215D2D48111E0C06091D8097091D9093F
:103DE00080914309909144094091DA095091DB098F
:103DF000DC01ED91FC916115710521F00088F189DC
:103E0000E02D16C00684F785E02D21E333E03A83E8
:103E100029834090D4095090D5096090D6097090BC
:103E2000D7094B825C826D827E82BE016F5F7F4FBD
:103E300019958130910509F0A8C09093C609809327
:103E4000C50987E0EBE3F2E0DE01119601900D92E7
:103E50008A95E1F7FE013196AAE4B9E06E0128E007
:103E6000C20ED11C81918D93EC15FD05D9F7E1149B
:103E7000F10429F00115110521F082EC03C082E064
:103E800001C082E880935109109252098FE080931B
:103E900053094FE050E065E479E0C501DBD3E1145C
:103EA000F10469F0AC0165E479E0C701D3D30115F1
:103EB000110529F0AC0165E479E0C801CBD3AC0170
:103EC0004550510965E479E080E1E5D3C9D86093B4
:103ED000C7097093C8098093C9099093CA09609370
:103EE000CB097093CC098093CD099093CE09809132
:103EF000430990914409DC01ED91FC910084F18526
:103F0000E02D1995892BB9F4ABD80091CB0910910C
:103F1000CC092091CD093091CE09DC01CB01801B69
:103F2000910BA20BB30B88399A43A105B105F8F2A6
:103F30008CEF9FEF1AC0C6010E949E410497C9F4FE
:103F400080914809811110C08BD86093CB09709380
:103F5000CC098093CD099093CE091092CF0910928D
:103F6000DF091092DE0918C090E09093DF0980937A
:103F7000DE098091430990914409DC01ED91FC91A7
:103F80000488F589E02D19951AC08EEF9FEF909364
:103F9000DF098093DE0913C069EB75E08CE898E0D7
:103FA0000E940215B5018CE898E00E942B1680E271
:103FB00094E00E94DD404ADB83E090E04BCD6DEA67
:103FC00075E08CE898E00E9402156091DE0970911E
:103FD000DF094AE050E08CE898E00E94CA1565E9E4
:103FE00075E08CE898E00E943B163AD8DC01CB01E2
:103FF00088579C4EAF4FBF4F80937A0B90937B0BAB
:10400000A0937C0BB0937D0B84EF9FEF23CD8BE5CA
:10401000C82E87E0D82E7E0129E0E20EF11C870130
:10402000A7CECF92DF92EF92FF920F931F93CF9381
:10403000DF938C017B016A010E94BD10EC01892B8A
:1040400009F182E08887A601DD0C660B770B4987B2
:104050005A876B877C8788819981009711F00E942D
:10406000EB59C7010E94E86599838883BE01C801A6
:10407000DF91CF911F910F91FF90EF90DF90CF9044
:104080000C94BC42DF91CF911F910F91FF90EF9064
:10409000DF90CF9008958F929F92AF92BF92CF9270
:1040A000DF92EF92FF920F931F93CF93DF93CDB7E1
:1040B000DEB7C150D1400FB6F894DEBF0FBECDBF02
:1040C000282F8091E20989832A83213090F02530BE
:1040D00010F0273171F48091E3099091E4099B83FA
:1040E0008C838091E5099091E6099D838E8396E00B
:1040F00001C092E08E010F5F1F4F213120F42F305D
:1041000030F48BEF01C08AEE820F823078F4309168
:10411000670A8091680AF801E90FF11D808381E048
:10412000890FF801E80FF11D9E5F30832F3021F1D8
:1041300050F4253091F0263009F0B1C030916B0A6F
:1041400080916C0A0EC0263109F48AC0273109F427
:1041500058C0203109F0A3C054C03091690A809141
:104160006A0AF801E90FF11D808381E0890FF801E7
:10417000E80FF11D9E5F92C04091690A50916A0A52
:10418000F801E90FF11D508382E0890F31E0390F0A
:10419000F801E30FF11D4083BA0167707727A3E0B0
:1041A00056954795AA95E1F7672B19F031E0340F42
:1041B00001C0342FB3E0B90FF801E80FF11D3083CF
:1041C000A4E0A90F60E070E04FEF4A0F6317B0F46E
:1041D00050E0CB0195958795400F511F880F991F8F
:1041E000FC01E559F54F60FD02C0808101C081816D
:1041F000FA0180836F5F7F4FAF5FE6CF9B2F930FF6
:104200004EC03091690A80916A0AF801E90FF11DE8
:10421000808381E0890FF801E80FF11D308363E0AE
:10422000690F9E5FF801E90FF11D932F990F90839D
:10423000EBE6FAE0862F40E0431780F4708151816D
:104240003296D801A80FB11D5C9351E0580FD801E8
:10425000A50FB11D8E5F7C934F5FEECF960F1FC0F1
:1042600080916B0A30916C0AF801E90FF11D3083DF
:1042700031E0390FF801E30FF11D808330916D0AB1
:1042800080916E0A42E0490FF801E40FF11D80832E
:1042900083E0890FF801E80FF11D9C5F30837801FE
:1042A000F8014FEF5FEFD02E8E2F801B8917A0F4FF
:1042B0008191482768E070E0DA01B695A79540FF44
:1042C00006C0AD0131E0432730EA532701C0AD01FC
:1042D0006150710989F7E8CFF801E90FF11D4083BA
:1042E00032E0C32EC90E9F5FF801E90FF11D508324
:1042F000F801EC0DF11D10828091E0099091E10927
:10430000DC01ED91FC910284F385E02DCF5FDE4F5F
:104310002883C150D1401995CF5FDE4F2881C1500D
:10432000D140019649F7E091F60AF091F70A3097EB
:1043300031F01995CF5FDE4F2881C150D140A09157
:10434000E009B091E1099E2D9D199C1588F4F701B3
:1043500061917F01ED91FC9111970190F081E02D29
:10436000CD01CF5FDE4F2883C150D1401995E2CFF8
:10437000ED91FC9111970680F781E02DCD01CF5F83
:10438000DE4F2883C150D1401995E091F80AF09191
:10439000F90ACF5FDE4F2881C150D140309731F00C
:1043A0001995CF5FDE4F2881C150D140CF5FDE4FDE
:1043B0002883C150D1400E9430184B015C0128E095
:1043C000D22EC12CCF5FDE4F2881C150D140E22ECA
:1043D000F12C8091E0099091E109DC01ED91FC91D3
:1043E0000084F185E02D1995892BC1F08091E009B9
:1043F0009091E109DC01ED91FC910284F385E02DBF
:1044000019959091E209891711F0CC2099F1F801E2
:10441000EC0DF11D8083DA94C39407C0E091F40A97
:10442000F091F50A309709F01995B5E0CB1222C04A
:10443000EA818E2F8F7790E08E159F0509F0A3C03B
:10444000E7FF04C08B81882349F181C08E2F90E063
:10445000FC013197E731F10568F48827EC53FF4FF1
:104460008F4F0C94BB6593E0D92E04C0DB8002C053
:1044700085E0D82E0E943018DC01CB0188199909FB
:10448000AA09BB09813D9740A105B10508F0D2C03A
:10449000D1109FCFF4E0FC1508F079C0AFEFBFEF6B
:1044A00040E0D12CC6010297242F30E028173907AD
:1044B000C4F4200F311FF9012081A22728E030E049
:1044C000BD0176956795A0FF06C0DB01F1E0AF273F
:1044D000F0EABF2701C0DB012150310989F74F5FA6
:1044E000E3CF800F911FFC0180818A134EC0F6013B
:1044F000EC0FFD1F80818B1348C049C04034D8F4B5
:10450000880F991FFC01E052F64FA5E0B0E0AC0F18
:10451000BD1FA80FB91F2C9130E0322F2227A4E035
:10452000B0E0AC0FBD1FA80FB91F8C91D901A82B0B
:10453000CD0190878783242F4F5F842F90E08617CB
:104540009707E4F22093F30A50FD61C080E01092D7
:10455000ED0A1092EF0A1092EE0A1092F20ACF5F63
:10456000DE4F0FB6F894DEBF0FBECDBFDF91CF9107
:104570001F910F91FF90EF90DF90CF90BF90AF9081
:104580009F908F90089581EEE2CF83EEE0CF8A81F5
:10459000853028F4833028F4813080F5D7CF8731F7
:1045A000A9F68B8190E0AC01559547953091F30ABF
:1045B00020E0822F90E084179507ECF42034C0F4BB
:1045C000FC013296EE0FFF1F880F991FBC0160524D
:1045D000764FCE018E0F9F1FDC018C9190E0982FBB
:1045E0008827E00FF11F3081832BFB0190878783A1
:1045F000322F2F5FDECF3093F30AA8CF5B81652F78
:1046000070E0759567952091F30A40E096CF4034AD
:1046100068F4880F991FFC01E052F64FD801A80FEB
:10462000B91F13968C9190E0908787834F5F4093DA
:10463000F30A8CCF82EE8BCFDC011696ED91FC91C4
:10464000179780E0309729F08F5F0280F381E02D8B
:10465000F9CF0895CF93DF93DC014E5F5F4FFC01EC
:104660009F012A1B3B0B9191992339F0EB01C40F59
:10467000D51F98834F5F5F4FF3CFCA01821B930B07
:10468000680F791FFB013297308331962083CA016E
:10469000DF91CF910895CF92DF92EF92FF920F9327
:1046A0001F93CF93DF9300D01F92CDB7DEB79A014F
:1046B000E0E0922F9F77220F232F221F330B31959B
:1046C0002115310509F0906801E00E0FA1E0B0E07E
:1046D000AC0FBD1FAE0FB11DFD019083211531053B
:1046E00011F0E02FE6CF10E0DB01A01BB10B149618
:1046F0008C93FE0131966F0180E090E08017910766
:1047000064F4F601F1906F019C01201B310B260F20
:10471000371FF901F5820196F1CF809143099091FD
:1047200044094F5F5F4F040F151FFC012081318149
:10473000F90122813381A801BD01F90119957C019C
:104740000E9430186093C7097093C8098093C90903
:104750009093CA0981E0E016F10609F080E00F901D
:104760000F900F900F90DF91CF911F910F91FF90BD
:10477000EF90DF90CF900895809143099091440984
:10478000009759F1DC01ED91FC910688F789E02D45
:104790001995811124C08091DE099091DF09892B40
:1047A000E1F48DEF9FEF9093DF098093DE09809114
:1047B000430990914409DC01ED91FC910680F78159
:1047C000E02D19958091430990914409DC01ED9108
:1047D000FC910488F589E02D199580E0089581E029
:1047E0000895EF92FF920F931F93CF93DF937C0175
:1047F0008B01EB0109900020E9F72197C61BD70B2D
:10480000BBDF8823A1F1F70101900020E9F7319780
:10481000EE19FF09CE010796E80FF91FE138F105FF
:1048200030F545E050E065E479E0C70113DFF801B9
:1048300020E030E02C173D0759F04191D901A80F35
:10484000B91FAD5BB64F12964C932F5F3F4FF2CF1F
:1048500025503109A901480F591F65E479E080E32B
:10486000DF91CF911F910F91FF90EF9014CF80E0D7
:10487000DF91CF911F910F91FF90EF900895CF920C
:10488000DF92EF92FF920F931F93CF93DF9300D0AD
:104890001F92CDB7DEB78C017B0129833A834B830E
:1048A0005C830E94BD106C0129813A814B815C813F
:1048B000892B19F183E0F6018087218732874387AE
:1048C000548780819181009711F00E94EB59C701B4
:1048D0000E94E865F60191838083B601C8010F90BC
:1048E0000F900F900F90DF91CF911F910F91FF903C
:1048F000EF90DF90CF900C94BC420F900F900F90F0
:104900000F90DF91CF911F910F91FF90EF90DF906B
:10491000CF900895EF92FF920F931F93CF93DF9361
:10492000CDB7DEB760970FB6F894DEBF0FBECDBF30
:104930007C0180E091E00E9456598C01892BD9F0CE
:104940001C821B821E821D828FEF9FEF98878F83B0
:1049500086E492E09A8389831A8619861C870B87DE
:1049600080E091E0988B8F871E861D86B701CE016F
:1049700001960E94BB37C80160960FB6F894DEBF5F
:104980000FBECDBFDF91CF911F910F91FF90EF90A0
:1049900008950F931F93CF93DF93EC012097F1F0CD
:1049A0000A811B81888587FD05C08E819F810097C4
:1049B00009F0EFDF8885843031F489859A85009786
:1049C00011F00E94EB5988819981009711F00E94A3
:1049D000EB59CE010E94EB59E801E0CFDF91CF9176
:1049E0001F910F910895CF93C82F462F61E070E07B
:1049F00089D361E070E08C2F8FD38111FACFCF91F2
:104A000008958F929F92AF92BF92CF92DF92EF92D2
:104A1000FF920F931F93CF93DF93B82E4B018A0120
:104A2000A22E68E270E078D3C82FD0E069E270E08F
:104A30008B2D72D3DC2FCC27C82B9E013770CB2C4B
:104A4000D12CC601880F991FAC014459594F6A01F6
:104A5000FA0180819181820F931FA801420F531F99
:104A60004130584098F060E078E07B01E21AF30AA8
:104A7000A701B4010E94EC10A8014E195F09B4010E
:104A80006E0D7F1DF6018081918102C0A801B401E5
:104A90000E94EC10A1100CC0C00FD11F4D2F68E276
:104AA00070E08B2D2FD34C2F69E270E08B2D2AD331
:104AB000DF91CF911F910F91FF90EF90DF90CF90FA
:104AC000BF90AF909F908F900895382F20916306EC
:104AD00090916206213208F049C080913F06811111
:104AE000FCCF42E040933F0630933E063FEF3093C9
:104AF0003D0610923C0620933B06A2E4B6E04BE153
:104B000056E0FA013E2F341B321718F43D913193D1
:104B1000F9CF10921A0620911A06990F922B9093B2
:104B20001A0690911906913061F41092190690912D
:104B30001A069093BB009091BC0093FDF8CF95ECC2
:104B400001C095EE9093BC0090913F069230E1F346
:104B500090913D069F3F79F080913D06803241F073
:104B600080913D06803331F084E005C081E003C0D0
:104B700082E001C083E01092410610926306109219
:104B800040060895DF92EF92FF920F931F93CF9309
:104B9000DF93CDB7DEB729970FB6F894DEBF0FBE0F
:104BA000CDBF8C017B01AE014F5F5F4F0E94593535
:104BB000D82E882309F459C0F7018081803109F487
:104BC00054C08FE18D83F801858196810E94C533A1
:104BD000B701F801858196810E94D53440E06EE4EA
:104BE000F801858196810E94FA3340E06B81F801DB
:104BF000858196810E94FA3340E06C81F8018581BD
:104C000096810E94FA33F7018081803139F040E0CB
:104C10006D81F801858196810E94FA33F8018581C2
:104C200096810E94C533B701F801858196810E9463
:104C3000D534F801408168E4858196810E94FA3379
:104C400064E170E080E090E00E94F817F801808154
:104C5000882331F06AE070E080E090E00E94F8176D
:104C6000F801858196810E94C5338D2D29960FB656
:104C7000F894DEBF0FBECDBFDF91CF911F910F9192
:104C8000FF90EF90DF900895EF92FF920F931F93A4
:104C9000CF93DF93EC018C01085F1F4F7E01699178
:104CA00070E084E0759567958A95E1F740E150E002
:104CB0008CE898E00E94CA15F70160816F7070E07F
:104CC00040E150E08CE898E00E94CA15C017D10777
:104CD00029F7DF91CF911F910F91FF90EF900895E9
:104CE000CF93DF931F92CDB7DEB76983DC01ED91DF
:104CF000FC910280F381E02D41E050E0BE016F5F46
:104D00007F4F19950F90DF91CF910895FC01818D10
:104D1000928D0895FC0184899589089521E333E0FB
:104D2000FC0131832083FB014089518962897389A9
:104D3000FC0142835383648375830895DC01ED9104
:104D4000FC91048CF58DE02D199480E00895FC0110
:104D50009485FB018485981303C081E0943009F4A5
:104D600080E0089521E0FC018485843009F420E08E
:104D7000822F089508950F931F93CF93DF931F926F
:104D8000CDB7DEB7FC01218D328D232B61F08C0174
:104D900041E050E0BE016F5F7F4F808D0E94B411F3
:104DA000181619061CF08FEF9FEF08C0F801818DCF
:104DB000928D0197928F818F898190E00F90DF9182
:104DC000CF911F910F910895FC0184850C94B4112B
:104DD000CF93DF931F92CDB7DEB741E050E0BE0125
:104DE0006F5F7F4FFC0184850E94B411181619066D
:104DF0001CF4898190E002C08FEF9FEF0F90DF914C
:104E0000CF910895FC018485843011F00C949411A5
:104E100080E090E008950F931F93CF93DF93CDB779
:104E2000DEB728970FB6F894DEBF0FBECDBF8C015A
:104E3000F801818D928D892B49F0D801ED91FC917B
:104E40000284F385E02DC8011995F2CF808D0E9470
:104E50009411181619065CF548E050E0BE016F5F2A
:104E60007F4FD80158968C910E94B4119C0118165E
:104E70001906DCF489819A81AB81BC81F801808BB1
:104E8000918BA28BB38B8D8190E0982F88272E81F8
:104E9000820F911D958B848B2F8130E0322F22273A
:104EA0008885280F311D328F218FC90102C080E013
:104EB00090E028960FB6F894DEBF0FBECDBFDF910D
:104EC000CF911F910F910895AF92BF92CF92DF9231
:104ED000FF920F931F93CF93DF938C015B01EA0145
:104EE000FC01C688D788F08C80E590E00E946F4373
:104EF0008F2D0E9482418C179D0720F48F2D0E94D8
:104F00008241EC019E01A501B6018F2D0E941D4139
:104F10000E946E43F801868997898C0F9D1F978B9D
:104F2000868BCE01DF91CF911F910F91FF90DF9083
:104F3000CF90BF90AF900895CF93DF93EC01888D11
:104F4000843061F00E942312E88DF0E0EE0FFF1F25
:104F5000EC58F94F1182108284E0888FDF91CF9155
:104F60000895EF92FF921F93CF93DF93FC01208D62
:104F7000243011F080E01CC07B01EC0110E0812F97
:104F80000E94EE12811102C0188F05C08831E1F332
:104F90001F5F1430A1F7888D843061F3FD86EC86A5
:104FA0001A8E198E20E0A70162E00E94371281E07C
:104FB000DF91CF911F91FF90EF9008950F931F9372
:104FC000CF93DF931F92CDB7DEB78C01DC01ED915B
:104FD000FC910084F185E02D1995892B51F0BE01DB
:104FE0006F5F7F4FF80184850E945C11898190E09A
:104FF00002C08FEF9FEF0F90DF91CF911F910F9124
:105000000895FC011382128288EE93E0A0E0B0E0E4
:1050100084839583A683B78382E792E0918380831C
:1050200081E393E097878687108A118A128A138A10
:1050300084E0808F0895CF92DF92EF92FF920F93DA
:105040001F93CF93DF93CDB7DEB7E1970FB6F894F8
:10505000DEBF0FBECDBF7C016A0101E313E01A83FE
:1050600009831B821C821D821E82CE01099668ABB9
:1050700079ABC7DF1DA30CA31EA21FA218A619A6F9
:105080008091370990913809A0913909B0913A0976
:105090008CA79DA7AEA7BFA78B839C83AD83BE8340
:1050A00018861F82AE014C5D5F4F68A979A9CE01B9
:1050B00001963ED481309105B1F4D701ED91FC9178
:1050C0000488F589E02D1BA70AA78EA19FA1A8A59A
:1050D000B9A58CA79DA7AEA7BFA7A601BE01665D17
:1050E0007F4FC7011995E1960FB6F894DEBF0FBE4A
:1050F000CDBFDF91CF911F910F91FF90EF90DF9087
:10510000CF9008959B0190E00496982F8827642FF4
:10511000820F931F0C943F110F931F93CF93DF9334
:105120001F92CDB7DEB790E00496982F88278C01A8
:10513000060F171F0E94CB108FE00E94E510812FF1
:105140000E94E510802F0E94E51080E00E94E5108B
:1051500089830E94C91089810F90DF91CF911F919F
:105160000F910895CF93FC01C08D80E590E00E94DF
:105170006F4360E270E08C2F36DC62E070E08C2FD1
:10518000CBDF84FD17C062E070E08C2FC5DF83FFAA
:105190000AC048E162E070E08C2FB4DF0E946E43E9
:1051A00080E090E010C00E946E4380E590E00E9495
:1051B0006F43E3CF40E162E070E08C2FA3DF0E94F9
:1051C0006E4381E090E0CF910895CF93DF93C82F95
:1051D000D62F472F60E170E095DF4D2F61E170E041
:1051E0008C2FDF91CF918ECFFF920F931F93CF9390
:1051F000DF93FB01DC0157961C921E92569758963E
:10520000FC908281811109C08381811106C0848153
:10521000811103C085818823F1F041155105D9F032
:105220008A01EF0180E590E00E946F43BE016E5F4E
:105230007F4F2F2D30E0922F882744E050E0845F8D
:105240009B4F0E941611B8018F2DBFDF0E946E4345
:1052500081E090E002C080E090E0DF91CF911F916B
:105260000F91FF900895FC018485843011F00C9417
:10527000EE1280E00895CF93DF93FC012485243063
:10528000C9F0EC01F0DF843181F0882371F08831BE
:1052900061F08C3161F4E881F9810084F185E02DC1
:1052A000CE01199521E0892B19F420E001C021E0FD
:1052B000822F01C080E0DF91CF910895CF92DF92DD
:1052C000EF92FF921F93CF93DF93FC01148514306C
:1052D00099F1EC0180E590E00E946F4368E070E096
:1052E000812F81DB0E946E430E9430186B017C018C
:1052F000CE01B9DF8823B1F061E070E080E090E09A
:105300000E94F8170E943018DC01CB018C199D090E
:10531000AE09BF09883E9340A105B10548F38C85CD
:105320000E942312EC85F0E0EE0FFF1FEC58F94FBE
:105330001182108284E08C87DF91CF911F91FF90C2
:10534000EF90DF90CF90089580E3FB018083329649
:10535000842F82958F7090E1899F401911244A30E3
:1053600014F4405D01C0495C4293482F8111F0CF95
:1053700008952F923F924F925F926F927F928F92F9
:105380009F92AF92BF92CF92DF92EF92FF920F93D4
:105390001F93CF93DF93CDB7DEB7E3970FB6F894A3
:1053A000DEBF0FBECDBF7C011A012B0139010E9467
:1053B00030184B015C0187010D5B1F4FC8012BDDCD
:1053C00018161906A4F00E943018DC01CB018819C8
:1053D0009909AA09BB09281639064A065B06D8F0BE
:1053E00062E370E080E090E00E94F817E7CF42E2CD
:1053F00050E0BE016F5F7F4FC8010E940512898196
:10540000823011F080E051C1F8018489958983349C
:105410009105C1F702C08FEF48C16D817E818F81F8
:1054200098850E94C3654B015C01F3016083718321
:105430008283938346E050E0B701685F7F4FCE01DF
:105440004D960E940166892BE9F6F70180819181D2
:10545000A281B38188169906AA06BB0698F28481B8
:105460009581A681B78188159905AA05BB0550F2DB
:1054700089899A89AB89BC8986879787A08BB18BEC
:105480008EECA82EB12CC80176DCF1E0AF1AB10881
:10549000D1F719A6670182E2C80ED11CF701B696B2
:1054A000FBA7EAA7C7018A969DA78CA73C974F0147
:1054B00089969FA78EA73897F9ABE8AB1701F6E15D
:1054C0002F0E311CC5979BAB8AABF801818D928D55
:1054D000181619060CF0E8C0C8014DDC833391059D
:1054E00009F4C0C0F4F481309105B1F11CF4892BAA
:1054F00061F3D0C083309105B1F1069709F0CAC0BD
:10550000C80139DC5C0144E050E06AA97BA9C8010C
:105510000E940512412C512CBB24F4E0AF1AB108B3
:105520003BC08A33910509F473C03CF4853391057F
:1055300069F0C69709F43AC0ADC08B33910509F400
:105540007CC08F3F910509F4C0CFA4C0C80113DC13
:10555000C80111DC89A7B9CFC8010DDC44E050E0D7
:1055600068A979A936C0C80106DC5C0144E050E0B6
:10557000B101C8010E940512412C512CBB2494E0BA
:10558000A91AB1084A145B040CF09FCFC801F3DBE1
:10559000EFEF4E1A5E0AF6CF4A145B040CF095CF7B
:1055A000C801E9DB8FEF481A580AF6CFC801E3DBE0
:1055B000B82EF701828D811110C0838D81110DC02D
:1055C000848D81110AC0858D811107C044E050E0AF
:1055D000B401C8010E94051278CFEEA5FFA5408056
:1055E000518062807380B401CE0183960E944C1674
:1055F0008DA19EA1AFA1B8A584159505A605B705F7
:1056000029F3BB2009F461CFC801B5DBBA94F9CF07
:10561000C801B1DB44E050E06AA57BA5C8010E9447
:105620000512F70166A177A180A591A50E94C36527
:1056300066A377A380A791A748CFC8019CDB44E06D
:1056400050E06CA57DA5C8010E940512F70162A576
:1056500073A584A595A50E94C36562A773A784A7B7
:1056600095A733CFC80187DB44E050E0B601C801FD
:105670000E940512F70162A173A184A195A10E9465
:10568000C36562A373A384A395A366A777A780AB22
:1056900091AB1BCFC8016FDBB82EBB2009F415CF2F
:1056A000C80169DBBA94F9CF89A5E3960FB6F894DF
:1056B000DEBF0FBECDBFDF91CF911F910F91FF9045
:1056C000EF90DF90CF90BF90AF909F908F907F90A2
:1056D0006F905F904F903F902F9008957F928F92A0
:1056E0009F92AF92BF92CF92DF92EF92FF920F9371
:1056F0001F93CF93DF93CDB7DEB7A6970FB6F8947D
:10570000DEBF0FBECDBF8C01762E942E852E20E2FB
:10571000B22ECE0101967C01FC012B2D11922A950F
:10572000E9F781E393E09AA389A38FEF8BA38CA37E
:105730008DA38EA3680183E4C80ED11C43E450E01E
:10574000BE016F5D7F4FC6014FDD019609F4B5C004
:1057500081E089838A8386E0A82EAB821C82F801CF
:1057600064817581868197810E94C3656D837E8384
:105770008F83988789869A8680E890E09C878B87BC
:105780004CE150E0B701C6019FDBF7012B2D1192D0
:105790002A95E9F7480188E0880E911CF401D701A9
:1057A00001900D92AA94E1F740E150E0B701C601E3
:1057B0008BDBF7011192BA94E9F796E0A92EB12C90
:1057C00040E250E0B701C6017FDBF1E0AF1AB1085B
:1057D000B9F783E6898392E89A8393E59B838C8368
:1057E00085E38D8381E08E837F829DE3988797E0B8
:1057F00099878A8786E0F401DE011B9601900D925D
:105800008A95E1F78CE0898B8A8B6DE274E0CE019A
:1058100043960E944066F8014385BE01675E7F4F54
:10582000C80192DDF8014485BE01655E7F4FC80165
:105830008BDDF8014585BE01635E7F4FC80184DDC5
:105840004EE150E0B701C6013FDBF3E07F121DC01F
:1058500082E3898384E08A83F80196859B83978518
:105860009C8390899D8391899E8396E39F838887FB
:10587000828D8987838D8A87848D8B87858D8C87A0
:105880004CE050E0B701C6011FDB87E3898386E067
:105890008A8391E09B8393E09C838D838FE08E834A
:1058A0008AE38F838BE388878FEF898749E050E015
:1058B000B701C60109DBC60155DCA6960FB6F89400
:1058C000DEBF0FBECDBFDF91CF911F910F91FF9033
:1058D000EF90DF90CF90BF90AF909F908F907F9090
:1058E00008958091360590913705009711F00E9438
:1058F000A419A8950895A8950E942C1B029754F00E
:105900000E94504C8091360590913705009711F018
:105910000E94A4190C948C0E61E08DE00C948D17FC
:105920008FEE97E00E94011460E08DE00C948D17DB
:105930002F923F924F925F926F927F928F929F929F
:10594000AF92BF92CF92DF92EF92FF920F931F938D
:10595000CF93DF93CDB7DEB765970FB6F894DEBF70
:105960000FBECDBF7C016B013A01FB0120E080E05E
:1059700090E06AE03191332309F140ED430F4A3062
:1059800080F4689FA001699F500D1124CA01C0973F
:10599000830F911D37FD9A958F3F910559F350F371
:1059A00013C03E3289F4233079F0D301A20FB11D28
:1059B00012968C932F5F80E090E0DCCF233021F4AF
:1059C000F301858381E020C0F70142815381648126
:1059D000758180913F0990914009A0914109B09152
:1059E0004209481759076A077B0709F48AC10E94D0
:1059F00030188701085F1F4F6F7077277C5FC801E1
:105A0000B0DA813019F080E090E0D9C181E393E011
:105A10009A838983F70182819381A481B5818B83E5
:105A20009C83AD83BE8345E350E0BE016F5F7F4F33
:105A3000C801DADB892B19F4C12CD12C5EC10E947C
:105A40003018F701778366837627672776277A836E
:105A5000698342E050E0BE016F5F7F4FC80134DAD6
:105A600081E090E09E878D8742E050E0BE01635F59
:105A70007F4FC80129DA80E091E09E878D8742E060
:105A800050E0BE01635F7F4FC8011EDA1E861D868F
:105A900042E050E0BE01635F7F4FC80115DA42E08B
:105AA00050E0BE01635F7F4FC8010EDA42E050E074
:105AB000BE01635F7F4FC80107DA5601F50180819F
:105AC000882301F1F6015F018191811113C0450125
:105AD0008C189D081814190484F48F8641E050E056
:105AE000BE01615F7F4FC801EFD9A401B601C801B3
:105AF000EBD903C08E3239F7EACF6501FFEFCF1A39
:105B0000DF0ADCCF1F8641E050E0BE01615F7F4FBE
:105B1000C801DAD9C12CDD24D394DE86CD8642E0DB
:105B200050E0BE01635F7F4FC801CED9DE86CD86CF
:105B300042E050E0BE01635F7F4FC801C5D9C80194
:105B400011DB892B09F478CF63E0A62EB12CF2E0AB
:105B50006F0E711C0E9430181B012C01C8015BD90B
:105B600018161906A4F00E943018DC01CB01821926
:105B70009309A409B50989389341A105B105D0F469
:105B800062E370E080E090E00E94F817E7CFF70151
:105B90004281538164817581808D918DA28DB38DF9
:105BA000481759076A077B0741F4848D958DC5977F
:105BB00021F406C02FEF3FEF96C02EEF3FEF93C0CA
:105BC000F70181A192A10C970CF4A1C04CE050E028
:105BD000BE016F5F7F4FC8010E9405128B8190E06C
:105BE000982F88272C81822B9A8B898B298130E0F2
:105BF000322F22274A81242BF701468157814217F1
:105C0000530709F081C097FF7FC08F709270892B76
:105C100009F0D2C0CF80D12CDC2CCC248885C82AB6
:105C2000C114D10409F4C5C0812C912C8D8190E060
:105C3000982F88272E81822B8816990608F46AC02F
:105C4000812C912C41E050E0BE016D5E7F4FC80178
:105C50000E9405128B89982F907C09F088C08111D1
:105C60007CC08B898111EECF42E050E0BE01615FC4
:105C70007F4FC8010E94051242E050E0BE01635F01
:105C80007F4FC8010E940512C80175D8C80173D89A
:105C9000C80171D8C8016FD842E050E0BE016F5E04
:105CA0007F4FC8010E9405128F8598898115914008
:105CB00009F061C02D853E85322723273227213008
:105CC000310509F058C089899A898115944009F0F5
:105CD0006DC044E050E0B301C8012C8B3D8B0E94A5
:105CE00005122C893D896901F1E0AF1AB10829F04C
:105CF0002FEFC216D20609F42DCFC8011DD9C60157
:105D00005EC08EEF9FEF5BC02CEF3FEFECCF2DEF2F
:105D10003FEFE9CF41E050E0BE01635F7F4FC80134
:105D20000E9405128D8581110FC08D858111F2CFE2
:105D3000C80121D8C8011FD8C8011DD8C8011BD867
:105D4000FFEF8F1A9F0A72CF8D859FEF980F9D8767
:105D5000882359F3C8010FD8F7CF8B899FEF980F8D
:105D60009B8B882309F47DCFC80105D8F6CFC801E5
:105D700002D81B8A76CF412C512C89899A89982781
:105D8000892798274816590638F4C8010E94BB266F
:105D90008FEF481A580AF1CFEFEF8E1A9E0A8C1433
:105DA0009D0409F04FCF26EF3FEF9DCF27EF3FEF48
:105DB0009ACF2AEF3FEF97CF2BEF3FEF94CF659627
:105DC0000FB6F894DEBF0FBECDBFDF91CF911F910C
:105DD0000F91FF90EF90DF90CF90BF90AF909F908A
:105DE0008F907F906F905F904F903F902F9008958D
:105DF0002F923F924F925F926F927F928F929F92DB
:105E0000AF92BF92CF92DF92EF92FF920F931F93C8
:105E1000CF93DF93CDB7DEB727970FB6F894DEBFE9
:105E20000FBECDBF8C010E94CC5A2FEC37E040E072
:105E300050E00E94ED61DC01CB010196A11DB11D76
:105E4000F80184839583A683B78380839183A2839B
:105E5000B3835801F3E4AF0EB11CC5016DD864E4FF
:105E600070E0C5017ED8882309F437C10E9430183C
:105E70002B013C01812C912C1D82C8018E5B9F4F10
:105E80009F838E8343E0342E58EEC52E53E0D52EEB
:105E9000E12CF12C62E0262EAE81BF818C91833003
:105EA00009F402C181111FC0F80184819581A68186
:105EB000B7810196A11DB11D84839583A683B78305
:105EC0000E9430186419750986099709A70196017F
:105ED0000E94CB61A90161E0C80100DC81E0AE81D4
:105EE000BF818C93C2C08430F1F4F8018481958124
:105EF000A681B7810196A11DB11D84839583A683D8
:105F0000B7830E9430186419750986099709A7019B
:105F100096010E94CB61A90163E0C801DFDBAE817D
:105F2000BF812C92A2C0813051F5F80142AD53AD32
:105F300064AD75AD9E012F5F3F4FC8011ADA8D83A6
:105F4000823009F092C089819A81AB81BC81F801CD
:105F500084839583A683B7830E94301864197509DA
:105F600086099709A70196010E94CB61A90163E008
:105F7000C801B4DBED81AE81BF81EC937DC082307E
:105F800009F073C0D801DA964D915D916D917C91C5
:105F9000DD979E012F5F3F4FC801EBD98D83853080
:105FA00009F05CC0EE81FF813082F80182A193A1EB
:105FB000A4A1B5A1892B8A2B8B2B41F484E893E013
:105FC000A0E0B0E082A393A3A4A3B5A3F80186A1A7
:105FD00097A1A0A5B1A5892B8A2B8B2B61F482A157
:105FE00093A1A4A1B5A1B695A7959795879586A3EA
:105FF00097A3A0A7B1A7F80182A593A5A4A5B5A5CD
:10600000892B8A2B8B2BA9F482A193A1A4A1B5A1E2
:10601000AC01BD0123E076956795579547952A9584
:10602000D1F7841B950BA60BB70B82A793A7A4A748
:10603000B5A7F80186A197A1A0A5B1A586A797A7A6
:10604000A0ABB1AB82A593A5A4A5B5A582AB93AB3C
:10605000A4ABB5AB88248394912C0EC0FD81F6309F
:1060600021F4AE81BF811C9207C0BD81BF3F21F4E6
:10607000EE81FF8110821D82F1E08F16910409F4F8
:106080000BCF0E943018DC01CB0184199509A609B9
:10609000B709F80126A937A940AD51AD281739072E
:1060A0004A075B0708F0F8CEC5010E949C27F8015B
:1060B00084819581A681B7810196A11DB11D84833C
:1060C0009583A683B7830E943018F801FE966083FB
:1060D000718382839383C40102C080E090E027969D
:1060E0000FB6F894DEBF0FBECDBFDF91CF911F91E9
:1060F0000F91FF90EF90DF90CF90BF90AF909F9067
:106100008F907F906F905F904F903F902F90089569
:106110009FE9980F963010F429EA05C09FEB980F7D
:10612000963018F429EC280F05C090ED980F9A309E
:1061300008F4292F822F08950F931F93CF93DF9395
:10614000282FDC01C42FD52F8A2F821B8617D0F46D
:106150008D01ED91F0E084E0F595E7958A95E1F702
:10616000EA56FD4F808188832296CE010197F8017F
:106170003081E32FEF70F0E0EA56FD4F3081FC01F3
:106180003083E2CFFA01E60FF11DE60FF11D108218
:10619000DF91CF911F910F91089585ED8093BC0001
:1061A0008091BC0084FDFCCF10923F060895409181
:1061B000C006262F30E0240F311D21323105DCF4DA
:1061C00020913F062430C9F4FC0180E090E086175E
:1061D00058F43091C0062191DC01A256B94FA30FAB
:1061E000B11D2C930196F3CF8091C006680F609388
:1061F000C00680E0089581E0089582E00895089542
:10620000E0917D0680917C06E81730F4F0E0E258DA
:10621000F94F808190E008958FEF9FEF089590915E
:106220007D0680917C06981750F4E92FF0E0E25843
:10623000F94F208130E09F5F90937D0602C02FEFE1
:106240003FEFC901089580917C0690E020917D0682
:10625000821B91090895CF92DF92EF92FF920F93E4
:106260001F93CF93DF937C01262F972F8A01809174
:106270004006882391F0C62FD72F6E01C40ED51E7D
:10628000CC15DD0569F06991D701ED91FC91019084
:10629000F081E02DC7011995F3CF642F822F87DF9E
:1062A000C801DF91CF911F910F91FF90EF90DF9088
:1062B000CF900895CF93DF931F92CDB7DEB7698358
:1062C000209140062223D1F020916306203240F035
:1062D00021E030E0FC013383228380E090E014C0B1
:1062E00080914106E82FF0E0EE5BF94F99819083B1
:1062F0008F5F809341068093630604C061E0CE0106
:10630000019655DF81E090E00F90DF91CF910895E5
:106310000895FC01818190913F069111FCCF91E09D
:1063200090933F0690933E062FEF20933D061092E8
:106330003C0610923B0690931A0690911A06880F1D
:10634000892B80931A0680911906813061F410928E
:10635000190680911A068093BB008091BC0083FDD2
:10636000F8CF85EC01C085EE8093BC0080913F069C
:106370008130E1F380913C06811103C080913C069D
:1063800001C081E0ABE1B6E02EE736E0F9019E2FD7
:10639000921B981718F49D919193F9CF10927D0656
:1063A00080937C0689E299E03ACF08951F920F927C
:1063B0000FB60F9211240BB60F922F933F934F936A
:1063C0005F936F937F938F939F93AF93BF93EF935D
:1063D000FF938091B900887F803609F49CC068F5EE
:1063E000883209F45BC090F4803109F454C038F469
:1063F000882309F4F6C0883009F44DC0F5C088310F
:1064000009F44CC0803209F45DC0EEC0803409F458
:1064100068C048F4803309F455C0883309F0E4C0FB
:1064200080933D06D8C0803509F44FC0883509F403
:106430005DC0883409F0D8C0D6C0883909F4C7C017
:10644000A8F4883709F467C038F4883609F463C0C3
:10645000803709F460C0C8C0883809F4B8C08039F2
:1064600009F45FC0803809F0BFC05BC0803B09F40D
:1064700086C038F4803A09F466C0883A09F47FC0CF
:10648000B3C0803C09F4A7C0883C09F4A4C0883B91
:1064900009F48AC0A9C080911A0610C090913C06E8
:1064A00080913B06981770F5E0913C0681E08E0FD5
:1064B00080933C06F0E0E55EF94F80818093BB005D
:1064C00085EC86C080933D068EC0E0913C0681E05D
:1064D0008E0F80933C068091BB00F0E0E55EF94FA3
:1064E000808390913C0680913B066EC0E0913C0613
:1064F00081E08E0F80933C068091BB00F0E0E55E6A
:10650000F94F808380913E0681116DC081E08093B8
:10651000190684EA61C083E080933F061092E40686
:10652000CFCF8091E406803208F051C0E091E406BC
:1065300081E08E0F8093E4068091BB00F0E0EC5385
:10654000F94F8083BDCF85EC8093BC0010923F064D
:106550008091E406803230F4E091E406F0E0EC5300
:10656000F94F10826091E40670E0E091C206F0916C
:10657000C30684EC96E019951092E40635C084E0D9
:1065800080933F061092C1061092C006E091BE06AD
:10659000F091BF0619958091C006811105C081E078
:1065A0008093C00610929E06E091C10681E08E0F96
:1065B0008093C106F0E0E256F94F80818093BB00E2
:1065C0009091C1068091C006981708F479CF85E8AC
:1065D0008093BC0009C085EC8093BC0010923F06FC
:1065E00003C010923D06D9DDFF91EF91BF91AF91AD
:1065F0009F918F917F916F915F914F913F912F91DB
:106600000F900BBE0F900FBE0F901F901895109219
:106610003F0681E080933E061092190661E084E116
:106620000E948D1761E085E10E948D17E9EBF0E093
:1066300080818E7F808380818D7F808388E48093BA
:10664000B80085E48093BC000895DC01E0E061506F
:1066500038F08D91E827F0E0E75DF94FE491F7CF4E
:106660008E2F089581E00C946525FC01818191E0D5
:106670009093400680936206109241061092630642
:1066800008951F93CF93DF93EC01162FEEDF61EE99
:1066900089E299E00FDE612F89E299E00BDECE01FD
:1066A000DF91CF911F91DECFAF92BF92CF92DF9259
:1066B000EF92FF921F93CF93DF93EC010E9430186B
:1066C0006B017C0128EEC20E23E0D21EE11CF11CFE
:1066D0008BE4A82EB12C0E9430186C157D058E0518
:1066E0009F0588F460EFCE01CCDFCE0112DE182FBB
:1066F00080FF11C0EF85F889309709F01995C50121
:106700000197F1F7E8CF81E08A8364E374E08CE8D5
:1067100098E00E942B16812FDF91CF911F91FF905F
:10672000EF90DF90CF90BF90AF9008951F93CF93DD
:10673000DF93EC01162FB8DFCE0197DF62ED89E21F
:1067400099E0B8DD212F30E02095309584E0220FCC
:10675000331F8A95E1F7612F622B89E299E0AADD68
:10676000CE0180DFCE01D5DD811711F084E08A8370
:10677000DF91CF911F910895CF93DF93EC0163ECEC
:1067800080DFCE01DF91CF91C4CD1F93CF93DF93F4
:10679000EC018ADFCE01F0DF60E0CE01C7DFCE0181
:1067A00083DFCE0162DF64EB89E299E083DDCE0115
:1067B00059DFCE0179DF182F82FF02C082E08A8381
:1067C0008881882331F0CE01D7DF682F6160CE0148
:1067D000ADDF11FB882780F9DF91CF911F910895DC
:1067E000CF93DF93EC01C8DF682F6460CE01DF91A7
:1067F000CF919CCFEF92FF921F93CF93DF931F9285
:10680000CDB7DEB77C01162F49834EDF4981442383
:1068100011F0C701E5DFC70128DF65EA89E299E0E9
:1068200049DD612F89E299E045DDC7010F90DF91D5
:10683000CF911F91FF90EF9015CF6F927F928F9223
:106840009F92AF92BF92CF92DF92EF92FF920F93FF
:106850001F93CF93DF93FC012485211196C0872ECF
:10686000762EEC0192DF811108C06FE374E08CE8B2
:1068700098E00E942B168FEF89C0CE0115DF40E013
:1068800060EFCE01B7DFE12CF12C66246A94CC24B2
:10689000C394D12C0E2D06950695069510E08E2DED
:1068A0008770560101C0AA0C8A95EAF78B85082EDD
:1068B000000C990BE816F90634F4FE01E00FF11F05
:1068C00093809A2006C099249394E816F90609F05B
:1068D000912CCE01E9DECE01C8DE68E789E299E0BD
:1068E000E9DC911002C060E001C060E889E299E053
:1068F000E1DCCE01B7DECE01D7DE282F2074982F41
:10690000907885FF13C02223B9F0482F50E060E053
:1069100070E022E08CE898E00E943B156BE474E0A4
:106920008CE898E00E942B168EEF30C0211104C035
:10693000911104C06E2C08C0992331F0FE01E00FC4
:10694000F11F8381A82A06C0FE01E00FF11FA09469
:106950008381A822A382FFEFEF1AFF0A80E4E816E2
:10696000F10409F097CF6B86EFEF6E1202C081E061
:106970008C87DE011396E72DF82D2B968D91819350
:10698000AC17BD07D9F781E001C080E0DF91CF915E
:106990001F910F91FF90EF90DF90CF90BF90AF903D
:1069A0009F908F907F906F900895CF92DF92EF929B
:1069B000FF920F931F93CF93DF931F92CDB7DEB754
:1069C0008C01F62E40E065E5798314DFCF2C7981C8
:1069D000D72E760188E0E80EF11CF60161916F0177
:1069E00040E0C80107DFCE14DF04B9F70F90DF9154
:1069F000CF911F910F91FF90EF90DF90CF9008956E
:106A0000AF92BF92CF92DF92EF92FF920F931F93BC
:106A1000CF93DF931F921F92CDB7DEB77C018A011F
:106A2000FC018581968169837A83AFDE69817A81F1
:106A3000882381F1F70185819681B7DF40E06EEB15
:106A4000F70185819681D6DE58016801F9E0CF0E05
:106A5000D11CF70105811681C80126DEC80105DEBB
:106A600066E989E299E026DCC801FCDDC8011CDE8C
:106A700061EEC80106DEC8014CDCF50181935F01BF
:106A8000EC15FD0531F7F701858196817EDE91E0F9
:106A9000813009F090E0892F0F900F90DF91CF9116
:106AA0001F910F91FF90EF90DF90CF90BF90AF902C
:106AB0000895CF93DF93EA01A3DF882331F068E0E4
:106AC000CE01C3DD91E02885821390E0892FDF910C
:106AD000CF910895CF93DF93CDB7DEB729970FB647
:106AE000F894DEBF0FBECDBFAE014F5F5F4FE1DF59
:106AF000882389F08D818F3361F020F48F3159F430
:106B000089E00CC08F3519F08F3739F004C08BE065
:106B100005C08AE003C080E001C08CE029960FB672
:106B2000F894DEBF0FBECDBFDF91CF910895FB017A
:106B300024813581428153812417350758F44081DF
:106B40005181DA01A20FB31F8C9384819581019644
:106B50009583848380E00895CF93DF93EC01E881EF
:106B6000F9810284F385E02DCE0119950196B9F7DC
:106B7000DF91CF910895EF92FF920F931F93CF93E0
:106B8000DF93009719F48FEF9FEF86C0FC01E48438
:106B9000F584D7010D911C91D801ED91FC910688E7
:106BA000F789E02DC8011995882369F3D801ED9183
:106BB000FC910084F185E02DC8011995D801ED9173
:106BC000FC91892B61F30284F385E02DC8011995AE
:106BD000EC010196C1F2F8018589882349F04C2F18
:106BE00050E060E070E02AE08CE898E00E943B15FD
:106BF000D70112968C91882309F44DC0C532D10576
:106C000009F049C0D801ED91FC910084F185E02D97
:106C1000C801199502975CF0D801ED91FC910688A6
:106C2000F789E02DC80119958111ECCFACCFD1E0E7
:106C3000C0E0D801ED91FC910284F385E02DC801FC
:106C400019958F3FBFEF9B0709F49DCF9C012154FD
:106C500031092A31310530F09C01215631092A31A0
:106C6000310538F48D2F8295807F829FC00D1124CD
:106C70000AC0C0978A30910530F49D2F9295907F7D
:106C8000989FC00D1124DD2311F0D0E0D2CF8C2FBE
:106C9000CC0F990B01C0CE01DF91CF911F910F91C5
:106CA000FF90EF9008950F931F93CF93DF93EC0124
:106CB0008B0165E574E00E944B1601151105B9F1D1
:106CC000F80161918F01662391F1603220F0623208
:106CD00011F06C3541F56CE5CE010E94FB14F80112
:106CE000319780818C30D1F044F48930D9F08A30EA
:106CF000B9F0883029F762E616C0823259F024F4E0
:106D00008D30F1F662E70FC08F3231F08C35C1F66D
:106D10006CE509C062E207C06FE205C066E603C029
:106D20006EE601C064E7CE010E94FB14C9CF62E2A7
:106D3000CE010E94FB1480E090E0DF91CF911F9183
:106D40000F9108950F931F93CF93DF930097B9F09E
:106D5000EC010C851D85D8018D919C91DC01ED9194
:106D6000FC910488F589E02D1995C8010E94EB5922
:106D7000CE01DF91CF911F910F910C94365BDF9183
:106D8000CF911F910F910895AF92BF92CF92DF9252
:106D9000EF92FF920F931F93CF93DF9300D01F9238
:106DA000CDB7DEB76115710509F493C06B01182FDB
:106DB000DB011C96AD90BC901D97F501E080F18041
:106DC000D701ED91FC910688F789E02DC70119954F
:106DD000811103C0C601B6DF7CC0F501928191111B
:106DE00014C0D701ED91FC910190F081E02D612F4D
:106DF000C7011995F7018589882309F467C0612FB8
:106E00008CE898E00E94FB1461C0812F8F7D815433
:106E10008A3138F380ED810F8A3018F383ED810FCA
:106E20008230F8F21F35E9F21E37D9F21132B1F093
:106E300086EC810F823090F08AED810F873070F000
:106E40001D3361F0812F8F7E8F3241F08DED810FE8
:106E5000823020F01B3511F01D3511F491FFC1CFA8
:106E600019821A821B821C82812F012E000C990B21
:106E70009F931F9387E594E09F938F938E010F5FFD
:106E80001F4F1F930F930E94BC660F900F900F909F
:106E90000F900F900F9083E0D82ED00ED701ED9178
:106EA000FC910190F081E02DD8016C91C7011995FA
:106EB000F7018589882331F0D8016C918CE898E03E
:106EC0000E94FB140F5F1F4FD012E8CF80E090E0CC
:106ED00002C08FEF9FEF0F900F900F900F90DF91F8
:106EE000CF911F910F91FF90EF90DF90CF90BF90C7
:106EF000AF900895CF92DF92EF92FF920F931F937E
:106F0000CF93DF938C017B0186E090E00E9456597D
:106F1000EC019093170580931605F801019000206D
:106F2000E9F7CF01801B910B0E9456596C01B80103
:106F30000E944066F80101900020E9F73197E01BBC
:106F4000F10BEC0DFD1D1082D982C882FB82EA8212
:106F500080910E0590910F059D838C83D0930F0532
:106F6000C0930E05DF91CF911F910F91FF90EF908D
:106F7000DF90CF9008958F929F92AF92BF92CF9261
:106F8000DF92EF92FF920F931F93CF93DF936115E0
:106F9000710509F4FBC0FB010085002E000C110BEC
:106FA000220B330B0730110508F0F0C0DB01EC01B8
:106FB000F8018827E552FF4F8F4F0C94BB656DE5B4
:106FC00074E006C019968C91882389F062E674E01B
:106FD000CE01DF91CF911F910F91FF90EF90DF9045
:106FE000CF90BF90AF909F908F900C94261567E63E
:106FF00074E0EECF19964D915D916D917C911C9747
:107000002AE030E0CE01DF91CF911F910F91FF90E8
:10701000EF90DF90CF90BF90AF909F908F900C94A7
:1070200083151996CD90DD90ED90FC901C9720E093
:1070300030E0A901C701B6010E948D6287FF09C037
:107040006DE674E0CE010E944B16F7FAF094F7F863
:10705000F094C701B6010E94FE624B015C012AE078
:10706000AB01BC01CE010E943B156FE674E0CE017E
:107070000E944B16C501B4010E942A639B01AC011A
:10708000C701B6010E9428622DEC3CEC4CE45DE3A4
:107090000E94296220E030E040E251E40E94E06377
:1070A0000E94FE62AB0160E070E02AE0CE010E9427
:1070B0003B156CC019966D917C911A97CE01DF91AA
:1070C000CF911F910F91FF90EF90DF90CF90BF90E5
:1070D000AF909F908F90E7CD16960D911C911797CA
:1070E0006BE5CE010E94FB14019619F48FEF9FEF20
:1070F0004FC00115110569F0B801CE013CDF0196C2
:10710000A9F3F801028113810115110591F36CE2D5
:10711000E8CF6DE52DC016960D911C9117976BE782
:10712000CE010E94FB14019609F301151105F9F037
:10713000F80160817181CE01B6DD0196B9F26AE392
:10714000CE010E94FB14019689F2B801CE0113DF33
:10715000019661F2F801028113810115110529F3ED
:107160006CE2CE010E94FB140196F9F6BFCF6DE7E9
:10717000CE010E94FB1421E030E0019611F020E0E6
:1071800030E088279927821B930B02C080E090E0B3
:10719000DF91CF911F910F91FF90EF90DF90CF90F3
:1071A000BF90AF909F908F900895CF93DF93EC01A5
:1071B000E881F9810284F385E02DCE0119958F3F96
:1071C0002FEF920771F0E881F9818132910594F3F4
:1071D0000684F785E02D682FCE01199580E090E0B8
:1071E00002C08FEF9FEFDF91CF910895EF92FF9252
:1071F0000F931F93CF93DF938C017B01DC01ED9103
:10720000FC910284F385E02D1995829749F584E07D
:10721000F701808786E090E00E945659EC01892BA7
:10722000F9F0E5EEF6E0F983E88380E091E0DF0134
:107230009C011D9221503040E1F79B838A831D827F
:107240001C82D801ED91FC910284F385E02DC801E8
:1072500019958F3FBFEF9B0731F4CE010E94EB5988
:107260008FEF9FEF70C08232910509F449C08032E0
:1072700091050CF445C08C35910511F0BE013EC05E
:10728000D801ED91FC910284F385E02DC801199598
:107290008F3FBFEF9B0709F38236910539F15CF40C
:1072A0008F32910501F18C359105D1F0829749F625
:1072B000BE0182E223C08E369105D9F03CF48636B9
:1072C000910509F0BECFBE018CE018C08237910550
:1072D00099F08437910509F0B4CFBE0189E00EC062
:1072E000BE018CE50BC0BE018FE208C0BE0188E084
:1072F00005C0BE018AE002C0BE018DE018DCA1CF4E
:107300008C819D81009749F0E881F9818E0F9F1F44
:10731000FC0131978081882319F0BE0180E007DCF1
:107320008C819D810E9456598C01009739F065EE41
:1073300076E00E944066CE010E94EB59F701128769
:10734000018780E090E0DF91CF911F910F91FF9036
:10735000EF90089569E277E08CE898E00C943B1692
:10736000CF93DF93C9E0D0E068EE73E080E090E077
:107370000E94F8174AE050E0BE018CE898E00E94B5
:107380001616219789F7DF91CF9108956F927F921A
:107390008F929F92AF92BF92CF92DF92EF92FF9225
:1073A0000F931F93CF93DF93CDB7DEB761970FB6DF
:1073B000F894DEBF0FBECDBF61E774E080917E0B15
:1073C00090917F0B0E947E428C010097D1F10E9428
:1073D0001C238230B1F560E0C8010E9471427C013B
:1073E00061E0C8010E947142DC0119960D911C9167
:1073F0001A97F701818521E090919205992309F46C
:10740000D5C2909170009E7F90937000109292056B
:1074100010920202109201028093000221110E9438
:10742000951AC8010E94BC1A67E878E08CE898E0D9
:107430000E9402154AE050E0B8018CE898E00E94F2
:10744000161665E774E080917E0B90917F0B0E9489
:107450007E429093EB078093EA07009709F4A7C058
:107460000E941C23082F10E00115110509F49FC08C
:10747000000F111F000F111FC8010E945659909351
:10748000E7078093E60710929B0510929A051092E9
:10749000ED071092EC071092990510929D0510923D
:1074A0009C050130F2E01F070CF489C2E12C72E068
:1074B000F72EC70101960E94565990939F0580931D
:1074C0009E0590939805809397058E0D9F1D909330
:1074D0009605809395050E9430186093240570935B
:1074E0002505809326059093270580E090E0E091A4
:1074F0009E05F0919F05E80FF91F10820196E8168E
:10750000F906ACF782E090E090939B0580939A0592
:1075100080E98093C9001092C8001092CD0083E0EA
:107520008093CC008EE08093CA00F0920502E09236
:10753000040220919E0530919F0580910402909154
:107540000502820F931F9093960580939505232B38
:1075500009F42EC265EE77E08CE898E00E940215EF
:107560004AE050E0B8018CE898E00E94161686E8E0
:1075700095E09093940580939305809136059091C2
:107580003705009739F0FC01EA5CFD4F8EE395E08A
:10759000918380836DE678E08CE898E00E94021584
:1075A0004AE050E0B8018CE898E00E94161600917D
:1075B0007E0B10917F0B6BE774E0C8019FD790930F
:1075C0002F0580932E05DC0116968D919C911797BF
:1075D00090932B0580932A0568E774E0C8018ED745
:1075E00090932D0580932C0561E874E0C80186D73F
:1075F000909331058093300568E874E0C8017ED728
:107600009093E9078093E8076DE874E0C80176D7A6
:10761000909334058093330561E678E08CE898E038
:107620000E943B166AE578E08CE898E00E9402151B
:1076300081E020912E0530912F05232B09F480E065
:107640000E943B4762E578E08CE898E00E940215D2
:1076500081E020912C0530912D05232B09F480E049
:107660000E943B476AE478E08CE898E00E940215AB
:1076700081E02091300530913105232B09F480E021
:107680000E943B4764E478E08CE898E00E94021591
:1076900081E02091E8073091E907232B09F480E08D
:1076A0000E943B476CE378E08CE898E00E9402156A
:1076B00081E02091330530913405232B09F480E0DB
:1076C0000E943B47E0913305F0913405309709F46F
:1076D00003C2809135058111FFC1E680F78081E109
:1076E00090E00E9456598C0188E1F8018183128252
:1076F0001082108A178610927D0610927C061092D6
:107700004106109263060E94073310931B050093F5
:107710001A0583E190E00E945659FC0188E891E344
:10772000928B818B168305831482108289E081837A
:1077300011E012831383F0932305E093220580EA7E
:1077400090E00E94565990931F0580931E0588E291
:1077500090E00E9456599093190580931805109255
:107760007D0610927C0610924106109263060E94DC
:10777000073380911A0590911B050E94353381E0F3
:107780000E946525811167C06DE178E08CE898E082
:107790000E943B16C0901A05D0901B05C6010E949E
:1077A000353340E060EFC60125D8C6010E94323370
:1077B000E0911A05F0911B0510836DEF77E08CE8DE
:1077C00098E00E943B1680911A0590911B050E943B
:1077D000C533882331F061EF77E08CE898E00E94B0
:1077E0003B1600912205109123050E9430184B0191
:1077F0005C01F0E18F0EF7E29F1EA11CB11CD801C5
:107800001596ED91FC9116978FEF83871486DF0113
:1078100013963B961D92AE17BF07E1F7F80114824D
:1078200077247394BE01665F7F4FD80115968D91C2
:107830009C91169702D818160CF4C3C08FEF9AE4E7
:1078400090931D0580931C05E0912205F09123057E
:10785000128281E001C080E08093350501E010E0F4
:1078600068E0B62EE114F10409F436C1F701808511
:10787000863009F097C0C080D180CE0101964C01BE
:10788000360190E1690E711CD6018C910E948830FE
:10789000A82EB2E0CB0ED11CF601319780810E9458
:1078A0008830A29450EFA5228A29F40181934F01D8
:1078B000C614D70449F7E0912005F0912105EE0F99
:1078C000FF1F8091180590911905E80FF91F11838A
:1078D0000083A0912005B091210523E0AA0FBB1FD2
:1078E0002A95E1F780911E0590911F05A80FB91FF9
:1078F000FE0131968B2D01900D928A95E1F767E399
:1079000078E08CE898E00E94021560912005709163
:1079100021054AE050E08CE898E00E94CA1560E337
:1079200078E08CE898E00E94021580912005909103
:10793000210533E0880F991F3A95E1F720911E0544
:1079400030911F05820F931F0E9444268CE898E017
:107950000E941316609120057091210543E0660F87
:10796000771F4A95E1F780911E0590911F05680FDA
:10797000791FDB018C91883261F48091220590910E
:1079800023050E94C22580911A0590911B050E9433
:10799000F033809120059091210501969093210567
:1079A00080932005F701E280F3805CCF20E034CDA6
:1079B0006EEC77E08CE898E00E943B16D8CD780119
:1079C00078CD0E943018681579058A059B0508F066
:1079D00035CF67E0CE010A960E9425339989891335
:1079E0006DC064EB73E08CE898E00E944B16D80100
:1079F0008C9181113AC015968D919C9116970E9499
:107A0000C533BE01665F7F4FF801858196810E9474
:107A1000D53440E064EBD80115968D919C91169772
:107A20000E94FA33F801C580D680C6010E94543303
:107A3000C6010E94353367E889E299E00E945A3115
:107A400060E889E299E00E945A31C6010E9432330F
:107A5000C6010E945433D82ED80115968D919C9161
:107A600016970E94C533D5FE30C0AE014F5F5F4F01
:107A7000BE01665F7F4FC8010E940035F801D180CA
:107A80008A85803129F1BE01665F7F4FC80122D807
:107A90008D1520F4D80111968C910AC08A85803109
:107AA00011F48CE005C0BE01665F7F4FC80112D89B
:107AB000F801818384818F5F8483B4CE6AEB73E0A5
:107AC0008CE898E00E944B16ADCED8017C92CDCFC9
:107AD000BCE0BD15F8F2E5CF61960FB6F894DEBFB5
:107AE0000FBECDBFDF91CF911F910F91FF90EF900F
:107AF000DF90CF90BF90AF909F908F907F906F90CE
:107B000008952F923F924F925F926F927F928F9241
:107B10009F92AF92BF92CF92DF92EF92FF920F931C
:107B20001F93CF93DF93CDB7DEB72B970FB6F894A3
:107B3000DEBF0FBECDBF8C012B0137DB019609F4F0
:107B4000C7C2D801ED91FC910284F385E02DC801F4
:107B500019957C018F3FBFEF9B0709F4B9C2D8018B
:107B6000ED91FC910684F785E02D682FC8011995E9
:107B7000B2E2EB16F10421F4B201C80137DBAAC26C
:107B8000EDE2EE16F10429F0C701C0970A9708F05C
:107B900045C1D801ED91FC910284F385E02DC80127
:107BA00019951C018F3FBFEF9B0709F491C28D9778
:107BB00081F4D801ED91FC910284F385E02DC80198
:107BC00019951C01019609F483C288248A94982C83
:107BD00003C088248394912CC101C097C12CD12C5F
:107BE0000A97C8F48AE0F82EFC9CC001FD9C900D19
:107BF0001124B101605371096C01C60ED71ED80162
:107C0000ED91FC910284F385E02DC80119951C01CA
:107C1000C0970A9748F3BEE22B163104C1F0C101A8
:107C20008F7D8534910599F0C89CC001C99C900D49
:107C3000D89C900D1124092E000CAA0BBB0BF2014D
:107C400081879287A387B48782E08087DDC0B601F1
:107C5000DD0C880B990B0E942C636B017C01FEE20A
:107C60002F163104B1F5D801ED91FC910284F38512
:107C7000E02DC80119951C01A12CB12C20E030E0A9
:107C800040E251E4C701B6010E94E0636B017C0150
:107C9000B10160537109072E000C880B990B0E94EB
:107CA0002C639B01AC01C701B6010E9429626B01E4
:107CB0007C01B1E0AB1AB108D801ED91FC910284CE
:107CC000F385E02DC80119951C01C0970A97B0F201
:107CD00002C0A12CB12CC1018F7D8534910509F022
:107CE00043C0D801ED91FC910284F385E02DC801D9
:107CF00019951C018B32910559F4D801ED91FC9135
:107D00000284F385E02DC80119951C01B1E00CC077
:107D10008D9761F4D801ED91FC910284F385E02DFB
:107D2000C80119951C01BFEFBE8302C0E1E0EE83DC
:107D3000612C712C4AE0C101C0978A309105C0F4D2
:107D4000469D9001479D300D11243901680E791E22
:107D5000D801ED91FC910284F385E02DC8014B8799
:107D600019951C014B85E7CFB1E0BE83612C712CC6
:107D7000B401990C880B990B0E942C63A701960102
:107D80000E94E0636B017C01B501BB0C880B990B71
:107D90000E942C634B015C01B301770C880B990B9B
:107DA0000E942C636F83788789879A87EE816E2F74
:107DB000EE0F770B880B990B0E942C639B01AC0193
:107DC0006F81788589859A850E94E0639B01AC016B
:107DD000C501B4010E9429629B01AC0160E070E022
:107DE00080E291E40E9443649B01AC01C701B601AB
:107DF0000E94E063D20119966D937D938D939C93BD
:107E00001C9783E018968C93D801ED91FC91068421
:107E1000F785E02D622DC801199521C0BBE5EB1651
:107E2000F10409F05CC0D801ED91FC910284F38566
:107E3000E02DC80119958B35910509F049C185E000
:107E4000F2018087C801B1D9D801ED91FC9102847B
:107E5000F385E02DC80119958D35910519F480E061
:107E600090E038C1D801ED91FC910684F785E02DB2
:107E7000682FC8011995DD24DA940E94BD107C0199
:107E8000009709F425C1DD2021F0F2019783868354
:107E900008C0D50113969C938E931297FC01B5826E
:107EA000A482C80182D9B701C8012BDE892B09F051
:107EB0000FC1C8017AD9D801ED91FC910284F385F4
:107EC000E02DC8011995D12C57018C329105A9F2EA
:107ED00021E030E08D35910509F082C07FC0BBE71D
:107EE000EB16F10409F081C0D801ED91FC910284F8
:107EF000F385E02DC80119958B37910509F0E8C08D
:107F000086E0F2018087C80150D9D801ED91FC913B
:107F10000284F385E02DC80119958D37910509F488
:107F20009ECFD801ED91FC910684F785E02D682F56
:107F3000C8011995BB24BA940E94BD107C0100971A
:107F400009F4C6C0BB2021F0F2019783868308C0E4
:107F5000D60113969C938E931297FC01D582C4820E
:107F6000C80123D9B701C80141D9019609F4B0C0AD
:107F7000C8011BD9D70119968D919C911A9711961A
:107F80009C938E931A961C921E921997D801ED918C
:107F9000FC910284F385E02DC8011995CA9709F078
:107FA00097C0C80102D9B701C801ABDD019609F439
:107FB0008FC0C801FAD8D801ED91FC910284F385F5
:107FC000E02DC8011995B12C67018C32910509F497
:107FD000B3CF21E030E08D37910511F420E030E09F
:107FE00088279927821B930B75C0BEE6EB16F10418
:107FF00011F519821A821B821C82D801ED91FC9125
:108000000484F585E02D44E050E0BE016F5F7F4FB2
:10801000C8011995049709F05BC044E050E06DE594
:1080200074E0CE0101960E945766009709F050C097
:10803000F20110864FC0F6E6EF16F10419F5CE01F5
:1080400001967C0185E0D7011D928A95E9F7D80158
:10805000ED91FC910484F585E02D45E050E0B701F9
:10806000C80119950597A1F545E050E067E674E071
:10807000C7010E945766009759F521E0F201208759
:10808000118628C0F4E7EF16F10411F519821A825F
:108090001B821C82D801ED91FC910484F585E02DB2
:1080A00044E050E0BE016F5F7F4FC801199504970F
:1080B00079F444E050E062E674E0CE0101960E945B
:1080C0005766009729F421E0F2012087218702C03A
:1080D0008FEF9FEF2B960FB6F894DEBF0FBECDBF8C
:1080E000DF91CF911F910F91FF90EF90DF90CF9094
:1080F000BF90AF909F908F907F906F905F904F90C8
:108100003F902F900895CF92DF92EF92FF92CF93FE
:10811000DF93EC010E9430186B017C0180914309D0
:1081200090914409DC01ED91FC910084F185E02DF2
:108130001995892B79F40E943018AB01BC014C19B8
:108140005D096E097F0948395A436105710530F3AD
:1081500080E00DC08091430990914409DC01ED91CC
:10816000FC910284F385E02D1995888381E0DF91ED
:10817000CF91FF90EF90DF90CF9008950F931F93D2
:10818000CF93DF93009781F08C010E94BD10EC012A
:10819000892B51F0C80109D8BE01C801B2DC019693
:1081A00031F4CE010E94C92480E090E001C0CE01EC
:1081B000DF91CF911F910F910895CF93DF93FC0131
:1081C00001900020E9F79F01281B390B285F3F4FE2
:1081D0002138310570F5EC010E94BC23882349F158
:1081E0008091C5099091C609019611F481E090E053
:1081F0009093C6098093C5098091C5099091C609DD
:1082000090934A0980934B0947E050E065E479E098
:10821000CE010E942A23FC01ED5BF64F1282AC01D5
:108220004450510965E479E082E8DF91CF910C94E4
:108230004B2380E0DF91CF9108959F92AF92BF9240
:10824000CF92DF92EF92FF920F931F93CF93DF9322
:10825000982E8B015A01690164E270E00E948C281B
:10826000E82EF12C65E270E0892D0E948C28FE2C0E
:10827000EE24E82AE701C00FD11F9E013770E92CD8
:10828000F12CC701880F991FAC014C59594F7A0145
:10829000FA0180819181820F931FA9014C0D5D1D10
:1082A0004130584090F000E018E0021B130BA80189
:1082B000B5010E941611A601401B510BB501600FBC
:1082C000711FF7018081918102C0A601B5010E9452
:1082D0001611CC0DDD1D4D2F64E270E0892D0E943A
:1082E00082284C2F65E270E0892DDF91CF911F919C
:1082F0000F91FF90EF90DF90CF90BF90AF909F9045
:108300000C948228FF920F931F93CF93DF93F82E44
:10831000C0E0D0E08F2D0E94CD108C01892B21F080
:108320008F2D0E94CD10EC01C017D10799F7CE0117
:10833000DF91CF911F910F91FF9008955F926F92FF
:108340007F928F929F92AF92BF92CF92DF92EF92E5
:10835000FF920F931F93CF93DF931F92CDB7DEB79A
:108360004C0185E499E0CFDE811125C021C00F5F6B
:108370001F4F8981F801ED5BF64F8183282F2F77FE
:1083800030E02C9DA0012D9D500D3C9D500D1124E1
:10839000A40EB51E37E0CC0CDD1CEE1CFF1C3A957C
:1083A000D1F787FF14C0CE010196ADDE8111DFCF7A
:1083B00080E090E085C070904509198201E010E0EE
:1083C000A12CB12CC12CD12C7601C394ECCF872DDC
:1083D000807F55245394803309F0512C8FEF800F08
:1083E000D4018C93552011F1C8018B5B964F8BDE25
:1083F0008823F1F2C8018A5B964F85DE8823C1F29B
:108400000E5F1F4FD401EC91F0E0ED5BF64FE3807F
:10841000F12CFE2CEE248481E80EF11C809145099C
:1084200081FF08C0B2E0EB0EF11C04C080E0E12C3B
:10843000F12C01C082E0C82ED12CC01AD10A9EEFC7
:10844000692E77247A94C601800F911F8A159B05A7
:1084500060F5CE01019657DE882309F4A9CF8091FB
:10846000DC099091DD090097A9F0552099F0F401FD
:108470002081A301421B51099A01200F311FE216EE
:10848000F30640F4DC01ED91FC910190F081E02DC8
:10849000698119950038110528F48981F801ED5B8F
:1084A000F64F82830F5F1F4FCECF8091DC099091F2
:1084B000DD09892B21F40138110508F079CFC801B5
:1084C0000F90DF91CF911F910F91FF90EF90DF9070
:1084D000CF90BF90AF909F908F907F906F905F9064
:1084E0000895FC0186819781009739F0662329F071
:1084F0006150FC0182819381F7CF08950F931F9300
:10850000CF93DF938B01FC01C681D781209759F06F
:10851000B801888199810E940E66892B21F00A801A
:10852000DB81C02DF3CFCE01DF91CF911F910F9151
:108530000895CF93DF939B01672B61F4E0918C0842
:10854000F0918D080190F081E02D682F8CE898E083
:10855000199508C0482F50E060E070E08CE898E082
:108560000E943B15EC018CE898E00E9413168C0FDA
:108570009D1FDF91CF910895DC011696ED91FC913E
:10858000179761157105A1F0309729F417967C9320
:108590006E931697089582819381009711F0FC01E4
:1085A000FACF73836283DB011596FC93EE931497E5
:1085B0000895CF93DF931F92CDB7DEB76983DC01B7
:1085C000ED91FC910280F381E02D41E050E0BE018D
:1085D0006F5F7F4F19950F90DF91CF910895DC0168
:1085E000ED91FC91068CF78DE02D199591E089278E
:1085F0000895862F089581E086270895CF92DF920F
:10860000EF92FF920F931F93CF93DF93CDB7DEB717
:10861000E1970FB6F894DEBF0FBECDBF7C016A01B3
:1086200001E313E01A8309831B821C821D821E82D0
:10863000CE01099668AB79AB0E9401281DA30CA35B
:108640001EA21FA218A619A6809137099091380979
:10865000A0913909B0913A098CA79DA7AEA7BFA7F1
:108660008B839C83AD83BE8318861F82AE014C5DD5
:108670005F4F68A979A9CE0101960E94982C81309C
:108680009105B1F4D701ED91FC910684F785E02DB9
:108690001BA70AA78EA19FA1A8A5B9A58CA79DA7D6
:1086A000AEA7BFA7A601BE01665D7F4FC7011995A2
:1086B000E1960FB6F894DEBF0FBECDBFDF91CF912C
:1086C0001F910F91FF90EF90DF90CF90089544E0BD
:1086D00050E0BC018FE090E00C94161108958CBD21
:1086E0009DBD08958F929F92AF92BF92CF92DF92DD
:1086F000EF92FF920F931F93CF936C015B017A016E
:10870000FC01C485C43041F481E090E0F60193831C
:10871000828380E090E049C08A014130584010F0E7
:1087200000E018E080E590E0DADF8C2FEBDD4C0113
:1087300063E070E08C2F0E948C28873111F08C311F
:1087400021F48016910670F302C000E010E080E58D
:1087500090E0C5DF9801A50160E070E08C2F6DDD31
:1087600060E270E08C2F0E94F32462E070E08C2FB6
:108770000E948C2884FD0FC063E070E08C2F0E9463
:108780008C28811104C08C2F0E942312BDCF80E55C
:1087900090E0A5DFEACF40E162E070E08C2F0E941C
:1087A0008228012B09F4B0CFC701CF911F910F91FF
:1087B000FF90EF90DF90CF90BF90AF909F908F9001
:1087C0000895CF92DF92FF920F931F93CF93DF9381
:1087D000FC012485243009F076C06A01EB018C018C
:1087E000F12C8F2D0E94EE12811103C0F801F48646
:1087F00007C08B7F8831D1F3F394F4E0FF12F1CFFF
:10880000F8018485843009F45EC02091060230911D
:1088100007022F5F3F4F11F420E030EC3093070246
:1088200020930602409106025091070220E061E089
:108830000E943712F801F4848A818F3F51F48B81B2
:108840008F3F91F48C818F3F79F48D818F3F61F45C
:1088500037C0811109C08B81811106C08C818111C3
:1088600003C08D81882361F1C114D10449F180E5F1
:1088700090E035DFBE016E5F7F4F8F2D90E0982F27
:10888000882744E050E0845F9B4F0E941611B60198
:108890008F2D0E94E52864E070E08F2D0E94F32464
:1088A000C8010E943329873189F061E070E080E0DF
:1088B00090E00E94F817C8010E9433298111F0CF7F
:1088C00084E0F801848780E090E002C081E090E0DD
:1088D000DF91CF911F910F91FF90DF90CF9008957E
:1088E0000F931F93CF93DF93EB0185E195E09F9367
:1088F0008F9384E195E09F938F9383E195E09F931D
:108900008F9382E195E09F938F9381E195E09F9310
:108910008F9380E195E09F938F9380E994E09F93FC
:108920008F938B818F938A818F930E94EC662DB7F2
:108930003EB7205F3F4F0FB6F8943EBF0FBE2DBF2E
:10894000069784F46FEE78E08CE898E00E940215B8
:108950006A817B818CE898E0DF91CF911F910F9124
:108960000C942B16ECD300E115E0C0E0D0E0F80148
:1089700061918F01CE010E94BD612196C630D10563
:10898000B1F761E079E08CE898E0DF91CF911F9139
:108990000F910C943B16CF93DF93CDB7DEB72C9796
:1089A0000FB6F894DEBF0FBECDBF1C821B821E82A5
:1089B0001D828FEF9FEF98878F838DE393E09A83DB
:1089C000898388E290E09A8789871C861B866FEDF1
:1089D00078E08CE898E00E943B1660917E0B7091E5
:1089E0007F0BCE0101960E94BB376FEFCE0101963F
:1089F0000E94161069ED78E08CE898E00E943B1622
:108A00002C960FB6F894DEBF0FBECDBFDF91CF918D
:108A10000895CF93DF93CDB7DEB769970FB6F8947B
:108A2000DEBF0FBECDBF8FE290E0A0E0B0E0898353
:108A30009A83AB83BC83FE01359685E1DF011D92ED
:108A40008A95E9F765EC78E08CE898E00E943B169F
:108A5000AE014E5F5F4F66E080E195E00E949C3082
:108A60001E8665EA74E0CE0101960E942166BE0171
:108A70006F5F7F4F8CE898E00E942B16CE01019625
:108A80009CDB1E866DEA74E0CE0101960E94216691
:108A9000BE016F5F7F4F8CE898E00E942B1667EB5A
:108AA00074E0CE0101960E94F1230E94261B699674
:108AB0000FB6F894DEBF0FBECDBFDF91CF91089502
:108AC0008F929F92AF92BF92CF92DF92EF92FF92DE
:108AD0000F931F93CF93DF93CDB7DEB7C554D10962
:108AE0000FB6F894DEBF0FBECDBF809115051F9263
:108AF0008F93809114051F928F93809113051F927D
:108B00008F93809112051F928F93809111051F9270
:108B10008F93809110051F928F9389EB94E09F9320
:108B20008F931F9280E28F93CE0101967C019F93D9
:108B30008F930E947F6661EC79E08CE898E00E9458
:108B40003B16B7018CE898E00E942B16FE01EF5B04
:108B5000FF4F80EC808388EA818388E5828382E00E
:108B600083831CA21BA288EE93E0A0E0B0E08DA35B
:108B70009EA3AFA3B8A784E08DA783E593E09AA353
:108B800089A384EE94E09FA78EA7F9ABE8AB80E5BC
:108B900090E09BAB8AAB1EAA6BEB75E384EC96E38B
:108BA0000E944C5B8C010FB6F894DEBF0FBECDBFA8
:108BB000892B71F183E090E00E945659F801958766
:108BC00084875E01F1E2AF0EB11CDC011196BC920C
:108BD000AE9212961C92C5010E943B29882319F07F
:108BE000C5010E945E298AA89BA868A979A96E017F
:108BF000B7E3CB0ED11CC6010E944C16A401B601EE
:108C0000C501DFDD892B09F088C0C8010E94A236AA
:108C100000E010E0ECA8FDA80115110509F45EC004
:108C2000E8ECEE16F10409F04BC066EB79E08CE855
:108C300098E00E943B161AAE19AE1CAE1BAE8FEF29
:108C40009FEF9EAF8DAF89E793E098AF8FAB2196F2
:108C50001FAF0EAF219780917E0B90917F0B0E94EA
:108C6000C924CE01C7968ADA90937F0B80937E0B3E
:108C7000C8010E94A23680917E0B90917F0B0097D5
:108C800079F460EA79E08CE898E00E943B160E9453
:108C90003018DC01CB018856954CAF4FBF4F32C026
:108CA0000E948A248C01BC018CE898E00E942B165B
:108CB000C8010E94EB590E94C63982E090E0C4C00E
:108CC00068E879E08CE898E00E9402154AE050E0FC
:108CD000B7018CE898E00E9416160CC066E779E0B0
:108CE0008CE898E00E943B166EE579E08CE898E00D
:108CF0000E943B160E943018DC01CB0188579C4E25
:108D0000AF4FBF4F80937A0B90937B0BA0937C0B5C
:108D1000B0937D0B85EF9FEF97C0BEA4AFA4FF92E9
:108D2000EF928AE599E09F938F931F930F930E9490
:108D3000D45BFF92EF9285E599E09F938F931F9309
:108D40000F930E94D45BD8011C96ED91FC911D9766
:108D500081E08283FF92EF9282E599E09F938F9367
:108D60001F930F930E94D45BD8011C96ED91FC9148
:108D70001D971282AF92BF928CE199E09F938F93DF
:108D80001F930F930E94D45B87E599E09F938F9385
:108D90001F930F930E94D45B1DAA1CAAD8011C9696
:108DA000ED91FC911D97A080B1800FB6F894DEBFC5
:108DB0000FBECDBF83E3E82EF12CD501ED91FC91E0
:108DC0000084F185E02DC501199541975CF4B1E06F
:108DD000EB1AF10839F064E170E080E090E00E9465
:108DE000F817EBCFDF92CF9280E199E09F938F93BA
:108DF0001F930F930E94F05B0F900F900F900F90B6
:108E00000F900F90019709F005CF8FA998AD9DABFA
:108E10008CAB20E080E08A3021F08D3031F0282FBB
:108E200004C02A3009F4F6CE2AE0C80126962FAFF6
:108E300026970E94965B26962FAD26978F3F59F76F
:108E4000C8010E94A236E6CECB5BDF4F0FB6F89486
:108E5000DEBF0FBECDBFDF91CF911F910F91FF906D
:108E6000EF90DF90CF90BF90AF909F908F9008953C
:108E700027DE0C94261B882319F069E079E002C0F4
:108E80006CE079E08CE898E00C943B16CF93DF938C
:108E9000CDB7DEB72C970FB6F894DEBF0FBECDBFAF
:108EA00066EB78E08CE898E00E943B161C821B82FF
:108EB0001E821D828FEF9FEF98878F838DE393E053
:108EC0009A83898388E290E09A8789871C861B862B
:108ED00080917E0B90917F0B0E94C924CE01019658
:108EE0004DD990937F0B80937E0B8CE898E00E9485
:108EF000131680917E0B90917F0B892B49F463EAC6
:108F000078E08CE898E00E943B1680E090E00AC090
:108F10006FEA78E08CE898E00E943B160E94C63920
:108F200081E090E02C960FB6F894DEBF0FBECDBF67
:108F3000DF91CF910895AADF0C94261B089580E05D
:108F400090E008958F929F92AF92BF92CF92DF925E
:108F5000EF92FF920F931F93CF93DF93CDB7DEB7BE
:108F6000A5970FB6F894DEBF0FBECDBF5C018B0195
:108F70007B01E40EF51ED7011C9266ED79E08CE8CA
:108F800098E00E940215B5018CE898E00E944B160B
:108F900061EF74E08CE898E00E944B16FE01319678
:108FA0006F012091860B3091870B2115310511F44B
:108FB00020E93BE0C601821B930B8A3F91053CF4FC
:108FC00061ED79E08CE898E00E943B16A5C019821B
:108FD0001A821B821C82FE01359680E1DF011D9200
:108FE0008A95E9F748018E149F0441F0F4016191DC
:108FF0004F018CE898E00E94FB14F5CF8CE898E0D4
:109000000E941316C8010E94440E7C016FE270E0BA
:10901000C5010E947466009741F0BC016F5F7F4FED
:1090200043E150E0C6010E946566B601CE01459657
:109030000E944807CE0145960E940C06882309F439
:109040006BC0E114F10469F03CF4FEEFEF16FFEFA2
:10905000FF060CF061C056C021E0E216F10471F188
:1090600051C06E018EE1C80ED11CE12CF12C96018D
:1090700001151105F1F0B3E0EB16F104D1F09FEF0B
:10908000E91AF90AC8012CA33DA30E94D85A5C0131
:109090006CE270E0C8010E942C668C012CA13DA1FD
:1090A000892B11F00F5F1F4FD601AD92BD926D015C
:1090B000DFCF00E0A70160E070E02AC00E94301816
:1090C0000091800B1091810B2091820B3091830BCA
:1090D000DC01CB01801B910BA20BB30B853F9140B0
:1090E000A105B10540F000E020E030E040E050E0B4
:1090F00061E070E00DC064EF74E08CE898E00E94DD
:109100002B160AC000E020E030E040E050E0B7015C
:10911000CE0145960E946107A5960FB6F894DEBF72
:109120000FBECDBFDF91CF911F910F91FF90EF90B8
:10913000DF90CF90BF90AF909F908F9008951F9336
:10914000CF93DF936CEE79E08CE898E00E940215F3
:10915000C0E1D5E01C2F1A5F499150E060E070E05B
:1091600020E18CE898E00E943B156AEE79E08CE8FB
:1091700098E00E9402151C13EFCF8CE898E0DF9175
:10918000CF911F910C941316AF92BF92CF92DF92A2
:10919000EF92FF920F931F93CF93DF9300D000D0F5
:1091A000CDB7DEB76AED79E08CE898E00E94021551
:1091B0008E010D5F1F4F7E0187E0E80EF11C580104
:1091C00081E3C82E83E0D82EDA82C9821B821C82FA
:1091D0001D821E8280E590E082DA44E050E0B50115
:1091E0008FE090E00E94EC1079DAF80141918F0154
:1091F00050E060E070E02AE08CE898E00E943B15C7
:1092000068ED79E08CE898E00E9402150E151F05C4
:10921000D9F68CE898E00E94131626960FB6F894BB
:10922000DEBF0FBECDBFDF91CF911F910F91FF9099
:10923000EF90DF90CF90BF90AF9008958F929F9264
:10924000AF92BF92CF92DF92EF92FF920F931F9354
:10925000CF93DF93F62EB72EE42EA52ED22E932E8B
:10926000C02E812EBC0180912E0590912F0546D9EC
:10927000EC01892B09F447C08885853009F043C08B
:1092800060E0CE012ED98C0161E0CE012AD9FC012B
:10929000C185D285D80119968D919C911A978230FB
:1092A000910551F087309105B1F0019761F56C2D72
:1092B000CE0103960E94F11A6F2DCE010E94F11A81
:1092C0006E2DCE0101960E94F11A6D2DCE010296EF
:1092D0000E94F11A18C03097B1F08085853099F45A
:1092E000C681D781209779F00C2D182D2D2D392D81
:1092F0004E2D5A2D6F2D7B2D89859A859FDF0A80F3
:10930000DB81C02DEFCFDF91CF911F910F91FF90A7
:10931000EF90DF90CF90BF90AF909F908F90089587
:109320005F926F927F928F929F92AF92BF92CF92F5
:10933000DF92EF92FF920F931F93CF93DF93CDB7FE
:10934000DEB7E4970FB6F894DEBF0FBECDBF5C0169
:109350007B016A01890119A21AA21BA21CA2FE01AB
:10936000B5968CE0DF011D928A95E9F760E473E021
:10937000CE0101960E94FD5AD5011296ED91FC9105
:1093800013976081718140E250E0CE0101960E9406
:109390004766B2E0EB16F104A1F054F4E114F104D5
:1093A000B9F0EA94EF2809F076C06DEE73E00BC0D7
:1093B00085E0E816F10429F099E0E916F10441F09E
:1093C0006AC060EF73E0CE0181960E94406645C09E
:1093D0000115110509F441C0612C712C8FEFA82EE5
:1093E00084E0B82E94E0592E7E01A1E3EA0EF11C30
:1093F0004601B1E08B1A91086C147D0474F5F801F4
:10940000808191810E5F1F4F9F938F93BF92AF9288
:109410001F925F92FF92EF920E947F6640E150E0C0
:10942000B701CE0181960E9447660FB6F894DEBF61
:109430000FBECDBF6814790461F062E075E0C7012A
:109440000E94406640E150E0B701CE0181960E9443
:1094500047669FEF691A790ACFCFBE016F5F7F4FD2
:109460008CE898E00E944B166EEC79E08CE898E06E
:109470000E940215BE016F5D7F4F8CE898E00E944C
:109480002B16BE016F5D7F4FCE0101960E94F12326
:1094900080E090E002C08FEF9FEFE4960FB6F89463
:1094A000DEBF0FBECDBFDF91CF911F910F91FF9017
:1094B000EF90DF90CF90BF90AF909F908F907F9074
:1094C0006F905F900895EF92FF920F931F93CF9349
:1094D000DF9300D000D0CDB7DEB78C017B0162E016
:1094E00070E00E947506892B19F4E982FA8205C0A2
:1094F0008F2D880F880BF9828A83A981BA81BB27B7
:1095000024E630E00E94CA652FE330E040E050E0FE
:109510000E94ED613A832983C8012B833C834D83EC
:109520005E830E94A106E82EF12CC8010E9451061C
:109530002B813C814D815E816217730784079507FB
:1095400079F4672B682B692B09F44AC082E0E8168E
:10955000F10471F085E0E816F10409F041C008C09B
:10956000232B242B252B41F182E0E816F104F9F49A
:1095700020E030E040E050E061E070E0C801D0DE83
:109580009E012F5F3F4F41E050E060E070E0C80176
:10959000C7DE61E0C8010E948C0649815A81052E10
:1095A000000C660B770BC8010E94190619C085E0F4
:1095B000E816F10429F7DCCF85E0E816F10481F024
:1095C00082E0E816F10461F062E0C8010E948C06B6
:1095D00020E030E040E050E062E070E0C801A0DE52
:1095E00080E090E026960FB6F894DEBF0FBECDBFA8
:1095F000DF91CF911F910F91FF90EF900895AF925F
:10960000BF92CF92DF92EF92FF920F931F93CF936F
:10961000DF93CDB7DEB7C154D1090FB6F894DEBFE2
:109620000FBECDBFCB018A014EE459E46CE470E07B
:1096300049835A836B837C83FE0135962CE1DF01DD
:109640001D922A95E9F74AAB5BAB6CAB7DABF1960B
:109650002CE0DF011D922A95E9F7AE014F5D5F4FC7
:1096600068E00E949C301AAABE016F5D7F4F809116
:109670003305909134050E947E427C01009771F180
:1096800068EE73E00E947E42FC01C184D284C11462
:10969000D104C9F041E150E0B601CE0181960E94AB
:1096A0006566B6018CE898E00E944B1667ED73E0A2
:1096B0008CE898E00E944B164AE050E0B8018CE834
:1096C00098E00E94161669ED73E0C7010E947E4281
:1096D000DC011996ED90FC901A9708C06CE07AE0D6
:1096E0008CE898E00E943B16E12CF12C0138BFEF8A
:1096F0001B0709F4C3C00535110509F4BFC06DEFA0
:1097000079E0CE0101960E94FD5A40E250E0BE0190
:109710006F5D7F4FCE0101960E9447661F930F93A6
:109720008FEF94E09F938F936E01E2E3CE0ED11CF6
:10973000DF92CF920E94BC66B601CE0101960E94D4
:10974000F1230F900F900F900F900F900F90E11456
:10975000F10409F493C080912E0590912F05009794
:1097600009F48CC0B7010E947E427C01009709F485
:1097700085C0DC0118968C91853009F07FC060E0CF
:10978000C7010E947142FC0181859285A385B48541
:109790000597A105B10509F071C0C7010E941C23FE
:1097A000843008F46BC08430B1F50E94BD106C01A8
:1097B000892B21F085E0D60118968C930E94BD106C
:1097C0005C01892B59F082E0F5018087012E000CA5
:1097D000220B330B01871287238734870E94BD1029
:1097E0008C01892B59F082E0F801808788EC90E0A9
:1097F000A0E0B0E081879287A387B487B501C60156
:109800000E94BC42B801C6010E94BC42B601C70119
:109810000E94BC4233C064E0C7010E9471426C01E7
:10982000009761F161E00E9471425C0160E0C60155
:109830000E947142012E000C220B330BDC011996A1
:109840000D931D932D933C931C97F5018185928573
:10985000A385B485892B8A2B8B2B39F4D7016D9185
:109860007C9184E095E00E94F12388EC90E0A0E0F8
:10987000B0E0F50181879287A387B487CF5BDF4F84
:109880000FB6F894DEBF0FBECDBFDF91CF911F9111
:109890000F91FF90EF90DF90CF90BF90AF90089521
:1098A0002F923F924F925F926F927F928F929F92F0
:1098B000AF92BF92CF92DF92EF92FF920F931F93DE
:1098C000CF93DF9300D0CDB7DEB72DB63EB60E9462
:1098D000BC23982E882309F442C10E9430186B01E2
:1098E0007C018091CB099091CC09A091CD09B091D8
:1098F000CE09A7019601281B390B4A0B5B0BDA0135
:10990000C90189399A43A105B105A8F48091C70915
:109910009091C809A091C909B091CA09A7019601FF
:10992000281B390B4A0B5B0BDA01C90189399A43B1
:10993000A105B105D0F12091CF0980914309909103
:109940004409222379F02CEF3FEF3093DF09209375
:10995000DE09DC01ED91FC910488F589E02D199573
:10996000912CFDC020EC2093450910924609DC01A2
:10997000ED91FC910280F381E02D42E050E065E43E
:1099800079E01995C092C709D092C809E092C90937
:10999000F092CA09C092CB09D092CC09E092CD09CD
:1099A000F092CE0981E08093CF0980914309909194
:1099B0004409DC01ED91FC910084F185E02D1995BD
:1099C000892B09F4CCC0CE0101960E949E418C01E6
:1099D000892B09F4C4C0C092CB09D092CC09E09283
:1099E000CD09F092CE0970904509872D807F803394
:1099F00009F09AC0E091D009F091D109FB83EA8384
:109A0000EF2B09F4ACC04DB65EB6A981B0E0CD0134
:109A10008D5B964FFC01638170E0762F6627848111
:109A2000680F711DCB0101962DB73EB7281B390B6E
:109A30000FB6F8943EBF0FBE2DBF4DB75EB74F5F58
:109A40005F4F5A0120E030E02617370769F0C9015F
:109A50008A0F9B1F8D5B964FFC018581FA018193D4
:109A6000AF012F5F3F4FF0CFC501820F931FFC0165
:109A70001082F72DF6708F2E42E0F4133EC0B9012C
:109A80006A0F7B1FAB014D5B564FFA01858190E059
:109A9000982F882746813C01640E711C4BEF5FEFC5
:109AA0004A1B5B0B421B530B400F511F665B764FEB
:109AB000C501EA81FB81199580E480934509809274
:109AC0004609709247096092480980914309909134
:109AD0004409DC01ED91FC910280F381E02D44E02A
:109AE00050E065E479E01995C092C709D092C809A1
:109AF000E092C909F092CA0911C04DEF5FEF4A1B0D
:109B00005B0B421B530B400F511F2A0F3B1FB90128
:109B1000685B764FC501EA81FB8119950FB6F89411
:109B20005EBE0FBE4DBE1BC0803CA9F480ED80938D
:109B30004509109246098091430990914409DC013E
:109B4000ED91FC910280F381E02D42E050E065E46C
:109B500079E0199504C0803D11F41092CF09892D48
:109B60000FB6F8943EBE0FBE2DBE0F900F900F9013
:109B7000DF91CF911F910F91FF90EF90DF90CF90E9
:109B8000BF90AF909F908F907F906F905F904F901D
:109B90003F902F900895FC0182819381A481B5812B
:109BA0008093D4099093D509A093D609B093D7098F
:109BB0008BE597E09093DB098093DA091092D9093D
:109BC0001092D80983E499E00895CF93DF93CDB73D
:109BD000DEB7C956D1090FB6F894DEBF0FBECDBFB0
:109BE000789484B5826084BD84B5816084BD85B578
:109BF000826085BD85B5816085BD80916E00816084
:109C000080936E0010928100809181008260809329
:109C1000810080918100816080938100809180002B
:109C20008160809380008091B10084608093B10056
:109C30008091B00081608093B0008091910082603B
:109C40008093910080919100816080939100809138
:109C500090008160809390008091A1008260809349
:109C6000A1008091A10081608093A1008091A0005B
:109C700081608093A0008091210182608093210106
:109C80008091210181608093210180912001816078
:109C90008093200180917A00846080937A00809183
:109CA0007A00826080937A0080917A00816080934C
:109CB0007A0080917A00806880937A001092C100C7
:109CC00088E395E0909375058093740510920F05D5
:109CD00010920E0526E040E052EC61E070E08CE866
:109CE00098E00E9400176BE672E08CE898E00E9412
:109CF0003B1686E0E2E1F2E0DE01DD9601900D9296
:109D00008A95E1F760E1C62E65E0D62EE12CF12CB4
:109D100000E010E0C8010E94B561D6018D936D018D
:109D200081508E3F18F4EE24E394F12C0F5F1F4F07
:109D30000630110579F7EF2879F462E572E08CE8D6
:109D400098E00E943B1686E0FE01FD96A0E1B5E09A
:109D500001900D928A95E1F7F2D961E08DE00E94C1
:109D6000BC1726E040E855E260E070E08FEE97E037
:109D70000E9400178BE79CE29093F50A8093F40A07
:109D80008CE89CE29093F70A8093F60A80E99CE2C3
:109D90009093F90A8093F80A64E170E080E090E023
:109DA0000E94F81710923505E0911A05F0911B05F5
:109DB000309721F081E79CE2908B878781E393E0E5
:109DC0009A8389838091FC0A9091FD0AA091FE0AF2
:109DD000B091FF0A8B839C83AD83BE83CE01019635
:109DE000DADE82EA97E49093D1098093D0098091DA
:109DF000360590913705892B59F488E392E00E944B
:109E000056598C010E94012810933705009336059E
:109E10008091360590913705009739F0FC01EA5C96
:109E2000FD4F8EE395E0918380836AEA79E38BE8C6
:109E300093E00E947A376BEC74E480E993E00E942F
:109E40007A376BE977E485E993E00E947A3768E333
:109E500077E48AE993E00E947A3760E774E48EE958
:109E600093E00E947A3760EB79E382EA93E00E9404
:109E70007A3769E075E487EA93E00E947A37EE2446
:109E8000E394F12CA8958CE898E00E947C13892B30
:109E900009F493C08CE898E00E945A13182F8A3076
:109EA00031F08D3021F0883009F076C060C0E0914B
:109EB0007405F091750510826BEA73E08CE898E008
:109EC0000E944B1663ED73E088E395E00E94045B0B
:109ED0009A838983FE0133966F0101E010E0B02E72
:109EE000A12E63ED73E080E090E00E94045BD60158
:109EF0008D939D936D010E31110539F40091160576
:109F000010911705C980DA8008C00F5F1F4F892B99
:109F100031F7F4CFF8010481158101151105A1F085
:109F2000F80160817181C6010E943766892B91F723
:109F3000D8011296ED91FC911397BE016F5F7F4F90
:109F40008B2D9A2D199506C062E972E08CE898E095
:109F50000E943B168CE898E00E94131662EA72E0B9
:109F60008CE898E00E94021588E395E010C068E054
:109F70008CE898E00E94FB1480917405909175051F
:109F8000F5E088339F0709F008F47DCF019790939F
:109F900075058093740577CF682F8CE898E00E9450
:109FA000FB14E0917405F0917505CF010196909333
:109FB000750580937405108366CF0E942C1B029751
:109FC0004CF06EDC8091360590913705009711F0CA
:109FD0000E94A41980913505882309F48BC28091D1
:109FE000330590913405892B09F484C20E943018FE
:109FF000009178051091790520917A0530917B05C3
:10A00000601771078207930708F474C20E94301822
:10A010002B013C018091220590912305009709F4C2
:10A0200057C2209176053091770560912005709197
:10A030002105261737070CF42CC10E9430189B010C
:10A04000AC0128573C4E4F4F5F4FAA962CAF3DAF07
:10A050004EAF5FAFAA976FEC72E08CE898E00E9479
:10A060003B16E0911A05F0911B05309739F4E09109
:10A070001805F091190580E090E00BC08FEF838701
:10A080001486DF0113963B961D92AE17BF07E1F7CA
:10A09000EECF2091200530912105821793070CF017
:10A0A00081C0208131812E7F219331930196F1CFA0
:10A0B0006091200570912105A3E0660F771FAA9596
:10A0C000E1F720911E0530911F05620F731F0E945A
:10A0D0001D3418160CF022C6C0902005D090210522
:10A0E000B4E1CB16D1040CF019C60E943018AA9620
:10A0F0002CAD3DAD4EAD5FADAA97621773078407D7
:10A10000950708F00BC6A0901E05B0901F054601EC
:10A1100033E0880C991C3A95E1F78A0C9B1C67E0A8
:10A12000C4010E942533D40117969C9189133AC02B
:10A1300000E010E00C151D05ECF548E050E0B4011E
:10A14000C5010E940166B8E0AB0EB11C892BC9F5B0
:10A15000000F111FE0911805F0911905E00FF11F94
:10A160008081918181609183808368EC72E08CE8CA
:10A1700098E00E940215809120059091210523E02E
:10A18000880F991F2A95E1F720911E0530911F0530
:10A19000820F931F0E94442661EC72E08CE898E0E5
:10A1A0000E943B1680911A0590911B05009709F0BB
:10A1B0007FCFB4C58091220590912305892B21F48E
:10A1C000F1CF0F5F1F4FB6CF8091200590912105F1
:10A1D000880F991F2091180530911905F901E80F92
:10A1E000F91F21E030E0318320836CEB72E08CE8D2
:10A1F00098E00E94021560912005709121054AE0C7
:10A2000050E08CE898E00E94CA1565EB72E08CE89B
:10A2100098E00E940215809120059091210513E09D
:10A22000880F991F1A95E1F720911E0530911F059F
:10A23000820F931F0E9444268CE898E00E94131618
:10A24000609120057091210503E0660F771F0A9544
:10A25000E1F780911E0590911F05680F791FDB01C2
:10A260008C91883261F480912205909123050E949F
:10A27000C22580911A0590911B050E94F0338091B0
:10A28000200590912105019690932105809320054A
:10A2900089CF00911E0510911F05A901F3E0440F1D
:10A2A000551FFA95E1F7040F151FD8014C9148325C
:10A2B00009F003C1AE01435C5F4FB8010E945935FC
:10A2C000882379F16DADB8E06B9FB00111242EADFC
:10A2D00030E0322F2227330F330F330F262B372B4B
:10A2E000F8018081803101F525966FAD259770E0EA
:10A2F00024968FAD2497AB01481B5109CA0196954E
:10A30000982F8827979587950E94A86560517109B5
:10A31000207F53E0220F331F5A95E1F7620F731F1E
:10A3200004C060E874EE01C0B901613854EE7507ED
:10A330006CF0072E000C880B990B0E942C6320E018
:10A3400030E040E05CE30E94E06304C060E070E065
:10A350008EEF92EC0E94F962E0911C05F0911D05D0
:10A360003097A1F00091760510917705980193E060
:10A37000220F331F9A95E1F7A0911E05B0911F059A
:10A380002A0F3B1FAB01B901C80119950091760551
:10A390001091770583E0000F111F8A95E1F78091F6
:10A3A0001E0590911F05080F191FC0902205D0901F
:10A3B0002305D8018C91803149F0B801C6010E9473
:10A3C0006A35B82E882309F46CC002C0BCE0BB2EED
:10A3D000F601858196810E94C533882309F461C006
:10A3E000B801D60115968D919C9116970E94D5348F
:10A3F000F601408164E4858196810E94FA33D6019A
:10A4000012968C91882309F44CC0E7EFEB0DE330F2
:10A4100040F4F0E0EE0FFF1FE85EFD4F208031803A
:10A4200004C07EEE272E72E0372E0115110599F13A
:10A43000F6018381882379F1808181112CC00E94EB
:10A4400030184B015C019101330C440B550BAA965B
:10A450002CAF3DAF4EAF5FAFAA97AE01435C5F4FED
:10A46000B801C6010E9400358DAD81111AC00E944D
:10A470003018DC01CB01AA962CAD3DAD4EAD5FADE1
:10A48000AA97821B930BA40BB50B88159905AA05F7
:10A49000BB0518F306C0B101330C880B990B0E9461
:10A4A000F81780917605909177050196909377053E
:10A4B0008093760564EC79E00DC02F5F3F4F3093B9
:10A4C00077052093760580ED97E00E94A86502C08D
:10A4D0006FEF7FEFCB01770FAA0BBB0B480E591E16
:10A4E0006A1E7B1E409278055092790560927A052B
:10A4F00070927B050E94301880912405909125056B
:10A50000A0912605B09127050E948C0E8091300500
:10A5100090913105892B09F4DDC280912E0590912F
:10A520002F05892B09F4D6C20E94301800917C05B2
:10A5300010917D0520917E0530917F050617170744
:10A540002807390708F0C6C2D12C9AE0292E312CF1
:10A5500023E1422E512C34E0A32EB12C4EE3842E65
:10A5600048E0942E00912A0510912B050115110544
:10A5700009F4B0C2D110AEC2D80118968C918530C2
:10A5800009F091C260E0C8010E947142FC0181851E
:10A590009285A385B48584309105A105B10529F084
:10A5A0000997A105B10509F07EC222E232E06F965B
:10A5B0003FAF2EAF6F97A1961FAF0EAFA197CE0101
:10A5C000835A9F4F0E94AE06A6968FADA697843001
:10A5D00021F0893009F4A5C054C2809128059091DA
:10A5E0002905892B09F04DC2F0922905E092280532
:10A5F00060E070E0CE01835A9F4F0E9475063C01D7
:10A6000061E070E0CE01835A9F4F0E9475066C0195
:10A6100026E240E855E260E070E08FEE97E00E94AD
:10A6200000176092E2098FEE97E09093E109809322
:10A63000E0091092ED0A1092EF0A1092EE0AD09201
:10A64000E409C092E309F092E609E092E50983E0AB
:10A650000E944B20182F811118C00091E70910911A
:10A66000E8096FEE72E08CE898E00E94021540E184
:10A6700050E0B8018CE898E00E941616B801CE01AF
:10A68000835A9F4F0E94634A0DC069ED72E08CE8C7
:10A6900098E00E94021560E170E0812F0E949942CB
:10A6A00000E010E01092290510922805E0912A059B
:10A6B000F0912B058281938142E252E05EAF4DAF73
:10A6C00021969FAF8EAF2197CE01CD960E94AE0608
:10A6D00080912A0590912B05892B09F4D2C1CE01D6
:10A6E000CD960E940C06882309F4CBC126968FAD27
:10A6F0002697843009F0C5C160E070E0CE01CD96A8
:10A700000E9475068615970509F0BBC161E070E0EF
:10A71000CE01CD960E9475068C159D0509F0B1C13C
:10A7200014C38091280590912905892B09F0A9C1AE
:10A73000F0922905E09228050E94BD108C01892B1A
:10A7400021F086E0D80118968C9360E473E0CE0186
:10A75000CD9653D7A196EEADFFADA19760817181E3
:10A760004FE150E0CE01CD960E9447666EEA73E05D
:10A77000CE01CD960E94216626E040E855E260E0D9
:10A7800070E08FEE97E00E94001760E070E0CE016D
:10A79000835A9F4F0E9475068093E2098FEE97E0DF
:10A7A0009093E1098093E0091092ED0A1092EF0A6C
:10A7B0001092EE0AE4E3F8E0F093E409E093E30991
:10A7C0003092E6092092E50983E00E944B20D82EC2
:10A7D00081117BC066E373E08CE898E00E9402156B
:10A7E00067EEC62E69E0D62ED6016D917D916D0182
:10A7F00040E150E08CE898E00E94CA1564E373E001
:10A800008CE898E00E940215BBEFCB16B9E0DB069E
:10A8100059F76091EB097091EC09072E000C880B39
:10A82000990B0E942C6320E030E048EC52E40E9437
:10A8300091629B01AC0164EB73E0C8010E943F246C
:10A840004091EF095091F00966EB73E0C8010E9456
:10A8500011206091F1097091F209072E000C880B0C
:10A86000990B0E942C6320E030E048EC52E40E94F7
:10A8700091629B01AC016AEB73E0C8010E943F2426
:10A880006091F3097091F409072E000C880B990B65
:10A890000E942C6320E030E040E251E40E9491628B
:10A8A0009B01AC0168EB73E0C8010E943F2440911A
:10A8B000E7095091E8096CEB73E0C8010E94112090
:10A8C0008CE898E00E9413160BC06EE173E08CE8F0
:10A8D00098E00E94021560E170E08D2D0E9499427F
:10A8E0008091E70983FF12C09092E4098092E30906
:10A8F000F092E609E092E50983E00E944B20811185
:10A900000CC04091E7095091E80902C040E050E0D6
:10A910006FEB73E0C8010E94112062E370E080E0F9
:10A9200090E00E94F8175092E4094092E309B09237
:10A93000E609A092E50983E00E944B20D82E811100
:10A9400083C064E173E08CE898E00E94021557EE42
:10A95000C52E59E0D52EF601619171916F014AE043
:10A9600050E08CE898E00E94CA1562E173E08CE840
:10A9700098E00E940215FFEECF16F9E0DF0659F7C6
:10A980006091E7097091E80961157105C9F0072E1A
:10A99000000C880B990B0E942C632DEE3EE94CE3D2
:10A9A0005EE30E94E06322E538EB42E152E40E945C
:10A9B00028629B01AC016EE973E0C8010E943F244C
:10A9C0006091E9097091EA09072E000C880B990B38
:10A9D0000E942C632DEE3EE94CE35EE30E94E063AF
:10A9E00022E538EB42E152E40E9428629B01AC016F
:10A9F00062EB73E0C8010E943F246091ED09709101
:10AA0000EE0916161706A4F4072E000C880B990BF6
:10AA10000E942C6320E030E040E251E40E94916209
:10AA20009B01AC0163EC73E0C8010E943F2407C0A6
:10AA300040E050E063EC73E0C8010E9411208CE814
:10AA400098E00E9413160BC06CEF72E08CE898E05F
:10AA50000E94021560E170E08D2D0E949942C801AC
:10AA60000E948A246C01BC01CE01CD960E94F12384
:10AA7000C601B1D4C8010E94C924109229051092C0
:10AA800028050E943018DC01CB018053984FAF4F4E
:10AA9000BF4F80937C0590937D05A0937E05B09376
:10AAA0007F05DD24D394E0912A05F0912B05828166
:10AAB000938190932B0580932A05892B09F052CD21
:10AAC000E0912E05F0912F058681978190932B05BB
:10AAD00080932A0500912E0510912F05011511056F
:10AAE00009F47BC00E943018809080059090810509
:10AAF000A0908205B090830586169706A806B90631
:10AB000008F06BC0D80116960D911C91179701158E
:10AB1000110509F43FC0F80180858530A9F560E092
:10AB2000C8010E947142FC0181859285A385B4858C
:10AB30000597A105B10541F5C8010E941C23853088
:10AB400018F161E0C8010E947142FC01318462E0A9
:10AB5000C8010E947142DC011996AD90BC901A9711
:10AB600063E0C8010E947142FC018184928464E028
:10AB7000C8010E9471426C01892B31F0C6010E940C
:10AB80001C23823008F0FEC0D80112960D911C9152
:10AB90001397BDCF0E943018DC01CB0188579C4E23
:10ABA000AF4FBF4F8093800590938105A09382059E
:10ABB000B0938305BE01635C7F4F8091860B9091BB
:10ABC000870B009711F480E99BE0681B790B4AE042
:10ABD00050E08CE898E00E94161600912C05109128
:10ABE0002D050115110509F496C00E9430188090BA
:10ABF000840590908505A0908605B09087058616FF
:10AC00009706A806B90608F086C0F801C680D78066
:10AC100083E0282EC114D10409F46EC0D601189621
:10AC20008C91863009F062C063E074E0C6010E9436
:10AC30007E42009719F0FC01018501C000E0D601B9
:10AC40008D919C91B5D4182F6EEC73E0C6010E94D3
:10AC50007E425C01892B49F560ED73E08CE898E059
:10AC60000E944B16412F50E060E070E02AE08CE833
:10AC700098E00E943B1565ED73E08CE898E00E9437
:10AC80004B166AE070E0802F0E94994240E050E04D
:10AC90006EEC73E0C6010E9411206EEC73E0C601F9
:10ACA0000E947E425C01892B09F11123F9F007FF14
:10ACB00017C160E0812F0E94BC17812F0E94651789
:10ACC00033243394019709F017C1632C712CF501DB
:10ACD0008485082E000C990B6816790609F49FC12B
:10ACE0008385882309F40AC181508387D60112968F
:10ACF000CD90DC9013978ECF0E943018DC01CB01F1
:10AD0000C296A11DB11D8093840590938505A093E3
:10AD10008605B09387050E942214B4C866EA72E0E3
:10AD20008CE898E00E940215609120057091210541
:10AD30004AE050E08CE898E00E94161610927705E1
:10AD40001092760560E47FE1C5CBB801CE01CD96C7
:10AD50000E94634AE0912A05F0912B05828193813C
:10AD600090932B0580932A05892B09F08ACEE091D8
:10AD70002E05F0912F058681978190932B05809366
:10AD80002A057FCE60E0C6010E947142DC0119965F
:10AD90004D905D906D907C901C9761E0C6010E9483
:10ADA0007142FC012185328543855485D8016D911E
:10ADB0007C91211531054105510559F48CE898E045
:10ADC0000E944B1667E773E08CE898E00E943B1600
:10ADD00013C02150310941095109DC0119962D9305
:10ADE0003D934D935C931C97232B242B252B21F40F
:10ADF00087EC93E00E94F123A8965FAE4EAEA89731
:10AE0000F801608171818CE898E00E944B1661E73F
:10AE100073E08CE898E00E9402154AE050E0B5012A
:10AE20008CE898E00E94CA1567E673E08CE898E029
:10AE30000E9402154AE050E0B2018CE898E00E94BE
:10AE4000CA1561E673E08CE898E00E9402154AE0BA
:10AE500050E0B4018CE898E00E94CA1561E0832DAF
:10AE60000E94BC17F2E08F16910489F025E082164B
:10AE7000910469F061E0C6010E947142FC01818584
:10AE80009285A385B485892B8A2B8B2B59F460E09E
:10AE9000832D0E948D176CE573E08CE898E00E948A
:10AEA0003B1672CEB2E04B0E511C4A145B043CF4CC
:10AEB00061E0832D0E948D1768E573E0EECFA896C0
:10AEC0002EAD3FADA8972A153B053CF060E0832DE1
:10AED0000E948D1763E573E0E0CF6FE473E0DDCF90
:10AEE00062E0812F0E94BC17812F0E9465173324D6
:10AEF0003394892B09F4E9CE312CE7CE412F50E071
:10AF000060E070E02AE08CE898E00E943B1567ED75
:10AF100073E08CE898E00E944B164AE050E0B301E1
:10AF20008CE898E00E94161669ED73E0C6010E9455
:10AF30007E422C016EED73E0C6010E947E424C0100
:10AF400063EE73E0C6010E947E428C0168EE73E0FE
:10AF5000C6010E947E42FC01892BF1F0611471044C
:10AF600041F08114910419F46DEE73E011C0D40125
:10AF700007C00115110519F460EF73E009C0D8018D
:10AF800019966D917C911A97DB018C91882321F0A1
:10AF9000818592850E94F12341145104E1F1F2016F
:10AFA00061857285CE01CD960E944807CE01CD966F
:10AFB0000E940C06882379F1672869F081149104B6
:10AFC00041F401E020E030E040E050E061E070E07A
:10AFD0001EC0D4010CC00115110541F401E020E0B0
:10AFE00030E040E050E062E070E011C0D801199616
:10AFF0008D919C911A97FC012081222361F00E947F
:10B00000440E01E020E030E040E050E0BC01CE0121
:10B01000CD960E946107D5011C963C9267CEF50142
:10B02000238664CE0F931F93E0E0FBE081E393E07F
:10B03000918380831282138214821582EFEEF7E0EF
:10B040001382128248EE53E060E070E0448355833F
:10B05000668377832BEA32E031832083A5EDB0E06D
:10B06000B587A487A4EDB0E0B787A687A0EDB0E0D0
:10B07000B18BA08BA1EDB0E0B38BA28BA2EDB0E0C1
:10B08000B58BA48BA6EDB0E0B78BA68B118E128E7C
:10B09000138E148EECE8F8E01382128244835583F9
:10B0A000668377833183208325EC30E035872487DE
:10B0B00024EC30E03787268720EC30E0318B208B82
:10B0C00021EC30E0338B228B22EC30E0358B248B6B
:10B0D00026EC30E0378B268B118E128E138E148E59
:10B0E000E6E0FBE02FEF20831282118214861386A4
:10B0F0000FEF1FEF98010783108721873287E3E165
:10B10000FBE0918380831282138214821582E9E22C
:10B11000F9E01382128244835583668377832DEB93
:10B1200032E031832083E9E1FBE091838083128266
:10B13000138214821582EFE1FBE0918380831282F7
:10B14000138214821582E5E2FBE0918380831282F0
:10B15000138214821582EBE2FBE0918380831282DA
:10B16000138214821582E1E3FBE0918380831282D3
:10B17000138214821582E7E3FBE0918380831282BD
:10B18000138214821582EDE3FBE0918380831282A7
:10B19000138214821582E5E3F9E0918380831282A1
:10B1A000138214821582EDE3F9E091838083128289
:10B1B000138214821582E3E4FBE091838083128280
:10B1C000138214821582E9E4FBE09183808312826A
:10B1D000138214821582EFE4FBE091838083128254
:10B1E000138214821582E2E6FBE09183808312824F
:10B1F000138214821582EAEFFAE09183808320ECB7
:10B20000228328EA238328E5248322E025831092E1
:10B21000F50A1092F40A1092F70A1092F60A1092A8
:10B22000F90A1092F80AE5E5FBE0138212824483E2
:10B230005583668377832BE033E03183208324E0DA
:10B2400024879093D3098093D2091092D409109245
:10B25000D5091092D6091092D7092FEF3FEF3093FE
:10B26000DF092093DE09F0934409E093430910922B
:10B27000DD091092DC09E8E6FBE09183808312820D
:10B28000138214821582EEE6FBE0918380831282A2
:10B29000138214821582E4E7FBE09183808312829B
:10B2A0001382148215821F910F910895CF93DF931B
:10B2B0008230910510F482E090E0E091880BF091EB
:10B2C000890B20E030E0C0E0D0E0309711F1408100
:10B2D000518148175907C0F04817590761F4828116
:10B2E0009381209719F09B838A832BC09093890BBD
:10B2F0008093880B26C02115310519F0421753079A
:10B3000018F49A01BE01DF01EF010280F381E02D04
:10B31000DCCF2115310509F1281B390B243031050B
:10B3200090F412968D919C9113976115710521F0FF
:10B33000FB019383828304C09093890B8093880BD5
:10B34000FD01329644C0FD01E20FF31F81939193FA
:10B35000225031092D933C933AC02091860B3091B5
:10B36000870B232B41F420910A0230910B0230937A
:10B37000870B2093860B209108023091090221153A
:10B38000310541F42DB73EB740910C0250910D02AA
:10B39000241B350BE091860BF091870BE217F30726
:10B3A000A0F42E1B3F0B2817390778F0AC014E5F35
:10B3B0005F4F2417350748F04E0F5F1F5093870BE0
:10B3C0004093860B8193919302C0E0E0F0E0CF01BF
:10B3D000DF91CF9108950F931F93CF93DF93009741
:10B3E00009F48CC0FC013297138212820091880B01
:10B3F0001091890B0115110581F420813181820F93
:10B40000931F2091860B3091870B2817390779F508
:10B41000F093870BE093860B71C0D80140E050E0B9
:10B42000AE17BF0750F412962D913C911397AD01C2
:10B430002115310509F1D901F3CF9D01DA013383DB
:10B44000228360817181860F971F8217930769F4A9
:10B45000EC0128813981260F371F2E5F3F4F318342
:10B4600020838A819B8193838283452B29F4F093E7
:10B47000890BE093880B42C01396FC93EE931297CE
:10B48000ED01499159919E01240F351FE217F307F1
:10B4900071F480819181840F951F029611969C937F
:10B4A0008E938281938113969C938E931297E0E002
:10B4B000F0E0D80112968D919C911397009719F0A6
:10B4C000F8018C01F6CF8D919C9198012E5F3F4F32
:10B4D000820F931F2091860B3091870B2817390715
:10B4E00069F4309729F41092890B1092880B02C0EE
:10B4F000138212821093870B0093860BDF91CF91FA
:10B500001F910F9108958F929F92AF92BF92CF9209
:10B51000DF92EF92FF92CF93DF93EC016881798104
:10B520008A819B81611571058105910521F464E291
:10B5300079ED8BE597E02DE133EF41E050E04DD719
:10B5400049015A019B01AC01A7EAB1E462D76B0142
:10B550007C01ACEEB4EFA501940167D7DC01CB010F
:10B560008C0D9D1DAE1DBF1DB7FF03C00197A10926
:10B57000B04888839983AA83BB83BC01CD019F77A0
:10B58000DF91CF91FF90EF90DF90CF90BF90AF9081
:10B590009F908F900895B7CF8EE092E0B4CF6093E4
:10B5A0000E0270930F02809310029093110208957F
:10B5B000FC0188279927E89421912032E9F329306A
:10B5C00010F02E30C8F32B3239F02D3231F468945C
:10B5D00003C044D0820F911D219120532A30C8F31B
:10B5E0001EF4909581959F4F08959111E4C5803286
:10B5F00019F089508550D0F70895FB01DC010590C2
:10B600000D920020E1F7089544E85BE000C0FA01E4
:10B61000A191B081009719F41097E1F0CD01DC0100
:10B62000CD010D90002011F4C00113C0FB01219148
:10B63000222319F02015D9F7F3CFFB012191201512
:10B6400019F41E92119606C02223C1F70D90002016
:10B65000A1F7D001FA01A193B08308957AE0979FF2
:10B66000902D879F802D910D11240895FC01238139
:10B6700027FF0FC0EAE8FBE0208131812817390756
:10B6800011F41182108232962BE0E039F207A1F713
:10B69000A2DE80E090E008950F931F93CF93DF9395
:10B6A000009731F46115710519F480E090E039C01C
:10B6B0008B01EC016EE070E081E090E062D5FC016E
:10B6C000892B99F380E883830115110571F01387A5
:10B6D000028781E8838380918A0B90918B0B892B61
:10B6E00021F4F0938B0BE0938A0B2097C9F0D1875C
:10B6F000C08783818260838380918C0B90918D0BB6
:10B70000892B71F4F0938D0BE0938C0B80918E0B51
:10B7100090918F0B892B21F4F0938F0BE0938E0B7C
:10B72000CF01DF91CF911F910F910895CF93DF93B8
:10B73000EC012B8120FF33C026FF0AC02F7B2B8317
:10B740008E819F8101969F838E838A8190E029C09C
:10B7500022FF0FC0E881F9818081082E000C990B2F
:10B76000009719F420622B831AC03196F983E8837D
:10B770000EC0EA85FB85199597FF09C02B810196BC
:10B7800011F080E201C080E1822B8B8308C02E8102
:10B790003F812F5F3F4F3F832E83992702C08FEF5A
:10B7A0009FEFDF91CF9108950F931F93CF93DF9376
:10B7B000CDB7DEB708851985F8018381886083835A
:10B7C000AE01445F5F4F6A857B85C80125D0F801D3
:10B7D0002381277F2383DF91CF911F910F910895BC
:10B7E0000F931F93CF93DF93CDB7DEB708851985ED
:10B7F000F801838188608383AE01445F5F4F6A856F
:10B800007B85C8019ED3F8012381277F2383DF91A5
:10B81000CF911F910F9108952F923F924F925F9277
:10B820006F927F928F929F92AF92BF92CF92DF9250
:10B83000EF92FF920F931F93CF93DF93CDB7DEB7B5
:10B840002C970FB6F894DEBF0FBECDBF7C016B0105
:10B850008A01FC0117821682838181FFB0C1CE016B
:10B8600001964C01F7019381F60193FD859193FFB9
:10B8700081916F01882309F49EC1853239F493FDCB
:10B88000859193FF81916F01853221F4B70190E09A
:10B89000BDD4E8CF512C312C20E02032A0F48B32E3
:10B8A00069F030F4803259F0833269F420612CC0A1
:10B8B0008D3239F0803339F4216026C02260246053
:10B8C00023C0286021C027FD27C030ED380F3A3053
:10B8D00078F426FF06C0FAE05F9E300D1124532E47
:10B8E00013C08AE0389E300D1124332E20620CC024
:10B8F0008E3221F426FD5FC1206406C08C3611F41F
:10B90000206802C0883641F4F60193FD859193FFCB
:10B9100081916F018111C1CF982F9F7D95549330F4
:10B9200028F40C5F1F4FFFE3F9830DC0833631F01D
:10B93000833771F0833509F057C021C0F801808149
:10B9400089830E5F1F4F44244394512C540114C02B
:10B950003801F2E06F0E711CF801A080B18026FF63
:10B9600003C0652D70E002C06FEF7FEFC5012C872B
:10B9700042D42C0183012C852F77222E16C038014A
:10B98000F2E06F0E711CF801A080B18026FF03C0A9
:10B99000652D70E002C06FEF7FEFC5012C8719D4D1
:10B9A0002C012C852068222E830123FC19C0832DB5
:10B9B00090E048165906A0F4B70180E290E026D442
:10B9C0003A94F5CFF50127FC859127FE81915F011F
:10B9D000B70190E01BD431103A94F1E04F1A5108AE
:10B9E0004114510479F7DEC0843611F0893631F5FF
:10B9F000F80127FF07C060817181828193810C5F0C
:10BA00001F4F08C060817181072E000C880B990BB5
:10BA10000E5F1F4F2F76722E97FF09C0909580956D
:10BA2000709561957F4F8F4F9F4F2068722E2AE04F
:10BA300030E0A4013CD4A82EA81843C0853729F4CF
:10BA40002F7EB22E2AE030E025C0F22FF97FBF2EE4
:10BA50008F36C1F018F4883579F0ADC0803719F011
:10BA6000883721F0A8C02F2F2061B22EB4FE0DC060
:10BA70008B2D8460B82E09C024FF0AC09F2F9660CA
:10BA8000B92E06C028E030E005C020E130E002C059
:10BA900020E132E0F801B7FE07C060817181828148
:10BAA00093810C5F1F4F06C06081718180E090E040
:10BAB0000E5F1F4FA401FBD3A82EA818FB2DFF7704
:10BAC0007F2E76FE0BC0372D3E7FA51450F474FEFA
:10BAD0000AC072FC08C0372D3E7E05C0BA2C372D37
:10BAE00003C0BA2C01C0B52C34FF0DC0FE01EA0D15
:10BAF000F11D8081803311F4397E09C032FF06C008
:10BB0000B394B39404C0832F867809F0B39433FDC3
:10BB100012C030FF06C05A2CB31418F4530C5B1833
:10BB2000B32CB31460F4B70180E290E03C876ED38D
:10BB3000B3943C85F6CFB31410F43B1801C0312CFC
:10BB400034FF11C0B70180E390E03C875FD33C85B0
:10BB500032FF16C031FD03C088E790E002C088E5DF
:10BB600090E0B7010CC0832F867851F031FF02C0FE
:10BB70008BE201C080E237FD8DE2B70190E046D351
:10BB8000A51430F4B70180E390E040D35A94F8CF85
:10BB9000AA94F401EA0DF11D8081B70190E036D33B
:10BBA000A110F6CF332009F45DCEB70180E290E01A
:10BBB0002DD33A94F7CFF7018681978102C08FEF9A
:10BBC0009FEF2C960FB6F894DEBF0FBECDBFDF916E
:10BBD000CF911F910F91FF90EF90DF90CF90BF908A
:10BBE000AF909F908F907F906F905F904F903F901D
:10BBF0002F90089520FD09C0FC0123FD05C022FF00
:10BC000002C07383628351834083089544FD10C052
:10BC100046FD10C0DB01FC01AA0FBB1FEE1FFF1F7A
:10BC20001094D1F76A0F7B1F8E1F9F1F31E003C056
:10BC300033E001C034E0660F771F881F991F315031
:10BC4000D1F7620F711D811D911D08950F931F93F0
:10BC5000CF93DF938C01C80169DDEC0197FD06C02D
:10BC6000C4DC892BC1F7B801CE0108D3CE01DF9126
:10BC7000CF911F910F9108958F929F92AF92BF9293
:10BC8000CF92DF92EF92FF920F931F93CF93DF93A8
:10BC90001F92CDB7DEB78C01C62E7A01298346DD0F
:10BCA000AC01552729814B32510521F04D32510508
:10BCB00061F42068CA94C11002C080E06FC0C8015E
:10BCC000298334DD298197FDF8CF322F3D7FD32E94
:10BCD000322F307339F5803329F5BB24BA94BC0C6C
:10BCE00009F449C0C801298321DD298197FD43C09A
:10BCF000382F3F7D383561F48D2D8264D82ECA945B
:10BD0000CA94CC20C1F1C80111DD97FF0BC033C02C
:10BD100026FF04C02D2D2260D22E03C03D2D32619E
:10BD2000D32ECB2C812C912C540120ED280F2830C0
:10BD300078F0D4FE03C0B801A1D21AC02A3040F076
:10BD4000D6FEF9CF2F7D3FEE320F3630A0F72750C9
:10BD50004D2DC501B4015ADF4B015C018D2D826070
:10BD6000D82ECA94CC2051F0C801E0DC97FFDDCF7B
:10BD7000D1FC04C0A2CF812C912C5401D7FE08C065
:10BD8000B094A09490948094811C911CA11CB11C2F
:10BD90002D2DB501A401C7012DDF81E00F90DF91AA
:10BDA000CF911F910F91FF90EF90DF90CF90BF90B8
:10BDB000AF909F908F9008956F927F928F929F92F5
:10BDC000AF92BF92CF92DF92EF92FF920F931F93A9
:10BDD000CF93DF93CDB7DEB7A1970FB6F894DEBF50
:10BDE0000FBECDBF5C017A01CE0101966C0180E2ED
:10BDF000F60111928A95E9F7F501838040E050E061
:10BE0000912C712C70E0A1E0B0E0F90183FC8591E8
:10BE100083FE81918F01982F9F01811103C080E0E3
:10BE200090E07AC08E3519F44115510549F1E72F9C
:10BE3000F0E0E417F5073CF48D3559F18D3219F433
:10BE4000772001F103C0711001C0982E892F8695CB
:10BE5000869586958601080F111D892F87703D01F3
:10BE600001C0660C8A95EAF7F801808186298083F3
:10BE7000991559F0991510F49F5FE8CF9150E6CFCE
:10BE800071E004C07724739401C0712C4F5F5F4F41
:10BE9000BCCF772019F08E8180628E83711103C030
:10BEA0009924939416C0F6019E012F5D3F4F808127
:10BEB00080958193E217F307D1F7F2CFE114F104F3
:10BEC00029F0F7018083C70101967C016150912C14
:10BED000E9F0C50169A32ADC69A197FD15C0282FE7
:10BEE000269526952695F601E20FF11D208130E07A
:10BEF000AC014770552702C0359527954A95E2F762
:10BF000020FDDCCFB501BAD1911089CFE114F10445
:10BF100011F0F7011082C801A1960FB6F894DEBFA8
:10BF20000FBECDBFDF91CF911F910F91FF90EF908A
:10BF3000DF90CF90BF90AF909F908F907F906F9049
:10BF400008954F925F927F928F929F92AF92BF928D
:10BF5000CF92DF92EF92FF920F931F93CF93DF93D5
:10BF60001F92CDB7DEB76C012B015A01FC0117827D
:10BF70001682712CF601F380F201F3FC8591F3FE39
:10BF80008191382F2F01882309F4E5C090E039838F
:10BF90002CDB3981892B19F0C60158DEEBCF353205
:10BFA00041F4F201F3FC3591F3FE31912F0135326A
:10BFB00059F4C6013983BADB398197FDCAC03817F5
:10BFC000C9F2B6015BD1C7C03A3239F4F3FC3591FE
:10BFD000F3FE31912F0151E001C050E0420110E029
:10BFE00020ED230F2A3088F45260612F70E080E04A
:10BFF00090E040E259830ADE162FF401F3FC3591FC
:10C00000F3FE31914F015981EBCF052F232F2401EE
:10C0100051FF03C0111102C09EC01FEF383619F046
:10C020003C3659F011C0F401F3FC2591F3FE219147
:10C030002F01283649F4052F08600460F201F3FC53
:10C040002591F3FE21912F01222309F484C0622F50
:10C0500070E086E492E02983B1D02981892B09F42C
:10C060007AC000FD07C0F501E080F180C5010296AD
:10C070005C0102C0E12CF12C2E3649F4F601468118
:10C08000578160E070E0202FC701B4DD73CF233605
:10C0900089F401FF11E0C60149DB97FD5AC0E114A4
:10C0A000F10429F0F7018083C70101967C0111504A
:10C0B00091F74BC02B3551F49201A701612FC601B6
:10C0C0007BDE2C01892B09F040C03AC0C6012983D0
:10C0D000BDDD298197FD3DC02F3641F128F424367E
:10C0E00019F1293631F124C0233769F02537E1F001
:10C0F0001FC0E114F10429F0F7018082C701019605
:10C100007C01115059F0C60111DB4C0197FD06C0AE
:10C110006CDA892B71F3B601C401B0D0E114F104DB
:10C12000A1F0F701108211C0006203C0006101C0DC
:10C130000064202FA701612FC6019EDD811105C07B
:10C14000F6018381807329F406C000FD13CF739438
:10C1500011CF772019F0872D90E002C08FEF9FEF6D
:10C160000F90DF91CF911F910F91FF90EF90DF9093
:10C17000CF90BF90AF909F908F907F905F904F90A7
:10C1800008950F931F93CF93DF93869F8001879F1E
:10C19000100D969F100D1124C80188D8EC0100974E
:10C1A00021F0A80160E070E01FD0CE01DF91CF91B7
:10C1B0001F910F910895992788270895FC010590F4
:10C1C000061621F00020D9F7C00108953197CF015C
:10C1D0000895FC010590615070400110D8F78095DA
:10C1E00090958E0F9F1F0895DC0101C06D93415003
:10C1F0005040E0F70895FC0161507040019001103B
:10C20000D8F7809590958E0F9F1F08950F931F93D9
:10C21000CF93DF93FB01238121FD03C08FEF9FEFBD
:10C2200028C022FF16C046815781248135814217DC
:10C23000530744F4A081B1819D012F5F3F4F3183AB
:10C2400020838C93268137812F5F3F4F378326834E
:10C2500010C0EB01092F182F0084F185E02D1995EE
:10C26000892BE1F68E819F8101969F838E83812F9A
:10C27000902FDF91CF911F910F910895FB012381A2
:10C2800020FF12C026FD10C08F3F3FEF930761F0E3
:10C2900082832F7D206423832681378121503109B9
:10C2A00037832683992708958FEF9FEF0895FA012A
:10C2B000AA27283051F1203181F1E8946F936E7FE5
:10C2C0006E5F7F4F8F4F9F4FAF4FB1E03ED0B4E0D6
:10C2D0003CD0670F781F891F9A1FA11D680F791F17
:10C2E0008A1F911DA11D6A0F711D811D911DA11D28
:10C2F00020D009F468943F912AE0269F1124301938
:10C30000305D3193DEF6CF010895462F4770405DD2
:10C310004193B3E00FD0C9F7F6CF462F4F70405D81
:10C320004A3318F0495D31FD4052419302D0A9F7DC
:10C33000EACFB4E0A6959795879577956795BA95D6
:10C34000C9F700976105710508959B01AC010A2E9C
:10C3500006945795479537952795BA95C9F7620F73
:10C36000731F841F951FA01D0895F999FECF92BDDC
:10C3700081BDF89A992780B50895262FF999FECFA7
:10C380001FBA92BD81BD20BD0FB6F894FA9AF99AF2
:10C390000FBE01960895A1E21A2EAA1BBB1BFD0138
:10C3A0000DC0AA1FBB1FEE1FFF1FA217B307E40794
:10C3B000F50720F0A21BB30BE40BF50B661F771FEC
:10C3C000881F991F1A9469F76095709580959095CC
:10C3D0009B01AC01BD01CF010895052E97FB16F41A
:10C3E00000940FD057FD05D0D6DF07FC02D046F4ED
:10C3F00008C050954095309521953F4F4F4F5F4F66
:10C40000089590958095709561957F4F8F4F9F4FC0
:10C4100008950FD0A59F900DB49F900DA49F800DFF
:10C42000911D11240895B7FFF4CFF3DF821B930B06
:10C430000895A29FB001B39FC001A39F700D811DFD
:10C440001124911DB29F700D811D1124911D08951D
:10C450005058BB27AA270ED075C166D130F06BD1DA
:10C4600020F031F49F3F11F41EF45BC10EF4E0950F
:10C47000E7FB51C1E92F77D180F3BA176207730741
:10C480008407950718F071F49EF58FC10EF4E095BE
:10C490000B2EBA2FA02D0B01B90190010C01CA017E
:10C4A000A0011124FF27591B99F0593F50F4503E29
:10C4B00068F11A16F040A22F232F342F4427585F1B
:10C4C000F3CF469537952795A795F0405395C9F733
:10C4D0007EF41F16BA0B620B730B840BBAF09150EB
:10C4E000A1F0FF0FBB1F661F771F881FC2F70EC08A
:10C4F000BA0F621F731F841F48F48795779567955D
:10C50000B795F7959E3F08F0B3CF9395880F08F045
:10C510009927EE0F979587950895D9D008F481E073
:10C5200008950CD00FC107D140F0FED030F021F4B7
:10C530005F3F19F0F0C0511139C1F3C014D198F325
:10C540009923C9F35523B1F3951B550BBB27AA2794
:10C5500062177307840738F09F5F5F4F220F331F06
:10C56000441FAA1FA9F333D00E2E3AF0E0E830D0D2
:10C5700091505040E695001CCAF729D0FE2F27D0D5
:10C58000660F771F881FBB1F261737074807AB07A3
:10C59000B0E809F0BB0B802DBF01FF2793585F4F18
:10C5A0002AF09E3F510568F0B6C000C15F3FECF332
:10C5B000983EDCF3869577956795B795F7959F5FDD
:10C5C000C9F7880F911D9695879597F90895E1E031
:10C5D000660F771F881FBB1F621773078407BA0790
:10C5E00020F0621B730B840BBA0BEE1F88F7E095EB
:10C5F000089504D06894B111D9C00895BCD088F0D2
:10C600009F5790F0B92F9927B751A0F0D1F0660F3E
:10C61000771F881F991F1AF0BA95C9F712C0B13059
:10C6200081F0C3D0B1E00895C0C0672F782F88276C
:10C63000B85F39F0B93FCCF3869577956795B39598
:10C64000D9F73EF490958095709561957F4F8F4F07
:10C650009F4F0895E89409C097FB3EF4909580950C
:10C66000709561957F4F8F4F9F4F9923A9F0F92FB8
:10C6700096E9BB279395F695879577956795B79536
:10C68000F111F8CFFAF4BB0F11F460FF1BC06F5F1C
:10C690007F4F8F4F9F4F16C0882311F096E911C02E
:10C6A000772321F09EE8872F762F05C0662371F04F
:10C6B00096E8862F70E060E02AF09A95660F771F63
:10C6C000881FDAF7880F9695879597F90895990F3F
:10C6D0000008550FAA0BE0E8FEEF16161706E8074C
:10C6E000F907C0F012161306E407F50798F0621B6D
:10C6F000730B840B950B39F40A2661F0232B242B42
:10C70000252B21F408950A2609F4A140A6958FEF60
:10C71000811D811D089597F99F6780E870E060E0B2
:10C7200008959FEF80EC089500240A9416161706CA
:10C7300018060906089500240A9412161306140612
:10C7400005060895092E0394000C11F4882352F075
:10C75000BB0F40F4BF2B11F460FF04C06F5F7F4F2D
:10C760008F4F9F4F089557FD9058440F551F59F014
:10C770005F3F71F04795880F97FB991F61F09F3FCE
:10C7800079F087950895121613061406551FF2CFF7
:10C790004695F1DF08C0161617061806991FF1CF47
:10C7A00086957105610508940895E894BB2766276E
:10C7B0007727CB0197F908958ADF08F48FEF089562
:10C7C0000BD0C0CFB1DF28F0B6DF18F0952309F009
:10C7D000A2CFA7CF1124EACFC6DFA0F3959FD1F354
:10C7E000950F50E0551F629FF001729FBB27F00D1F
:10C7F000B11D639FAA27F00DB11DAA1F649F662774
:10C80000B00DA11D661F829F2227B00DA11D621FC2
:10C81000739FB00DA11D621F839FA00D611D221F7C
:10C82000749F3327A00D611D231F849F600D211D60
:10C83000822F762F6A2F11249F5750408AF0E1F003
:10C8400088234AF0EE0FFF1FBB1F661F771F881F4C
:10C8500091505040A9F79E3F510570F05CCFA6CF94
:10C860005F3FECF3983EDCF3869577956795B79537
:10C87000F795E7959F5FC1F7FE2B880F911D969561
:10C88000879597F90895FA01EE0FFF1F309621055D
:10C89000310599F16115710561F48038BFE39B079B
:10C8A00049F168949038810561F08038BFEF9B07AB
:10C8B00041F0992342F5FF3FE1053105210511F1D2
:10C8C000E8940894E795D901AA2329F4AB2FBE2F49
:10C8D000F85FD0F310C0FF5F70F4A695E0F7F7396A
:10C8E00050F019F0FF3A38F49F779F930CD00F90D7
:10C8F00007FC905808953EF014CF60E070E080E8A7
:10C900009FE308954FE79F775F934F933F932F9354
:10C910009ED02F913F914F915F9152DF05C019F446
:10C920000EF0F9CE42CFFDCE26DFC8F39638C0F721
:10C9300007F80F92E8942BE33AEA48EB5FE74EDF03
:10C940000F920F920F924DB75EB70F92C0D0E4ECEA
:10C95000F1E016D04F915F91EF91FF91E595EE1FB9
:10C96000FF1F49F0FE57E0684427EE0F441FFA9579
:10C97000E1F74195550B32D00F9007FE26C0089580
:10C98000DF93CF931F930F93FF92EF92DF927B0180
:10C990008C01689405C0DA2EEF011EDFFE01E894D9
:10C9A000A5912591359145915591AEF3EF0162DD49
:10C9B000FE019701A801DA9479F7DF90EF90FF90DC
:10C9C0000F911F91CF91DF9108959B01AC0160E021
:10C9D00070E080E89FE3A5CD9ECEACC0CCDEE8F34E
:10C9E0009923D9F3940F511DBBF39150504094F00B
:10C9F00059F0882332F0660F771F881F91505040FE
:10CA0000C1F79E3F510544F7880F911D9695879574
:10CA100097F908955F3FACF0983E9CF0BB27869550
:10CA200077956795B79508F4B1609395C1F7BB0FFB
:10CA300058F711F460FFE8CF6F5F7F4F8F4F9F4F24
:10CA4000E3CFB4CE0EF076C06CCE689464CE93DEA5
:10CA5000C8F39923D1F3C6F3DF93CF931F930F93BA
:10CA6000FF92C92FDD2788232AF02197660F771FB1
:10CA7000881FDAF720E030E040E85FEB9FE3883979
:10CA800020F0803E30F021968F77E3DCECEEF1E091
:10CA900003C0DFDCE9E1F2E073DF8B01BE01EC01F2
:10CAA000FB2E6F5771097595771F880B990BD4DD95
:10CAB00028E132E741E35FE38FDEAF2D9801AE015D
:10CAC000FF900F911F91CF91DF91D4DC3BCEFA0103
:10CAD000DC01AA0FBB1F9B01AC01BF5728F4222722
:10CAE0003327442750781FC0B75188F4AB2F002458
:10CAF000469537952795011CA395D2F3002069F040
:10CB0000220F331F441FB395DAF30DD0A1CC61304F
:10CB10007105A0E88A07B94630F49B01AC0166278D
:10CB2000772788279078309621F0208331834283BD
:10CB3000538308959F3F31F0915020F48795779566
:10CB40006795B795880F911D9695879597F90895E4
:10CB500097FB072E16F4009406D077FD08D020D05E
:10CB600007FC05D03EF4909581959F4F08957095F0
:10CB700061957F4F0895EE0FFF1F881F8BBF0790B1
:10CB8000F691E02D1994692796276927782787273A
:10CB9000782708954EDCB7FF0895821B930B089504
:10CBA000AA1BBB1B51E107C0AA1FBB1FA617B707D3
:10CBB00010F0A61BB70B881F991F5A95A9F78095EF
:10CBC0009095BC01CD01089581E090E0F89425C1D5
:10CBD0000F931F93CF93DF938C01FC0101900020F2
:10CBE000E9F7CF01801B910B0E945659EC01009789
:10CBF00011F0B80145D0CE01DF91CF911F910F9177
:10CC00000895FB01DC0104C08D910190801921F48D
:10CC100041505040C8F7881B990B0895FB01DC0177
:10CC20008D9181341CF08B350CF4805E6191613400
:10CC30001CF06B350CF4605E861B611189F3990B57
:10CC40000895FB01DC010D900020E9F71197019098
:10CC50000D920020E1F70895FC018191861721F0E3
:10CC60008823D9F7992708953197CF010895FB01BB
:10CC7000DC018D91019080190110D9F3990B089571
:10CC8000FB01DC0101900D920020E1F70895FB010A
:10CC9000DC010D900020E9F711974150504028F039
:10CCA000019000200D92C9F708951C920895FB0190
:10CCB000DC014150504030F08D910190801919F401
:10CCC0000020B9F7881B990B0895FB01DC01415046
:10CCD000504048F001900D920020C9F701C01D920C
:10CCE00041505040E0F70895FC0181E090E0019050
:10CCF000061609F4CF010020D1F7019708950F938C
:10CD00001F93CF93DF93CDB7DEB72E970FB6F8946E
:10CD1000DEBF0FBECDBF0E891F89888D998D26E09D
:10CD20002C831A83098397FF02C080E090E8019763
:10CD30009E838D83AE01445E5F4F6A8D7B8DCE01F5
:10CD400001960E940C5C4D815E8157FD0AC02F81C7
:10CD50003885421753070CF49A01F801E20FF31FCC
:10CD600010822E960FB6F894DEBF0FBECDBFDF91B6
:10CD7000CF911F910F9108950F931F93CF93DF933E
:10CD8000CDB7DEB72E970FB6F894DEBF0FBECDBF7E
:10CD90000E891F8986E08C831A8309838FEF9FE7B2
:10CDA0009E838D83AE01465E5F4F688D798DCE0187
:10CDB00001960E940C5C2F813885F801E20FF31F69
:10CDC00010822E960FB6F894DEBF0FBECDBFDF9156
:10CDD000CF911F910F910895CF93DF93CDB7DEB719
:10CDE0002E970FB6F894DEBF0FBECDBF85E08C83C3
:10CDF0008C899D899A838983AE01485E5F4F6E89D5
:10CE00007F89CE0101969DD82E960FB6F894DEBF8D
:0ECE10000FBECDBFDF91CF910895F894FFCFF4
:10CE1E0003100001200000C00000900B80000100F4
:10CE2E000000DEADBEEFFE005E00BC00770100002C
:10CE3E0000006107000000000000000001005E001D
:10CE4E0000004172742D4E6574000000044D515463
:10CE5E005404000000001B0F07139F47AC355A0FF8
:10CE6E00380F680FD60F111000000000930F071334
:10CE7E009F47AC35DD0F5A10680FD60F111000000A
:10CE8E000000702664279F4715108626BB267C114E
:10CE9E00B1277B129C27F4281B28B2280B270512DA
:10CEAE009E268E268A26303132333435363738393F
:10CEBE004142434445460000000000BB1307134B9C
:10CECE001301147C135A136E13000000005A312BF9
:10CEDE00319F47FF3023310F31003100000000F940
:10CEEE0014F9149F47F914F914F914F914F914F9F3
:10CEFE0014F914F914F914F91400000000F91407C8
:10CF0E00139F479E47F914F914F91400000000F915
:10CF1E001407139F479E4700000000D94272439F9B
:10CF2E0047BA260227E826DE27E143FE42E4265EC4
:10CF3E00293B29B226FB42F942A726EF4200000008
:10CF4E0000D01500000000F91400000000161007B4
:10CF5E00139F47AC35AB0F2D10680FD60F11100075
:10CF6E00000000D94272439F47BA260227E826DE08
:10CF7E0027E143FE42E4265E293B29B226FB42F915
:10CF8E0042A726EF4200000000930F07139F47AC05
:10CF9E0035DD0F4A10680FD60F111068656C7000E2
:10CFAE0073617665006C6F6164006765740073650C
:10CFBE0074006B696C6C00726571000D0A005F7312
:10CFCE0074617400560052504D004900737700662C
:10CFDE006C7400707772002F616C61726D0053007B
:10CFEE00496E3A20002F003D006974656D00736331
:10CFFE006D640072636D6400656D6974004F4E0060
:10D00E004F4646005245535400544F47474C450037
:10D01E0048414C54003B002F6D79686F6D652F6F42
:10D02E0075742F526573746F7265537461746500F5
:10D03E002F6D79686F6D652F696E2F230057495AD2
:10D04E006E65740031772054696D656F757400528A
:10D05E0065736574206572726F720020636F6D70F8
:10D06E005F6964210022002525253278006E756CDB
:10D07E006C00747275650066616C7365002D002E10
:10D08E0000646D7800646D78696E006974656D7307
:10D09E00006D6F64627573006D717474006F77004C
:10D0AE0025783A25783A25783A25783A25783A251A
:10D0BE007825D181002F726573702F23002F726532
:10D0CE00712F636F6E660031002F253032782D255B
:10D0DE003032782D253032782D253032782D25308E
:10D0EE0032782D253032782E636F6E6669672E6A20
:10D0FE00736F6E003139322E3136382E38382E326B
:10D10E00005D20006F6E20536B69707065640025A2
:0ED11E0064002C002F616C61726D6F666600FC
:00000001FF
